Archive member included to satisfy reference by file (symbol)

c:/renesas/ra/e2studio_v2023-07_fsp_v4.6.0/toolchains/gcc_arm/arm-gnu-toolchain-12.2.mpacbti-rel1-mingw-w64-i686-arm-none-eabi/bin/../lib/gcc/arm-none-eabi/12.2.1/thumb/v8-m.main+fp/hard\libgcc.a(_arm_muldf3.o)
                              ./src/adc_temp.o (__aeabi_dmul)
c:/renesas/ra/e2studio_v2023-07_fsp_v4.6.0/toolchains/gcc_arm/arm-gnu-toolchain-12.2.mpacbti-rel1-mingw-w64-i686-arm-none-eabi/bin/../lib/gcc/arm-none-eabi/12.2.1/thumb/v8-m.main+fp/hard\libgcc.a(_arm_addsubdf3.o)
                              ./src/adc_temp.o (__aeabi_dsub)
c:/renesas/ra/e2studio_v2023-07_fsp_v4.6.0/toolchains/gcc_arm/arm-gnu-toolchain-12.2.mpacbti-rel1-mingw-w64-i686-arm-none-eabi/bin/../lib/gcc/arm-none-eabi/12.2.1/thumb/v8-m.main+fp/hard\libgcc.a(_arm_muldivdf3.o)
                              ./src/adc_temp.o (__aeabi_ddiv)
c:/renesas/ra/e2studio_v2023-07_fsp_v4.6.0/toolchains/gcc_arm/arm-gnu-toolchain-12.2.mpacbti-rel1-mingw-w64-i686-arm-none-eabi/bin/../lib/gcc/arm-none-eabi/12.2.1/thumb/v8-m.main+fp/hard\libgcc.a(_arm_cmpdf2.o)
                              ./src/usart.o (__aeabi_dcmpeq)
c:/renesas/ra/e2studio_v2023-07_fsp_v4.6.0/toolchains/gcc_arm/arm-gnu-toolchain-12.2.mpacbti-rel1-mingw-w64-i686-arm-none-eabi/bin/../lib/gcc/arm-none-eabi/12.2.1/thumb/v8-m.main+fp/hard\libgcc.a(_arm_unorddf2.o)
                              ./src/usart.o (__aeabi_dcmpun)
c:/renesas/ra/e2studio_v2023-07_fsp_v4.6.0/toolchains/gcc_arm/arm-gnu-toolchain-12.2.mpacbti-rel1-mingw-w64-i686-arm-none-eabi/bin/../lib/gcc/arm-none-eabi/12.2.1/thumb/v8-m.main+fp/hard\libgcc.a(_arm_fixdfsi.o)
                              ./src/adc_temp.o (__aeabi_d2iz)
c:/renesas/ra/e2studio_v2023-07_fsp_v4.6.0/toolchains/gcc_arm/arm-gnu-toolchain-12.2.mpacbti-rel1-mingw-w64-i686-arm-none-eabi/bin/../lib/gcc/arm-none-eabi/12.2.1/thumb/v8-m.main+fp/hard\libgcc.a(_arm_fixunsdfsi.o)
                              ./src/hal_entry.o (__aeabi_d2uiz)
c:/renesas/ra/e2studio_v2023-07_fsp_v4.6.0/toolchains/gcc_arm/arm-gnu-toolchain-12.2.mpacbti-rel1-mingw-w64-i686-arm-none-eabi/bin/../lib/gcc/arm-none-eabi/12.2.1/thumb/v8-m.main+fp/hard\libgcc.a(_aeabi_ldivmod.o)
                              ./ra/fsp/src/r_sci_uart/r_sci_uart.o (__aeabi_ldivmod)
c:/renesas/ra/e2studio_v2023-07_fsp_v4.6.0/toolchains/gcc_arm/arm-gnu-toolchain-12.2.mpacbti-rel1-mingw-w64-i686-arm-none-eabi/bin/../lib/gcc/arm-none-eabi/12.2.1/thumb/v8-m.main+fp/hard\libgcc.a(_udivmoddi4.o)
                              c:/renesas/ra/e2studio_v2023-07_fsp_v4.6.0/toolchains/gcc_arm/arm-gnu-toolchain-12.2.mpacbti-rel1-mingw-w64-i686-arm-none-eabi/bin/../lib/gcc/arm-none-eabi/12.2.1/thumb/v8-m.main+fp/hard\libgcc.a(_aeabi_ldivmod.o) (__udivmoddi4)
c:/renesas/ra/e2studio_v2023-07_fsp_v4.6.0/toolchains/gcc_arm/arm-gnu-toolchain-12.2.mpacbti-rel1-mingw-w64-i686-arm-none-eabi/bin/../lib/gcc/arm-none-eabi/12.2.1/thumb/v8-m.main+fp/hard\libgcc.a(_dvmd_tls.o)
                              c:/renesas/ra/e2studio_v2023-07_fsp_v4.6.0/toolchains/gcc_arm/arm-gnu-toolchain-12.2.mpacbti-rel1-mingw-w64-i686-arm-none-eabi/bin/../lib/gcc/arm-none-eabi/12.2.1/thumb/v8-m.main+fp/hard\libgcc.a(_aeabi_ldivmod.o) (__aeabi_ldiv0)
c:/renesas/ra/e2studio_v2023-07_fsp_v4.6.0/toolchains/gcc_arm/arm-gnu-toolchain-12.2.mpacbti-rel1-mingw-w64-i686-arm-none-eabi/bin/../lib/gcc/arm-none-eabi/12.2.1/thumb/v8-m.main+fp/hard\libg_nano.a(libc_a-exit.o)
                              c:/renesas/ra/e2studio_v2023-07_fsp_v4.6.0/toolchains/gcc_arm/arm-gnu-toolchain-12.2.mpacbti-rel1-mingw-w64-i686-arm-none-eabi/bin/../lib/gcc/arm-none-eabi/12.2.1/thumb/v8-m.main+fp/hard/rdimon-crt0.o (exit)
c:/renesas/ra/e2studio_v2023-07_fsp_v4.6.0/toolchains/gcc_arm/arm-gnu-toolchain-12.2.mpacbti-rel1-mingw-w64-i686-arm-none-eabi/bin/../lib/gcc/arm-none-eabi/12.2.1/thumb/v8-m.main+fp/hard\libg_nano.a(libc_a-itoa.o)
                              ./src/packet.o (__itoa)
c:/renesas/ra/e2studio_v2023-07_fsp_v4.6.0/toolchains/gcc_arm/arm-gnu-toolchain-12.2.mpacbti-rel1-mingw-w64-i686-arm-none-eabi/bin/../lib/gcc/arm-none-eabi/12.2.1/thumb/v8-m.main+fp/hard\libg_nano.a(libc_a-strtol.o)
                              ./src/packet.o (strtol)
c:/renesas/ra/e2studio_v2023-07_fsp_v4.6.0/toolchains/gcc_arm/arm-gnu-toolchain-12.2.mpacbti-rel1-mingw-w64-i686-arm-none-eabi/bin/../lib/gcc/arm-none-eabi/12.2.1/thumb/v8-m.main+fp/hard\libg_nano.a(libc_a-utoa.o)
                              ./src/packet.o (__utoa)
c:/renesas/ra/e2studio_v2023-07_fsp_v4.6.0/toolchains/gcc_arm/arm-gnu-toolchain-12.2.mpacbti-rel1-mingw-w64-i686-arm-none-eabi/bin/../lib/gcc/arm-none-eabi/12.2.1/thumb/v8-m.main+fp/hard\libg_nano.a(libc_a-ctype_.o)
                              c:/renesas/ra/e2studio_v2023-07_fsp_v4.6.0/toolchains/gcc_arm/arm-gnu-toolchain-12.2.mpacbti-rel1-mingw-w64-i686-arm-none-eabi/bin/../lib/gcc/arm-none-eabi/12.2.1/thumb/v8-m.main+fp/hard\libg_nano.a(libc_a-strtol.o) (_ctype_)
c:/renesas/ra/e2studio_v2023-07_fsp_v4.6.0/toolchains/gcc_arm/arm-gnu-toolchain-12.2.mpacbti-rel1-mingw-w64-i686-arm-none-eabi/bin/../lib/gcc/arm-none-eabi/12.2.1/thumb/v8-m.main+fp/hard\libg_nano.a(libc_a-findfp.o)
                              c:/renesas/ra/e2studio_v2023-07_fsp_v4.6.0/toolchains/gcc_arm/arm-gnu-toolchain-12.2.mpacbti-rel1-mingw-w64-i686-arm-none-eabi/bin/../lib/gcc/arm-none-eabi/12.2.1/thumb/v8-m.main+fp/hard\libg_nano.a(libc_a-exit.o) (__stdio_exit_handler)
c:/renesas/ra/e2studio_v2023-07_fsp_v4.6.0/toolchains/gcc_arm/arm-gnu-toolchain-12.2.mpacbti-rel1-mingw-w64-i686-arm-none-eabi/bin/../lib/gcc/arm-none-eabi/12.2.1/thumb/v8-m.main+fp/hard\libg_nano.a(libc_a-fwalk.o)
                              c:/renesas/ra/e2studio_v2023-07_fsp_v4.6.0/toolchains/gcc_arm/arm-gnu-toolchain-12.2.mpacbti-rel1-mingw-w64-i686-arm-none-eabi/bin/../lib/gcc/arm-none-eabi/12.2.1/thumb/v8-m.main+fp/hard\libg_nano.a(libc_a-findfp.o) (_fwalk_sglue)
c:/renesas/ra/e2studio_v2023-07_fsp_v4.6.0/toolchains/gcc_arm/arm-gnu-toolchain-12.2.mpacbti-rel1-mingw-w64-i686-arm-none-eabi/bin/../lib/gcc/arm-none-eabi/12.2.1/thumb/v8-m.main+fp/hard\libg_nano.a(libc_a-stdio.o)
                              c:/renesas/ra/e2studio_v2023-07_fsp_v4.6.0/toolchains/gcc_arm/arm-gnu-toolchain-12.2.mpacbti-rel1-mingw-w64-i686-arm-none-eabi/bin/../lib/gcc/arm-none-eabi/12.2.1/thumb/v8-m.main+fp/hard\libg_nano.a(libc_a-findfp.o) (__sread)
c:/renesas/ra/e2studio_v2023-07_fsp_v4.6.0/toolchains/gcc_arm/arm-gnu-toolchain-12.2.mpacbti-rel1-mingw-w64-i686-arm-none-eabi/bin/../lib/gcc/arm-none-eabi/12.2.1/thumb/v8-m.main+fp/hard\libg_nano.a(libc_a-memset.o)
                              c:/renesas/ra/e2studio_v2023-07_fsp_v4.6.0/toolchains/gcc_arm/arm-gnu-toolchain-12.2.mpacbti-rel1-mingw-w64-i686-arm-none-eabi/bin/../lib/gcc/arm-none-eabi/12.2.1/thumb/v8-m.main+fp/hard/rdimon-crt0.o (memset)
c:/renesas/ra/e2studio_v2023-07_fsp_v4.6.0/toolchains/gcc_arm/arm-gnu-toolchain-12.2.mpacbti-rel1-mingw-w64-i686-arm-none-eabi/bin/../lib/gcc/arm-none-eabi/12.2.1/thumb/v8-m.main+fp/hard\libg_nano.a(libc_a-strncmp.o)
                              ./src/packet.o (strncmp)
c:/renesas/ra/e2studio_v2023-07_fsp_v4.6.0/toolchains/gcc_arm/arm-gnu-toolchain-12.2.mpacbti-rel1-mingw-w64-i686-arm-none-eabi/bin/../lib/gcc/arm-none-eabi/12.2.1/thumb/v8-m.main+fp/hard\libg_nano.a(libc_a-closer.o)
                              c:/renesas/ra/e2studio_v2023-07_fsp_v4.6.0/toolchains/gcc_arm/arm-gnu-toolchain-12.2.mpacbti-rel1-mingw-w64-i686-arm-none-eabi/bin/../lib/gcc/arm-none-eabi/12.2.1/thumb/v8-m.main+fp/hard\libg_nano.a(libc_a-stdio.o) (_close_r)
c:/renesas/ra/e2studio_v2023-07_fsp_v4.6.0/toolchains/gcc_arm/arm-gnu-toolchain-12.2.mpacbti-rel1-mingw-w64-i686-arm-none-eabi/bin/../lib/gcc/arm-none-eabi/12.2.1/thumb/v8-m.main+fp/hard\libg_nano.a(libc_a-reent.o)
                              c:/renesas/ra/e2studio_v2023-07_fsp_v4.6.0/toolchains/gcc_arm/arm-gnu-toolchain-12.2.mpacbti-rel1-mingw-w64-i686-arm-none-eabi/bin/../lib/gcc/arm-none-eabi/12.2.1/thumb/v8-m.main+fp/hard\libg_nano.a(libc_a-closer.o) (errno)
c:/renesas/ra/e2studio_v2023-07_fsp_v4.6.0/toolchains/gcc_arm/arm-gnu-toolchain-12.2.mpacbti-rel1-mingw-w64-i686-arm-none-eabi/bin/../lib/gcc/arm-none-eabi/12.2.1/thumb/v8-m.main+fp/hard\libg_nano.a(libc_a-impure.o)
                              c:/renesas/ra/e2studio_v2023-07_fsp_v4.6.0/toolchains/gcc_arm/arm-gnu-toolchain-12.2.mpacbti-rel1-mingw-w64-i686-arm-none-eabi/bin/../lib/gcc/arm-none-eabi/12.2.1/thumb/v8-m.main+fp/hard\libg_nano.a(libc_a-strtol.o) (_impure_ptr)
c:/renesas/ra/e2studio_v2023-07_fsp_v4.6.0/toolchains/gcc_arm/arm-gnu-toolchain-12.2.mpacbti-rel1-mingw-w64-i686-arm-none-eabi/bin/../lib/gcc/arm-none-eabi/12.2.1/thumb/v8-m.main+fp/hard\libg_nano.a(libc_a-lseekr.o)
                              c:/renesas/ra/e2studio_v2023-07_fsp_v4.6.0/toolchains/gcc_arm/arm-gnu-toolchain-12.2.mpacbti-rel1-mingw-w64-i686-arm-none-eabi/bin/../lib/gcc/arm-none-eabi/12.2.1/thumb/v8-m.main+fp/hard\libg_nano.a(libc_a-stdio.o) (_lseek_r)
c:/renesas/ra/e2studio_v2023-07_fsp_v4.6.0/toolchains/gcc_arm/arm-gnu-toolchain-12.2.mpacbti-rel1-mingw-w64-i686-arm-none-eabi/bin/../lib/gcc/arm-none-eabi/12.2.1/thumb/v8-m.main+fp/hard\libg_nano.a(libc_a-readr.o)
                              c:/renesas/ra/e2studio_v2023-07_fsp_v4.6.0/toolchains/gcc_arm/arm-gnu-toolchain-12.2.mpacbti-rel1-mingw-w64-i686-arm-none-eabi/bin/../lib/gcc/arm-none-eabi/12.2.1/thumb/v8-m.main+fp/hard\libg_nano.a(libc_a-stdio.o) (_read_r)
c:/renesas/ra/e2studio_v2023-07_fsp_v4.6.0/toolchains/gcc_arm/arm-gnu-toolchain-12.2.mpacbti-rel1-mingw-w64-i686-arm-none-eabi/bin/../lib/gcc/arm-none-eabi/12.2.1/thumb/v8-m.main+fp/hard\libg_nano.a(libc_a-writer.o)
                              c:/renesas/ra/e2studio_v2023-07_fsp_v4.6.0/toolchains/gcc_arm/arm-gnu-toolchain-12.2.mpacbti-rel1-mingw-w64-i686-arm-none-eabi/bin/../lib/gcc/arm-none-eabi/12.2.1/thumb/v8-m.main+fp/hard\libg_nano.a(libc_a-stdio.o) (_write_r)
c:/renesas/ra/e2studio_v2023-07_fsp_v4.6.0/toolchains/gcc_arm/arm-gnu-toolchain-12.2.mpacbti-rel1-mingw-w64-i686-arm-none-eabi/bin/../lib/gcc/arm-none-eabi/12.2.1/thumb/v8-m.main+fp/hard\libg_nano.a(libc_a-errno.o)
                              ./ra/fsp/src/bsp/mcu/all/bsp_sbrk.o (__errno)
c:/renesas/ra/e2studio_v2023-07_fsp_v4.6.0/toolchains/gcc_arm/arm-gnu-toolchain-12.2.mpacbti-rel1-mingw-w64-i686-arm-none-eabi/bin/../lib/gcc/arm-none-eabi/12.2.1/thumb/v8-m.main+fp/hard\libg_nano.a(libc_a-init.o)
                              c:/renesas/ra/e2studio_v2023-07_fsp_v4.6.0/toolchains/gcc_arm/arm-gnu-toolchain-12.2.mpacbti-rel1-mingw-w64-i686-arm-none-eabi/bin/../lib/gcc/arm-none-eabi/12.2.1/thumb/v8-m.main+fp/hard/rdimon-crt0.o (__libc_init_array)
c:/renesas/ra/e2studio_v2023-07_fsp_v4.6.0/toolchains/gcc_arm/arm-gnu-toolchain-12.2.mpacbti-rel1-mingw-w64-i686-arm-none-eabi/bin/../lib/gcc/arm-none-eabi/12.2.1/thumb/v8-m.main+fp/hard\libg_nano.a(libc_a-lock.o)
                              c:/renesas/ra/e2studio_v2023-07_fsp_v4.6.0/toolchains/gcc_arm/arm-gnu-toolchain-12.2.mpacbti-rel1-mingw-w64-i686-arm-none-eabi/bin/../lib/gcc/arm-none-eabi/12.2.1/thumb/v8-m.main+fp/hard\libg_nano.a(libc_a-findfp.o) (__retarget_lock_init_recursive)
c:/renesas/ra/e2studio_v2023-07_fsp_v4.6.0/toolchains/gcc_arm/arm-gnu-toolchain-12.2.mpacbti-rel1-mingw-w64-i686-arm-none-eabi/bin/../lib/gcc/arm-none-eabi/12.2.1/thumb/v8-m.main+fp/hard\libg_nano.a(libc_a-strcpy.o)
                              ./src/packet.o (strcpy)
c:/renesas/ra/e2studio_v2023-07_fsp_v4.6.0/toolchains/gcc_arm/arm-gnu-toolchain-12.2.mpacbti-rel1-mingw-w64-i686-arm-none-eabi/bin/../lib/gcc/arm-none-eabi/12.2.1/thumb/v8-m.main+fp/hard\libg_nano.a(libc_a-aeabi_memcpy.o)
                              ./src/usart.o (__aeabi_memcpy4)
c:/renesas/ra/e2studio_v2023-07_fsp_v4.6.0/toolchains/gcc_arm/arm-gnu-toolchain-12.2.mpacbti-rel1-mingw-w64-i686-arm-none-eabi/bin/../lib/gcc/arm-none-eabi/12.2.1/thumb/v8-m.main+fp/hard\libg_nano.a(libc_a-aeabi_memclr.o)
                              ./src/packet.o (__aeabi_memclr8)
c:/renesas/ra/e2studio_v2023-07_fsp_v4.6.0/toolchains/gcc_arm/arm-gnu-toolchain-12.2.mpacbti-rel1-mingw-w64-i686-arm-none-eabi/bin/../lib/gcc/arm-none-eabi/12.2.1/thumb/v8-m.main+fp/hard\libg_nano.a(libc_a-memcpy-stub.o)
                              ./src/angle.o (memcpy)
c:/renesas/ra/e2studio_v2023-07_fsp_v4.6.0/toolchains/gcc_arm/arm-gnu-toolchain-12.2.mpacbti-rel1-mingw-w64-i686-arm-none-eabi/bin/../lib/gcc/arm-none-eabi/12.2.1/thumb/v8-m.main+fp/hard\libg_nano.a(libc_a-strlen.o)
                              ./src/packet.o (strlen)
c:/renesas/ra/e2studio_v2023-07_fsp_v4.6.0/toolchains/gcc_arm/arm-gnu-toolchain-12.2.mpacbti-rel1-mingw-w64-i686-arm-none-eabi/bin/../lib/gcc/arm-none-eabi/12.2.1/thumb/v8-m.main+fp/hard\libg_nano.a(libc_a-freer.o)
                              c:/renesas/ra/e2studio_v2023-07_fsp_v4.6.0/toolchains/gcc_arm/arm-gnu-toolchain-12.2.mpacbti-rel1-mingw-w64-i686-arm-none-eabi/bin/../lib/gcc/arm-none-eabi/12.2.1/thumb/v8-m.main+fp/hard\libg_nano.a(libc_a-reent.o) (_free_r)
c:/renesas/ra/e2studio_v2023-07_fsp_v4.6.0/toolchains/gcc_arm/arm-gnu-toolchain-12.2.mpacbti-rel1-mingw-w64-i686-arm-none-eabi/bin/../lib/gcc/arm-none-eabi/12.2.1/thumb/v8-m.main+fp/hard\libg_nano.a(libc_a-mallocr.o)
                              c:/renesas/ra/e2studio_v2023-07_fsp_v4.6.0/toolchains/gcc_arm/arm-gnu-toolchain-12.2.mpacbti-rel1-mingw-w64-i686-arm-none-eabi/bin/../lib/gcc/arm-none-eabi/12.2.1/thumb/v8-m.main+fp/hard\libg_nano.a(libc_a-findfp.o) (_malloc_r)
c:/renesas/ra/e2studio_v2023-07_fsp_v4.6.0/toolchains/gcc_arm/arm-gnu-toolchain-12.2.mpacbti-rel1-mingw-w64-i686-arm-none-eabi/bin/../lib/gcc/arm-none-eabi/12.2.1/thumb/v8-m.main+fp/hard\libg_nano.a(libc_a-mlock.o)
                              c:/renesas/ra/e2studio_v2023-07_fsp_v4.6.0/toolchains/gcc_arm/arm-gnu-toolchain-12.2.mpacbti-rel1-mingw-w64-i686-arm-none-eabi/bin/../lib/gcc/arm-none-eabi/12.2.1/thumb/v8-m.main+fp/hard\libg_nano.a(libc_a-freer.o) (__malloc_lock)
c:/renesas/ra/e2studio_v2023-07_fsp_v4.6.0/toolchains/gcc_arm/arm-gnu-toolchain-12.2.mpacbti-rel1-mingw-w64-i686-arm-none-eabi/bin/../lib/gcc/arm-none-eabi/12.2.1/thumb/v8-m.main+fp/hard\libg_nano.a(libc_a-fflush.o)
                              c:/renesas/ra/e2studio_v2023-07_fsp_v4.6.0/toolchains/gcc_arm/arm-gnu-toolchain-12.2.mpacbti-rel1-mingw-w64-i686-arm-none-eabi/bin/../lib/gcc/arm-none-eabi/12.2.1/thumb/v8-m.main+fp/hard\libg_nano.a(libc_a-findfp.o) (_fflush_r)
c:/renesas/ra/e2studio_v2023-07_fsp_v4.6.0/toolchains/gcc_arm/arm-gnu-toolchain-12.2.mpacbti-rel1-mingw-w64-i686-arm-none-eabi/bin/../lib/gcc/arm-none-eabi/12.2.1/thumb/v8-m.main+fp/hard\libg_nano.a(libc_a-sbrkr.o)
                              c:/renesas/ra/e2studio_v2023-07_fsp_v4.6.0/toolchains/gcc_arm/arm-gnu-toolchain-12.2.mpacbti-rel1-mingw-w64-i686-arm-none-eabi/bin/../lib/gcc/arm-none-eabi/12.2.1/thumb/v8-m.main+fp/hard\libg_nano.a(libc_a-mallocr.o) (_sbrk_r)
c:/renesas/ra/e2studio_v2023-07_fsp_v4.6.0/toolchains/gcc_arm/arm-gnu-toolchain-12.2.mpacbti-rel1-mingw-w64-i686-arm-none-eabi/bin/../lib/gcc/arm-none-eabi/12.2.1/thumb/v8-m.main+fp/hard\libg_nano.a(libc_a-aeabi_memset-soft.o)
                              c:/renesas/ra/e2studio_v2023-07_fsp_v4.6.0/toolchains/gcc_arm/arm-gnu-toolchain-12.2.mpacbti-rel1-mingw-w64-i686-arm-none-eabi/bin/../lib/gcc/arm-none-eabi/12.2.1/thumb/v8-m.main+fp/hard\libg_nano.a(libc_a-aeabi_memclr.o) (__aeabi_memset)
c:/renesas/ra/e2studio_v2023-07_fsp_v4.6.0/toolchains/gcc_arm/arm-gnu-toolchain-12.2.mpacbti-rel1-mingw-w64-i686-arm-none-eabi/bin/../lib/gcc/arm-none-eabi/12.2.1/thumb/v8-m.main+fp/hard\librdimon_nano.a(arm_librdimon_a-_exit.o)
                              c:/renesas/ra/e2studio_v2023-07_fsp_v4.6.0/toolchains/gcc_arm/arm-gnu-toolchain-12.2.mpacbti-rel1-mingw-w64-i686-arm-none-eabi/bin/../lib/gcc/arm-none-eabi/12.2.1/thumb/v8-m.main+fp/hard\libg_nano.a(libc_a-exit.o) (_exit)
c:/renesas/ra/e2studio_v2023-07_fsp_v4.6.0/toolchains/gcc_arm/arm-gnu-toolchain-12.2.mpacbti-rel1-mingw-w64-i686-arm-none-eabi/bin/../lib/gcc/arm-none-eabi/12.2.1/thumb/v8-m.main+fp/hard\librdimon_nano.a(arm_librdimon_a-_kill.o)
                              c:/renesas/ra/e2studio_v2023-07_fsp_v4.6.0/toolchains/gcc_arm/arm-gnu-toolchain-12.2.mpacbti-rel1-mingw-w64-i686-arm-none-eabi/bin/../lib/gcc/arm-none-eabi/12.2.1/thumb/v8-m.main+fp/hard\librdimon_nano.a(arm_librdimon_a-_exit.o) (_kill_shared)
c:/renesas/ra/e2studio_v2023-07_fsp_v4.6.0/toolchains/gcc_arm/arm-gnu-toolchain-12.2.mpacbti-rel1-mingw-w64-i686-arm-none-eabi/bin/../lib/gcc/arm-none-eabi/12.2.1/thumb/v8-m.main+fp/hard\librdimon_nano.a(arm_librdimon_a-syscalls.o)
                              c:/renesas/ra/e2studio_v2023-07_fsp_v4.6.0/toolchains/gcc_arm/arm-gnu-toolchain-12.2.mpacbti-rel1-mingw-w64-i686-arm-none-eabi/bin/../lib/gcc/arm-none-eabi/12.2.1/thumb/v8-m.main+fp/hard\libg_nano.a(libc_a-readr.o) (_read)

Discarded input sections

 .text          0x00000000        0x0 c:/renesas/ra/e2studio_v2023-07_fsp_v4.6.0/toolchains/gcc_arm/arm-gnu-toolchain-12.2.mpacbti-rel1-mingw-w64-i686-arm-none-eabi/bin/../lib/gcc/arm-none-eabi/12.2.1/thumb/v8-m.main+fp/hard/crti.o
 .data          0x00000000        0x0 c:/renesas/ra/e2studio_v2023-07_fsp_v4.6.0/toolchains/gcc_arm/arm-gnu-toolchain-12.2.mpacbti-rel1-mingw-w64-i686-arm-none-eabi/bin/../lib/gcc/arm-none-eabi/12.2.1/thumb/v8-m.main+fp/hard/crti.o
 .bss           0x00000000        0x0 c:/renesas/ra/e2studio_v2023-07_fsp_v4.6.0/toolchains/gcc_arm/arm-gnu-toolchain-12.2.mpacbti-rel1-mingw-w64-i686-arm-none-eabi/bin/../lib/gcc/arm-none-eabi/12.2.1/thumb/v8-m.main+fp/hard/crti.o
 .text          0x00000000        0x0 c:/renesas/ra/e2studio_v2023-07_fsp_v4.6.0/toolchains/gcc_arm/arm-gnu-toolchain-12.2.mpacbti-rel1-mingw-w64-i686-arm-none-eabi/bin/../lib/gcc/arm-none-eabi/12.2.1/thumb/v8-m.main+fp/hard/crtbegin.o
 .data          0x00000000        0x0 c:/renesas/ra/e2studio_v2023-07_fsp_v4.6.0/toolchains/gcc_arm/arm-gnu-toolchain-12.2.mpacbti-rel1-mingw-w64-i686-arm-none-eabi/bin/../lib/gcc/arm-none-eabi/12.2.1/thumb/v8-m.main+fp/hard/crtbegin.o
 .bss           0x00000000        0x0 c:/renesas/ra/e2studio_v2023-07_fsp_v4.6.0/toolchains/gcc_arm/arm-gnu-toolchain-12.2.mpacbti-rel1-mingw-w64-i686-arm-none-eabi/bin/../lib/gcc/arm-none-eabi/12.2.1/thumb/v8-m.main+fp/hard/crtbegin.o
 .rodata.all_implied_fbits
                0x00000000       0x24 c:/renesas/ra/e2studio_v2023-07_fsp_v4.6.0/toolchains/gcc_arm/arm-gnu-toolchain-12.2.mpacbti-rel1-mingw-w64-i686-arm-none-eabi/bin/../lib/gcc/arm-none-eabi/12.2.1/thumb/v8-m.main+fp/hard/crtbegin.o
 .data.__dso_handle
                0x00000000        0x4 c:/renesas/ra/e2studio_v2023-07_fsp_v4.6.0/toolchains/gcc_arm/arm-gnu-toolchain-12.2.mpacbti-rel1-mingw-w64-i686-arm-none-eabi/bin/../lib/gcc/arm-none-eabi/12.2.1/thumb/v8-m.main+fp/hard/crtbegin.o
 .text          0x00000000       0xf8 c:/renesas/ra/e2studio_v2023-07_fsp_v4.6.0/toolchains/gcc_arm/arm-gnu-toolchain-12.2.mpacbti-rel1-mingw-w64-i686-arm-none-eabi/bin/../lib/gcc/arm-none-eabi/12.2.1/thumb/v8-m.main+fp/hard/rdimon-crt0.o
 .data          0x00000000      0x118 c:/renesas/ra/e2studio_v2023-07_fsp_v4.6.0/toolchains/gcc_arm/arm-gnu-toolchain-12.2.mpacbti-rel1-mingw-w64-i686-arm-none-eabi/bin/../lib/gcc/arm-none-eabi/12.2.1/thumb/v8-m.main+fp/hard/rdimon-crt0.o
 .bss           0x00000000        0x0 c:/renesas/ra/e2studio_v2023-07_fsp_v4.6.0/toolchains/gcc_arm/arm-gnu-toolchain-12.2.mpacbti-rel1-mingw-w64-i686-arm-none-eabi/bin/../lib/gcc/arm-none-eabi/12.2.1/thumb/v8-m.main+fp/hard/rdimon-crt0.o
 .ARM.extab     0x00000000        0x0 c:/renesas/ra/e2studio_v2023-07_fsp_v4.6.0/toolchains/gcc_arm/arm-gnu-toolchain-12.2.mpacbti-rel1-mingw-w64-i686-arm-none-eabi/bin/../lib/gcc/arm-none-eabi/12.2.1/thumb/v8-m.main+fp/hard/rdimon-crt0.o
 .ARM.exidx     0x00000000       0x10 c:/renesas/ra/e2studio_v2023-07_fsp_v4.6.0/toolchains/gcc_arm/arm-gnu-toolchain-12.2.mpacbti-rel1-mingw-w64-i686-arm-none-eabi/bin/../lib/gcc/arm-none-eabi/12.2.1/thumb/v8-m.main+fp/hard/rdimon-crt0.o
 .debug_line_str
                0x00000000       0xea c:/renesas/ra/e2studio_v2023-07_fsp_v4.6.0/toolchains/gcc_arm/arm-gnu-toolchain-12.2.mpacbti-rel1-mingw-w64-i686-arm-none-eabi/bin/../lib/gcc/arm-none-eabi/12.2.1/thumb/v8-m.main+fp/hard/rdimon-crt0.o
 .ARM.attributes
                0x00000000       0x24 c:/renesas/ra/e2studio_v2023-07_fsp_v4.6.0/toolchains/gcc_arm/arm-gnu-toolchain-12.2.mpacbti-rel1-mingw-w64-i686-arm-none-eabi/bin/../lib/gcc/arm-none-eabi/12.2.1/thumb/v8-m.main+fp/hard/rdimon-crt0.o
 .text          0x00000000        0x0 ./src/adc_temp.o
 .data          0x00000000        0x0 ./src/adc_temp.o
 .bss           0x00000000        0x0 ./src/adc_temp.o
 .text          0x00000000        0x0 ./src/angle.o
 .data          0x00000000        0x0 ./src/angle.o
 .bss           0x00000000        0x0 ./src/angle.o
 .text.tad2141_power
                0x00000000       0x98 ./src/angle.o
 .text.tad2141_EOL_Programming
                0x00000000      0x288 ./src/angle.o
 .text          0x00000000        0x0 ./src/control_table.o
 .data          0x00000000        0x0 ./src/control_table.o
 .bss           0x00000000        0x0 ./src/control_table.o
 .text          0x00000000        0x0 ./src/global_variables.o
 .data          0x00000000        0x0 ./src/global_variables.o
 .bss           0x00000000        0x0 ./src/global_variables.o
 .text          0x00000000        0x0 ./src/hal_entry.o
 .data          0x00000000        0x0 ./src/hal_entry.o
 .bss           0x00000000        0x0 ./src/hal_entry.o
 .text.led_toggle
                0x00000000       0x1c ./src/hal_entry.o
 .text          0x00000000        0x0 ./src/interpolation.o
 .data          0x00000000        0x0 ./src/interpolation.o
 .bss           0x00000000        0x0 ./src/interpolation.o
 .text          0x00000000        0x0 ./src/monitor.o
 .data          0x00000000        0x0 ./src/monitor.o
 .bss           0x00000000        0x0 ./src/monitor.o
 .text          0x00000000        0x0 ./src/packet.o
 .data          0x00000000        0x0 ./src/packet.o
 .bss           0x00000000        0x0 ./src/packet.o
 .text          0x00000000        0x0 ./src/pid.o
 .data          0x00000000        0x0 ./src/pid.o
 .bss           0x00000000        0x0 ./src/pid.o
 .text.PIDReset_int
                0x00000000        0xc ./src/pid.o
 .text.PIDUpdate_int
                0x00000000       0x54 ./src/pid.o
 .text          0x00000000        0x0 ./src/power_monitor.o
 .data          0x00000000        0x0 ./src/power_monitor.o
 .bss           0x00000000        0x0 ./src/power_monitor.o
 .text          0x00000000        0x0 ./src/sintable.o
 .data          0x00000000        0x0 ./src/sintable.o
 .bss           0x00000000        0x0 ./src/sintable.o
 .text.my_sin1000
                0x00000000       0x7c ./src/sintable.o
 .text          0x00000000        0x0 ./src/usart.o
 .data          0x00000000        0x0 ./src/usart.o
 .bss           0x00000000        0x0 ./src/usart.o
 .text.us_putc  0x00000000       0x30 ./src/usart.o
 .text.us_puts  0x00000000       0x78 ./src/usart.o
 .text.us_putsbd
                0x00000000       0x28 ./src/usart.o
 .text.us_rx_purge
                0x00000000       0x3c ./src/usart.o
 .rodata.us_printf.str1.4
                0x00000000       0x10 ./src/usart.o
 .text.us_printf
                0x00000000      0xc50 ./src/usart.o
 .text.us_deinit
                0x00000000       0x20 ./src/usart.o
 .bss.buf.0     0x00000000      0x400 ./src/usart.o
 .text          0x00000000        0x0 ./ra_gen/common_data.o
 .data          0x00000000        0x0 ./ra_gen/common_data.o
 .bss           0x00000000        0x0 ./ra_gen/common_data.o
 .text.g_common_init
                0x00000000        0x4 ./ra_gen/common_data.o
 .text          0x00000000        0x0 ./ra_gen/hal_data.o
 .data          0x00000000        0x0 ./ra_gen/hal_data.o
 .bss           0x00000000        0x0 ./ra_gen/hal_data.o
 .text.g_hal_init
                0x00000000        0x4 ./ra_gen/hal_data.o
 .rodata.g_uart4
                0x00000000        0xc ./ra_gen/hal_data.o
 .rodata.g_i2c3
                0x00000000        0xc ./ra_gen/hal_data.o
 .rodata.g_spi2
                0x00000000        0xc ./ra_gen/hal_data.o
 .rodata.g_timer5
                0x00000000        0xc ./ra_gen/hal_data.o
 .rodata.g_timer0
                0x00000000        0xc ./ra_gen/hal_data.o
 .rodata.g_adc0
                0x00000000       0x10 ./ra_gen/hal_data.o
 .rodata.g_flash0
                0x00000000        0xc ./ra_gen/hal_data.o
 .rodata.g_crc0
                0x00000000        0xc ./ra_gen/hal_data.o
 .rodata.g_rtc0
                0x00000000        0xc ./ra_gen/hal_data.o
 .rodata.g_rtc0_cfg
                0x00000000       0x20 ./ra_gen/hal_data.o
 .rodata.g_rtc0_err_cfg
                0x00000000        0x8 ./ra_gen/hal_data.o
 .bss.g_rtc0_ctrl
                0x00000000       0x18 ./ra_gen/hal_data.o
 .text          0x00000000        0x0 ./ra_gen/main.o
 .data          0x00000000        0x0 ./ra_gen/main.o
 .bss           0x00000000        0x0 ./ra_gen/main.o
 .text          0x00000000        0x0 ./ra_gen/pin_data.o
 .data          0x00000000        0x0 ./ra_gen/pin_data.o
 .bss           0x00000000        0x0 ./ra_gen/pin_data.o
 .text          0x00000000        0x0 ./ra_gen/vector_data.o
 .data          0x00000000        0x0 ./ra_gen/vector_data.o
 .bss           0x00000000        0x0 ./ra_gen/vector_data.o
 .text          0x00000000        0x0 ./ra/fsp/src/r_sci_uart/r_sci_uart.o
 .data          0x00000000        0x0 ./ra/fsp/src/r_sci_uart/r_sci_uart.o
 .bss           0x00000000        0x0 ./ra/fsp/src/r_sci_uart/r_sci_uart.o
 .text.R_SCI_UART_Read
                0x00000000       0x34 ./ra/fsp/src/r_sci_uart/r_sci_uart.o
 .text.R_SCI_UART_CallbackSet
                0x00000000       0x10 ./ra/fsp/src/r_sci_uart/r_sci_uart.o
 .text.R_SCI_UART_InfoGet
                0x00000000       0x28 ./ra/fsp/src/r_sci_uart/r_sci_uart.o
 .text.R_SCI_UART_ReadStop
                0x00000000       0x3c ./ra/fsp/src/r_sci_uart/r_sci_uart.o
 .text.R_SCI_UART_Close
                0x00000000       0xd4 ./ra/fsp/src/r_sci_uart/r_sci_uart.o
 .text.R_SCI_UART_Abort
                0x00000000       0x84 ./ra/fsp/src/r_sci_uart/r_sci_uart.o
 .rodata.g_uart_on_sci
                0x00000000       0x24 ./ra/fsp/src/r_sci_uart/r_sci_uart.o
 .text          0x00000000        0x0 ./ra/fsp/src/r_sci_spi/r_sci_spi.o
 .data          0x00000000        0x0 ./ra/fsp/src/r_sci_spi/r_sci_spi.o
 .bss           0x00000000        0x0 ./ra/fsp/src/r_sci_spi/r_sci_spi.o
 .text.R_SCI_SPI_CallbackSet
                0x00000000       0x10 ./ra/fsp/src/r_sci_spi/r_sci_spi.o
 .text.R_SCI_SPI_Close
                0x00000000       0xd4 ./ra/fsp/src/r_sci_spi/r_sci_spi.o
 .text.R_SCI_SPI_Write
                0x00000000      0x10c ./ra/fsp/src/r_sci_spi/r_sci_spi.o
 .text.R_SCI_SPI_Read
                0x00000000      0x114 ./ra/fsp/src/r_sci_spi/r_sci_spi.o
 .text.R_SCI_SPI_CalculateBitrate
                0x00000000       0xbc ./ra/fsp/src/r_sci_spi/r_sci_spi.o
 .rodata.g_spi_on_sci
                0x00000000       0x18 ./ra/fsp/src/r_sci_spi/r_sci_spi.o
 .text          0x00000000        0x0 ./ra/fsp/src/r_sci_i2c/r_sci_i2c.o
 .data          0x00000000        0x0 ./ra/fsp/src/r_sci_i2c/r_sci_i2c.o
 .bss           0x00000000        0x0 ./ra/fsp/src/r_sci_i2c/r_sci_i2c.o
 .text.R_SCI_I2C_Abort
                0x00000000       0x2c ./ra/fsp/src/r_sci_i2c/r_sci_i2c.o
 .text.R_SCI_I2C_CallbackSet
                0x00000000       0x10 ./ra/fsp/src/r_sci_i2c/r_sci_i2c.o
 .text.R_SCI_I2C_StatusGet
                0x00000000       0x18 ./ra/fsp/src/r_sci_i2c/r_sci_i2c.o
 .text.R_SCI_I2C_Close
                0x00000000       0x58 ./ra/fsp/src/r_sci_i2c/r_sci_i2c.o
 .text.sci_i2c_notify
                0x00000000       0x38 ./ra/fsp/src/r_sci_i2c/r_sci_i2c.o
 .rodata.g_i2c_master_on_sci
                0x00000000       0x20 ./ra/fsp/src/r_sci_i2c/r_sci_i2c.o
 .text          0x00000000        0x0 ./ra/fsp/src/r_rtc/r_rtc.o
 .data          0x00000000        0x0 ./ra/fsp/src/r_rtc/r_rtc.o
 .bss           0x00000000        0x0 ./ra/fsp/src/r_rtc/r_rtc.o
 .text.R_RTC_Close
                0x00000000       0xe8 ./ra/fsp/src/r_rtc/r_rtc.o
 .text.R_RTC_CalendarAlarmSet
                0x00000000      0x210 ./ra/fsp/src/r_rtc/r_rtc.o
 .text.R_RTC_CalendarAlarmGet
                0x00000000       0xd0 ./ra/fsp/src/r_rtc/r_rtc.o
 .text.R_RTC_PeriodicIrqRateSet
                0x00000000       0x7c ./ra/fsp/src/r_rtc/r_rtc.o
 .text.R_RTC_InfoGet
                0x00000000       0x1c ./ra/fsp/src/r_rtc/r_rtc.o
 .text.R_RTC_CallbackSet
                0x00000000       0x10 ./ra/fsp/src/r_rtc/r_rtc.o
 .text.R_RTC_ClockSourceSet
                0x00000000       0x90 ./ra/fsp/src/r_rtc/r_rtc.o
 .text.R_RTC_CalendarTimeGet
                0x00000000      0x188 ./ra/fsp/src/r_rtc/r_rtc.o
 .text.R_RTC_Open
                0x00000000       0x88 ./ra/fsp/src/r_rtc/r_rtc.o
 .text.R_RTC_CalendarTimeSet
                0x00000000      0x1b8 ./ra/fsp/src/r_rtc/r_rtc.o
 .text.R_RTC_ErrorAdjustmentSet
                0x00000000       0x94 ./ra/fsp/src/r_rtc/r_rtc.o
 .text.rtc_alarm_periodic_isr
                0x00000000       0x70 ./ra/fsp/src/r_rtc/r_rtc.o
 .rodata.g_rtc_on_rtc
                0x00000000       0x2c ./ra/fsp/src/r_rtc/r_rtc.o
 .text          0x00000000        0x0 ./ra/fsp/src/r_ioport/r_ioport.o
 .data          0x00000000        0x0 ./ra/fsp/src/r_ioport/r_ioport.o
 .bss           0x00000000        0x0 ./ra/fsp/src/r_ioport/r_ioport.o
 .text          0x00000000        0x0 ./ra/fsp/src/r_gpt/r_gpt.o
 .data          0x00000000        0x0 ./ra/fsp/src/r_gpt/r_gpt.o
 .bss           0x00000000        0x0 ./ra/fsp/src/r_gpt/r_gpt.o
 .text.R_GPT_Stop
                0x00000000        0xc ./ra/fsp/src/r_gpt/r_gpt.o
 .text.R_GPT_Reset
                0x00000000        0xc ./ra/fsp/src/r_gpt/r_gpt.o
 .text.R_GPT_Enable
                0x00000000       0x30 ./ra/fsp/src/r_gpt/r_gpt.o
 .text.R_GPT_Disable
                0x00000000       0x18 ./ra/fsp/src/r_gpt/r_gpt.o
 .text.R_GPT_PeriodSet
                0x00000000       0x30 ./ra/fsp/src/r_gpt/r_gpt.o
 .text.R_GPT_InfoGet
                0x00000000       0x44 ./ra/fsp/src/r_gpt/r_gpt.o
 .text.R_GPT_StatusGet
                0x00000000       0x14 ./ra/fsp/src/r_gpt/r_gpt.o
 .text.R_GPT_CallbackSet
                0x00000000       0x10 ./ra/fsp/src/r_gpt/r_gpt.o
 .text.R_GPT_Close
                0x00000000       0xa0 ./ra/fsp/src/r_gpt/r_gpt.o
 .text.R_GPT_CounterSet
                0x00000000        0xc ./ra/fsp/src/r_gpt/r_gpt.o
 .text.R_GPT_OutputEnable
                0x00000000       0x18 ./ra/fsp/src/r_gpt/r_gpt.o
 .text.R_GPT_OutputDisable
                0x00000000       0x18 ./ra/fsp/src/r_gpt/r_gpt.o
 .text.R_GPT_AdcTriggerSet
                0x00000000       0x10 ./ra/fsp/src/r_gpt/r_gpt.o
 .text.R_GPT_PwmOutputDelaySet
                0x00000000        0x4 ./ra/fsp/src/r_gpt/r_gpt.o
 .text.R_GPT_PwmOutputDelayInitialize
                0x00000000        0x4 ./ra/fsp/src/r_gpt/r_gpt.o
 .text.gpt_counter_overflow_isr
                0x00000000       0xb8 ./ra/fsp/src/r_gpt/r_gpt.o
 .text.gpt_capture_a_isr
                0x00000000       0xc8 ./ra/fsp/src/r_gpt/r_gpt.o
 .text.gpt_capture_b_isr
                0x00000000       0xc8 ./ra/fsp/src/r_gpt/r_gpt.o
 .rodata.g_timer_on_gpt
                0x00000000       0x30 ./ra/fsp/src/r_gpt/r_gpt.o
 .text          0x00000000        0x0 ./ra/fsp/src/r_flash_hp/r_flash_hp.o
 .data          0x00000000        0x0 ./ra/fsp/src/r_flash_hp/r_flash_hp.o
 .bss           0x00000000        0x0 ./ra/fsp/src/r_flash_hp/r_flash_hp.o
 .text.R_FLASH_HP_StatusGet
                0x00000000       0x1c ./ra/fsp/src/r_flash_hp/r_flash_hp.o
 .text.R_FLASH_HP_IdCodeSet
                0x00000000        0x4 ./ra/fsp/src/r_flash_hp/r_flash_hp.o
 .text.R_FLASH_HP_AccessWindowSet
                0x00000000        0x4 ./ra/fsp/src/r_flash_hp/r_flash_hp.o
 .text.R_FLASH_HP_AccessWindowClear
                0x00000000        0x4 ./ra/fsp/src/r_flash_hp/r_flash_hp.o
 .text.R_FLASH_HP_StartUpAreaSelect
                0x00000000        0x4 ./ra/fsp/src/r_flash_hp/r_flash_hp.o
 .text.R_FLASH_HP_InfoGet
                0x00000000       0x2c ./ra/fsp/src/r_flash_hp/r_flash_hp.o
 .text.R_FLASH_HP_CallbackSet
                0x00000000       0x10 ./ra/fsp/src/r_flash_hp/r_flash_hp.o
 .text.R_FLASH_HP_BankSwap
                0x00000000        0x4 ./ra/fsp/src/r_flash_hp/r_flash_hp.o
 .text.R_FLASH_HP_BlankCheck
                0x00000000      0x1b0 ./ra/fsp/src/r_flash_hp/r_flash_hp.o
 .text.flash_hp_reset
                0x00000000      0x180 ./ra/fsp/src/r_flash_hp/r_flash_hp.o
 .text.R_FLASH_HP_Reset
                0x00000000        0x4 ./ra/fsp/src/r_flash_hp/r_flash_hp.o
 .text.R_FLASH_HP_UpdateFlashClockFreq
                0x00000000      0x108 ./ra/fsp/src/r_flash_hp/r_flash_hp.o
 .text.fcu_fiferr_isr
                0x00000000       0x94 ./ra/fsp/src/r_flash_hp/r_flash_hp.o
 .text.fcu_frdyi_isr
                0x00000000      0x1ac ./ra/fsp/src/r_flash_hp/r_flash_hp.o
 .rodata.g_flash_on_flash_hp
                0x00000000       0x3c ./ra/fsp/src/r_flash_hp/r_flash_hp.o
 .rodata.g_flash_data_region
                0x00000000        0x8 ./ra/fsp/src/r_flash_hp/r_flash_hp.o
 .rodata.g_data_flash_macro_info
                0x00000000       0x10 ./ra/fsp/src/r_flash_hp/r_flash_hp.o
 .rodata.g_flash_code_region
                0x00000000        0x8 ./ra/fsp/src/r_flash_hp/r_flash_hp.o
 .rodata.g_code_flash_macro_info
                0x00000000       0x20 ./ra/fsp/src/r_flash_hp/r_flash_hp.o
 .text          0x00000000        0x0 ./ra/fsp/src/r_dtc/r_dtc.o
 .data          0x00000000        0x0 ./ra/fsp/src/r_dtc/r_dtc.o
 .bss           0x00000000        0x0 ./ra/fsp/src/r_dtc/r_dtc.o
 .text          0x00000000        0x0 ./ra/fsp/src/r_crc/r_crc.o
 .data          0x00000000        0x0 ./ra/fsp/src/r_crc/r_crc.o
 .bss           0x00000000        0x0 ./ra/fsp/src/r_crc/r_crc.o
 .text.R_CRC_CalculatedValueGet
                0x00000000       0x34 ./ra/fsp/src/r_crc/r_crc.o
 .text.R_CRC_SnoopEnable
                0x00000000        0x4 ./ra/fsp/src/r_crc/r_crc.o
 .text.R_CRC_SnoopDisable
                0x00000000        0x4 ./ra/fsp/src/r_crc/r_crc.o
 .rodata.g_crc_on_crc
                0x00000000       0x18 ./ra/fsp/src/r_crc/r_crc.o
 .text          0x00000000        0x0 ./ra/fsp/src/r_agt/r_agt.o
 .data          0x00000000        0x0 ./ra/fsp/src/r_agt/r_agt.o
 .bss           0x00000000        0x0 ./ra/fsp/src/r_agt/r_agt.o
 .text.R_AGT_Start
                0x00000000       0x60 ./ra/fsp/src/r_agt/r_agt.o
 .text.R_AGT_Stop
                0x00000000       0x24 ./ra/fsp/src/r_agt/r_agt.o
 .text.R_AGT_Disable
                0x00000000       0x1c ./ra/fsp/src/r_agt/r_agt.o
 .text.R_AGT_PeriodSet
                0x00000000       0x4c ./ra/fsp/src/r_agt/r_agt.o
 .text.R_AGT_DutyCycleSet
                0x00000000        0x4 ./ra/fsp/src/r_agt/r_agt.o
 .text.R_AGT_InfoGet
                0x00000000       0xe8 ./ra/fsp/src/r_agt/r_agt.o
 .text.R_AGT_StatusGet
                0x00000000       0x44 ./ra/fsp/src/r_agt/r_agt.o
 .text.R_AGT_CallbackSet
                0x00000000       0x10 ./ra/fsp/src/r_agt/r_agt.o
 .text.R_AGT_Close
                0x00000000       0x74 ./ra/fsp/src/r_agt/r_agt.o
 .text.R_AGT_Reset
                0x00000000       0x3c ./ra/fsp/src/r_agt/r_agt.o
 .rodata.g_timer_on_agt
                0x00000000       0x30 ./ra/fsp/src/r_agt/r_agt.o
 .text          0x00000000        0x0 ./ra/fsp/src/r_adc/r_adc.o
 .data          0x00000000        0x0 ./ra/fsp/src/r_adc/r_adc.o
 .bss           0x00000000        0x0 ./ra/fsp/src/r_adc/r_adc.o
 .text.R_ADC_CallbackSet
                0x00000000       0x10 ./ra/fsp/src/r_adc/r_adc.o
 .text.R_ADC_ScanGroupStart
                0x00000000        0x4 ./ra/fsp/src/r_adc/r_adc.o
 .text.R_ADC_ScanStop
                0x00000000        0xc ./ra/fsp/src/r_adc/r_adc.o
 .text.R_ADC_StatusGet
                0x00000000       0x10 ./ra/fsp/src/r_adc/r_adc.o
 .text.R_ADC_Read32
                0x00000000       0x1c ./ra/fsp/src/r_adc/r_adc.o
 .text.R_ADC_Calibrate
                0x00000000        0x4 ./ra/fsp/src/r_adc/r_adc.o
 .text.R_ADC_OffsetSet
                0x00000000        0x4 ./ra/fsp/src/r_adc/r_adc.o
 .text.r_adc_call_callback
                0x00000000       0x54 ./ra/fsp/src/r_adc/r_adc.o
 .text.R_ADC_InfoGet
                0x00000000       0x6c ./ra/fsp/src/r_adc/r_adc.o
 .text.R_ADC_Close
                0x00000000       0xf4 ./ra/fsp/src/r_adc/r_adc.o
 .text.R_ADC_SampleStateCountSet
                0x00000000       0x14 ./ra/fsp/src/r_adc/r_adc.o
 .text.adc_scan_end_isr
                0x00000000       0x5c ./ra/fsp/src/r_adc/r_adc.o
 .text.adc_scan_end_b_isr
                0x00000000       0x64 ./ra/fsp/src/r_adc/r_adc.o
 .text.adc_window_compare_isr
                0x00000000      0x118 ./ra/fsp/src/r_adc/r_adc.o
 .rodata.g_adc_on_adc
                0x00000000       0x34 ./ra/fsp/src/r_adc/r_adc.o
 .text          0x00000000        0x0 ./ra/fsp/src/bsp/mcu/all/bsp_clocks.o
 .data          0x00000000        0x0 ./ra/fsp/src/bsp/mcu/all/bsp_clocks.o
 .bss           0x00000000        0x0 ./ra/fsp/src/bsp/mcu/all/bsp_clocks.o
 .text.bsp_prv_operating_mode_set
                0x00000000       0x60 ./ra/fsp/src/bsp/mcu/all/bsp_clocks.o
 .text.bsp_prv_prepare_pll
                0x00000000        0xc ./ra/fsp/src/bsp/mcu/all/bsp_clocks.o
 .text.prv_clock_dividers_set
                0x00000000        0xc ./ra/fsp/src/bsp/mcu/all/bsp_clocks.o
 .text.bsp_prv_clock_set
                0x00000000       0xb0 ./ra/fsp/src/bsp/mcu/all/bsp_clocks.o
 .text.R_BSP_SubClockStabilizeWait
                0x00000000        0x8 ./ra/fsp/src/bsp/mcu/all/bsp_clocks.o
 .text.R_BSP_OctaclkUpdate
                0x00000000        0x4 ./ra/fsp/src/bsp/mcu/all/bsp_clocks.o
 .text.R_BSP_SourceClockHzGet
                0x00000000        0xc ./ra/fsp/src/bsp/mcu/all/bsp_clocks.o
 .text          0x00000000        0x0 ./ra/fsp/src/bsp/mcu/all/bsp_common.o
 .data          0x00000000        0x0 ./ra/fsp/src/bsp/mcu/all/bsp_common.o
 .bss           0x00000000        0x0 ./ra/fsp/src/bsp/mcu/all/bsp_common.o
 .text.R_FSP_VersionGet
                0x00000000       0x10 ./ra/fsp/src/bsp/mcu/all/bsp_common.o
 .text.__assert_func
                0x00000000        0x4 ./ra/fsp/src/bsp/mcu/all/bsp_common.o
 .text          0x00000000        0x0 ./ra/fsp/src/bsp/mcu/all/bsp_delay.o
 .data          0x00000000        0x0 ./ra/fsp/src/bsp/mcu/all/bsp_delay.o
 .bss           0x00000000        0x0 ./ra/fsp/src/bsp/mcu/all/bsp_delay.o
 .text          0x00000000        0x0 ./ra/fsp/src/bsp/mcu/all/bsp_group_irq.o
 .data          0x00000000        0x0 ./ra/fsp/src/bsp/mcu/all/bsp_group_irq.o
 .bss           0x00000000        0x0 ./ra/fsp/src/bsp/mcu/all/bsp_group_irq.o
 .text.R_BSP_GroupIrqWrite
                0x00000000       0x10 ./ra/fsp/src/bsp/mcu/all/bsp_group_irq.o
 .text          0x00000000        0x0 ./ra/fsp/src/bsp/mcu/all/bsp_guard.o
 .data          0x00000000        0x0 ./ra/fsp/src/bsp/mcu/all/bsp_guard.o
 .bss           0x00000000        0x0 ./ra/fsp/src/bsp/mcu/all/bsp_guard.o
 .debug_info    0x00000000       0x6c ./ra/fsp/src/bsp/mcu/all/bsp_guard.o
 .debug_abbrev  0x00000000       0x26 ./ra/fsp/src/bsp/mcu/all/bsp_guard.o
 .debug_aranges
                0x00000000       0x18 ./ra/fsp/src/bsp/mcu/all/bsp_guard.o
 .debug_line    0x00000000       0x46 ./ra/fsp/src/bsp/mcu/all/bsp_guard.o
 .debug_str     0x00000000      0x1a8 ./ra/fsp/src/bsp/mcu/all/bsp_guard.o
 .comment       0x00000000       0x56 ./ra/fsp/src/bsp/mcu/all/bsp_guard.o
 .ARM.attributes
                0x00000000       0x3a ./ra/fsp/src/bsp/mcu/all/bsp_guard.o
 .text          0x00000000        0x0 ./ra/fsp/src/bsp/mcu/all/bsp_io.o
 .data          0x00000000        0x0 ./ra/fsp/src/bsp/mcu/all/bsp_io.o
 .bss           0x00000000        0x0 ./ra/fsp/src/bsp/mcu/all/bsp_io.o
 .text          0x00000000        0x0 ./ra/fsp/src/bsp/mcu/all/bsp_irq.o
 .data          0x00000000        0x0 ./ra/fsp/src/bsp/mcu/all/bsp_irq.o
 .bss           0x00000000        0x0 ./ra/fsp/src/bsp/mcu/all/bsp_irq.o
 .rodata.g_interrupt_event_link_select
                0x00000000       0xc0 ./ra/fsp/src/bsp/mcu/all/bsp_irq.o
 .text          0x00000000        0x0 ./ra/fsp/src/bsp/mcu/all/bsp_register_protection.o
 .data          0x00000000        0x0 ./ra/fsp/src/bsp/mcu/all/bsp_register_protection.o
 .bss           0x00000000        0x0 ./ra/fsp/src/bsp/mcu/all/bsp_register_protection.o
 .text          0x00000000        0x0 ./ra/fsp/src/bsp/mcu/all/bsp_rom_registers.o
 .data          0x00000000        0x0 ./ra/fsp/src/bsp/mcu/all/bsp_rom_registers.o
 .bss           0x00000000        0x0 ./ra/fsp/src/bsp/mcu/all/bsp_rom_registers.o
 .option_setting_bps_sel3
                0x00000000        0x4 ./ra/fsp/src/bsp/mcu/all/bsp_rom_registers.o
 .option_setting_pbps_sec3
                0x00000000        0x4 ./ra/fsp/src/bsp/mcu/all/bsp_rom_registers.o
 .option_setting_bps_sec3
                0x00000000        0x4 ./ra/fsp/src/bsp/mcu/all/bsp_rom_registers.o
 .text          0x00000000        0x0 ./ra/fsp/src/bsp/mcu/all/bsp_sbrk.o
 .data          0x00000000        0x0 ./ra/fsp/src/bsp/mcu/all/bsp_sbrk.o
 .bss           0x00000000        0x0 ./ra/fsp/src/bsp/mcu/all/bsp_sbrk.o
 .text._sbrk    0x00000000       0x40 ./ra/fsp/src/bsp/mcu/all/bsp_sbrk.o
 .bss.current_heap_end.0
                0x00000000        0x4 ./ra/fsp/src/bsp/mcu/all/bsp_sbrk.o
 .debug_info    0x00000000      0x134 ./ra/fsp/src/bsp/mcu/all/bsp_sbrk.o
 .debug_abbrev  0x00000000       0xce ./ra/fsp/src/bsp/mcu/all/bsp_sbrk.o
 .debug_loclists
                0x00000000       0xa5 ./ra/fsp/src/bsp/mcu/all/bsp_sbrk.o
 .debug_aranges
                0x00000000       0x20 ./ra/fsp/src/bsp/mcu/all/bsp_sbrk.o
 .debug_rnglists
                0x00000000       0x13 ./ra/fsp/src/bsp/mcu/all/bsp_sbrk.o
 .debug_line    0x00000000      0x231 ./ra/fsp/src/bsp/mcu/all/bsp_sbrk.o
 .debug_str     0x00000000      0x232 ./ra/fsp/src/bsp/mcu/all/bsp_sbrk.o
 .comment       0x00000000       0x56 ./ra/fsp/src/bsp/mcu/all/bsp_sbrk.o
 .debug_frame   0x00000000       0x28 ./ra/fsp/src/bsp/mcu/all/bsp_sbrk.o
 .ARM.attributes
                0x00000000       0x3a ./ra/fsp/src/bsp/mcu/all/bsp_sbrk.o
 .text          0x00000000        0x0 ./ra/fsp/src/bsp/mcu/all/bsp_security.o
 .data          0x00000000        0x0 ./ra/fsp/src/bsp/mcu/all/bsp_security.o
 .bss           0x00000000        0x0 ./ra/fsp/src/bsp/mcu/all/bsp_security.o
 .rodata.gp_start_of_nonsecure_callable_ram
                0x00000000        0x4 ./ra/fsp/src/bsp/mcu/all/bsp_security.o
 .rodata.gp_start_of_nonsecure_ram
                0x00000000        0x4 ./ra/fsp/src/bsp/mcu/all/bsp_security.o
 .rodata.gp_start_of_nonsecure_data_flash
                0x00000000        0x4 ./ra/fsp/src/bsp/mcu/all/bsp_security.o
 .rodata.gp_start_of_nonsecure_callable_flash
                0x00000000        0x4 ./ra/fsp/src/bsp/mcu/all/bsp_security.o
 .rodata.gp_start_of_nonsecure_flash
                0x00000000        0x4 ./ra/fsp/src/bsp/mcu/all/bsp_security.o
 .debug_info    0x00000000      0x116 ./ra/fsp/src/bsp/mcu/all/bsp_security.o
 .debug_abbrev  0x00000000       0x6f ./ra/fsp/src/bsp/mcu/all/bsp_security.o
 .debug_aranges
                0x00000000       0x18 ./ra/fsp/src/bsp/mcu/all/bsp_security.o
 .debug_line    0x00000000      0x1a0 ./ra/fsp/src/bsp/mcu/all/bsp_security.o
 .debug_str     0x00000000      0x2a8 ./ra/fsp/src/bsp/mcu/all/bsp_security.o
 .comment       0x00000000       0x56 ./ra/fsp/src/bsp/mcu/all/bsp_security.o
 .ARM.attributes
                0x00000000       0x3a ./ra/fsp/src/bsp/mcu/all/bsp_security.o
 .text          0x00000000        0x0 ./ra/fsp/src/bsp/cmsis/Device/RENESAS/Source/startup.o
 .data          0x00000000        0x0 ./ra/fsp/src/bsp/cmsis/Device/RENESAS/Source/startup.o
 .bss           0x00000000        0x0 ./ra/fsp/src/bsp/cmsis/Device/RENESAS/Source/startup.o
 .text          0x00000000        0x0 ./ra/fsp/src/bsp/cmsis/Device/RENESAS/Source/system.o
 .data          0x00000000        0x0 ./ra/fsp/src/bsp/cmsis/Device/RENESAS/Source/system.o
 .bss           0x00000000        0x0 ./ra/fsp/src/bsp/cmsis/Device/RENESAS/Source/system.o
 .text.R_BSP_WarmStart
                0x00000000        0x4 ./ra/fsp/src/bsp/cmsis/Device/RENESAS/Source/system.o
 .text          0x00000000      0x254 c:/renesas/ra/e2studio_v2023-07_fsp_v4.6.0/toolchains/gcc_arm/arm-gnu-toolchain-12.2.mpacbti-rel1-mingw-w64-i686-arm-none-eabi/bin/../lib/gcc/arm-none-eabi/12.2.1/thumb/v8-m.main+fp/hard\libgcc.a(_arm_muldf3.o)
 .data          0x00000000        0x0 c:/renesas/ra/e2studio_v2023-07_fsp_v4.6.0/toolchains/gcc_arm/arm-gnu-toolchain-12.2.mpacbti-rel1-mingw-w64-i686-arm-none-eabi/bin/../lib/gcc/arm-none-eabi/12.2.1/thumb/v8-m.main+fp/hard\libgcc.a(_arm_muldf3.o)
 .bss           0x00000000        0x0 c:/renesas/ra/e2studio_v2023-07_fsp_v4.6.0/toolchains/gcc_arm/arm-gnu-toolchain-12.2.mpacbti-rel1-mingw-w64-i686-arm-none-eabi/bin/../lib/gcc/arm-none-eabi/12.2.1/thumb/v8-m.main+fp/hard\libgcc.a(_arm_muldf3.o)
 .debug_line_str
                0x00000000       0xe2 c:/renesas/ra/e2studio_v2023-07_fsp_v4.6.0/toolchains/gcc_arm/arm-gnu-toolchain-12.2.mpacbti-rel1-mingw-w64-i686-arm-none-eabi/bin/../lib/gcc/arm-none-eabi/12.2.1/thumb/v8-m.main+fp/hard\libgcc.a(_arm_muldf3.o)
 .debug_frame   0x00000000       0x30 c:/renesas/ra/e2studio_v2023-07_fsp_v4.6.0/toolchains/gcc_arm/arm-gnu-toolchain-12.2.mpacbti-rel1-mingw-w64-i686-arm-none-eabi/bin/../lib/gcc/arm-none-eabi/12.2.1/thumb/v8-m.main+fp/hard\libgcc.a(_arm_muldf3.o)
 .ARM.attributes
                0x00000000       0x26 c:/renesas/ra/e2studio_v2023-07_fsp_v4.6.0/toolchains/gcc_arm/arm-gnu-toolchain-12.2.mpacbti-rel1-mingw-w64-i686-arm-none-eabi/bin/../lib/gcc/arm-none-eabi/12.2.1/thumb/v8-m.main+fp/hard\libgcc.a(_arm_muldf3.o)
 .data          0x00000000        0x0 c:/renesas/ra/e2studio_v2023-07_fsp_v4.6.0/toolchains/gcc_arm/arm-gnu-toolchain-12.2.mpacbti-rel1-mingw-w64-i686-arm-none-eabi/bin/../lib/gcc/arm-none-eabi/12.2.1/thumb/v8-m.main+fp/hard\libgcc.a(_arm_addsubdf3.o)
 .bss           0x00000000        0x0 c:/renesas/ra/e2studio_v2023-07_fsp_v4.6.0/toolchains/gcc_arm/arm-gnu-toolchain-12.2.mpacbti-rel1-mingw-w64-i686-arm-none-eabi/bin/../lib/gcc/arm-none-eabi/12.2.1/thumb/v8-m.main+fp/hard\libgcc.a(_arm_addsubdf3.o)
 .data          0x00000000        0x0 c:/renesas/ra/e2studio_v2023-07_fsp_v4.6.0/toolchains/gcc_arm/arm-gnu-toolchain-12.2.mpacbti-rel1-mingw-w64-i686-arm-none-eabi/bin/../lib/gcc/arm-none-eabi/12.2.1/thumb/v8-m.main+fp/hard\libgcc.a(_arm_muldivdf3.o)
 .bss           0x00000000        0x0 c:/renesas/ra/e2studio_v2023-07_fsp_v4.6.0/toolchains/gcc_arm/arm-gnu-toolchain-12.2.mpacbti-rel1-mingw-w64-i686-arm-none-eabi/bin/../lib/gcc/arm-none-eabi/12.2.1/thumb/v8-m.main+fp/hard\libgcc.a(_arm_muldivdf3.o)
 .data          0x00000000        0x0 c:/renesas/ra/e2studio_v2023-07_fsp_v4.6.0/toolchains/gcc_arm/arm-gnu-toolchain-12.2.mpacbti-rel1-mingw-w64-i686-arm-none-eabi/bin/../lib/gcc/arm-none-eabi/12.2.1/thumb/v8-m.main+fp/hard\libgcc.a(_arm_cmpdf2.o)
 .bss           0x00000000        0x0 c:/renesas/ra/e2studio_v2023-07_fsp_v4.6.0/toolchains/gcc_arm/arm-gnu-toolchain-12.2.mpacbti-rel1-mingw-w64-i686-arm-none-eabi/bin/../lib/gcc/arm-none-eabi/12.2.1/thumb/v8-m.main+fp/hard\libgcc.a(_arm_cmpdf2.o)
 .text          0x00000000       0x2c c:/renesas/ra/e2studio_v2023-07_fsp_v4.6.0/toolchains/gcc_arm/arm-gnu-toolchain-12.2.mpacbti-rel1-mingw-w64-i686-arm-none-eabi/bin/../lib/gcc/arm-none-eabi/12.2.1/thumb/v8-m.main+fp/hard\libgcc.a(_arm_unorddf2.o)
 .data          0x00000000        0x0 c:/renesas/ra/e2studio_v2023-07_fsp_v4.6.0/toolchains/gcc_arm/arm-gnu-toolchain-12.2.mpacbti-rel1-mingw-w64-i686-arm-none-eabi/bin/../lib/gcc/arm-none-eabi/12.2.1/thumb/v8-m.main+fp/hard\libgcc.a(_arm_unorddf2.o)
 .bss           0x00000000        0x0 c:/renesas/ra/e2studio_v2023-07_fsp_v4.6.0/toolchains/gcc_arm/arm-gnu-toolchain-12.2.mpacbti-rel1-mingw-w64-i686-arm-none-eabi/bin/../lib/gcc/arm-none-eabi/12.2.1/thumb/v8-m.main+fp/hard\libgcc.a(_arm_unorddf2.o)
 .debug_line_str
                0x00000000       0xe2 c:/renesas/ra/e2studio_v2023-07_fsp_v4.6.0/toolchains/gcc_arm/arm-gnu-toolchain-12.2.mpacbti-rel1-mingw-w64-i686-arm-none-eabi/bin/../lib/gcc/arm-none-eabi/12.2.1/thumb/v8-m.main+fp/hard\libgcc.a(_arm_unorddf2.o)
 .debug_frame   0x00000000       0x20 c:/renesas/ra/e2studio_v2023-07_fsp_v4.6.0/toolchains/gcc_arm/arm-gnu-toolchain-12.2.mpacbti-rel1-mingw-w64-i686-arm-none-eabi/bin/../lib/gcc/arm-none-eabi/12.2.1/thumb/v8-m.main+fp/hard\libgcc.a(_arm_unorddf2.o)
 .ARM.attributes
                0x00000000       0x26 c:/renesas/ra/e2studio_v2023-07_fsp_v4.6.0/toolchains/gcc_arm/arm-gnu-toolchain-12.2.mpacbti-rel1-mingw-w64-i686-arm-none-eabi/bin/../lib/gcc/arm-none-eabi/12.2.1/thumb/v8-m.main+fp/hard\libgcc.a(_arm_unorddf2.o)
 .data          0x00000000        0x0 c:/renesas/ra/e2studio_v2023-07_fsp_v4.6.0/toolchains/gcc_arm/arm-gnu-toolchain-12.2.mpacbti-rel1-mingw-w64-i686-arm-none-eabi/bin/../lib/gcc/arm-none-eabi/12.2.1/thumb/v8-m.main+fp/hard\libgcc.a(_arm_fixdfsi.o)
 .bss           0x00000000        0x0 c:/renesas/ra/e2studio_v2023-07_fsp_v4.6.0/toolchains/gcc_arm/arm-gnu-toolchain-12.2.mpacbti-rel1-mingw-w64-i686-arm-none-eabi/bin/../lib/gcc/arm-none-eabi/12.2.1/thumb/v8-m.main+fp/hard\libgcc.a(_arm_fixdfsi.o)
 .data          0x00000000        0x0 c:/renesas/ra/e2studio_v2023-07_fsp_v4.6.0/toolchains/gcc_arm/arm-gnu-toolchain-12.2.mpacbti-rel1-mingw-w64-i686-arm-none-eabi/bin/../lib/gcc/arm-none-eabi/12.2.1/thumb/v8-m.main+fp/hard\libgcc.a(_arm_fixunsdfsi.o)
 .bss           0x00000000        0x0 c:/renesas/ra/e2studio_v2023-07_fsp_v4.6.0/toolchains/gcc_arm/arm-gnu-toolchain-12.2.mpacbti-rel1-mingw-w64-i686-arm-none-eabi/bin/../lib/gcc/arm-none-eabi/12.2.1/thumb/v8-m.main+fp/hard\libgcc.a(_arm_fixunsdfsi.o)
 .data          0x00000000        0x0 c:/renesas/ra/e2studio_v2023-07_fsp_v4.6.0/toolchains/gcc_arm/arm-gnu-toolchain-12.2.mpacbti-rel1-mingw-w64-i686-arm-none-eabi/bin/../lib/gcc/arm-none-eabi/12.2.1/thumb/v8-m.main+fp/hard\libgcc.a(_aeabi_ldivmod.o)
 .bss           0x00000000        0x0 c:/renesas/ra/e2studio_v2023-07_fsp_v4.6.0/toolchains/gcc_arm/arm-gnu-toolchain-12.2.mpacbti-rel1-mingw-w64-i686-arm-none-eabi/bin/../lib/gcc/arm-none-eabi/12.2.1/thumb/v8-m.main+fp/hard\libgcc.a(_aeabi_ldivmod.o)
 .text          0x00000000        0x0 c:/renesas/ra/e2studio_v2023-07_fsp_v4.6.0/toolchains/gcc_arm/arm-gnu-toolchain-12.2.mpacbti-rel1-mingw-w64-i686-arm-none-eabi/bin/../lib/gcc/arm-none-eabi/12.2.1/thumb/v8-m.main+fp/hard\libgcc.a(_udivmoddi4.o)
 .data          0x00000000        0x0 c:/renesas/ra/e2studio_v2023-07_fsp_v4.6.0/toolchains/gcc_arm/arm-gnu-toolchain-12.2.mpacbti-rel1-mingw-w64-i686-arm-none-eabi/bin/../lib/gcc/arm-none-eabi/12.2.1/thumb/v8-m.main+fp/hard\libgcc.a(_udivmoddi4.o)
 .bss           0x00000000        0x0 c:/renesas/ra/e2studio_v2023-07_fsp_v4.6.0/toolchains/gcc_arm/arm-gnu-toolchain-12.2.mpacbti-rel1-mingw-w64-i686-arm-none-eabi/bin/../lib/gcc/arm-none-eabi/12.2.1/thumb/v8-m.main+fp/hard\libgcc.a(_udivmoddi4.o)
 .ARM.extab.text.__udivmoddi4
                0x00000000        0x0 c:/renesas/ra/e2studio_v2023-07_fsp_v4.6.0/toolchains/gcc_arm/arm-gnu-toolchain-12.2.mpacbti-rel1-mingw-w64-i686-arm-none-eabi/bin/../lib/gcc/arm-none-eabi/12.2.1/thumb/v8-m.main+fp/hard\libgcc.a(_udivmoddi4.o)
 .data          0x00000000        0x0 c:/renesas/ra/e2studio_v2023-07_fsp_v4.6.0/toolchains/gcc_arm/arm-gnu-toolchain-12.2.mpacbti-rel1-mingw-w64-i686-arm-none-eabi/bin/../lib/gcc/arm-none-eabi/12.2.1/thumb/v8-m.main+fp/hard\libgcc.a(_dvmd_tls.o)
 .bss           0x00000000        0x0 c:/renesas/ra/e2studio_v2023-07_fsp_v4.6.0/toolchains/gcc_arm/arm-gnu-toolchain-12.2.mpacbti-rel1-mingw-w64-i686-arm-none-eabi/bin/../lib/gcc/arm-none-eabi/12.2.1/thumb/v8-m.main+fp/hard\libgcc.a(_dvmd_tls.o)
 .text          0x00000000        0x0 c:/renesas/ra/e2studio_v2023-07_fsp_v4.6.0/toolchains/gcc_arm/arm-gnu-toolchain-12.2.mpacbti-rel1-mingw-w64-i686-arm-none-eabi/bin/../lib/gcc/arm-none-eabi/12.2.1/thumb/v8-m.main+fp/hard\libg_nano.a(libc_a-exit.o)
 .data          0x00000000        0x0 c:/renesas/ra/e2studio_v2023-07_fsp_v4.6.0/toolchains/gcc_arm/arm-gnu-toolchain-12.2.mpacbti-rel1-mingw-w64-i686-arm-none-eabi/bin/../lib/gcc/arm-none-eabi/12.2.1/thumb/v8-m.main+fp/hard\libg_nano.a(libc_a-exit.o)
 .bss           0x00000000        0x0 c:/renesas/ra/e2studio_v2023-07_fsp_v4.6.0/toolchains/gcc_arm/arm-gnu-toolchain-12.2.mpacbti-rel1-mingw-w64-i686-arm-none-eabi/bin/../lib/gcc/arm-none-eabi/12.2.1/thumb/v8-m.main+fp/hard\libg_nano.a(libc_a-exit.o)
 .text.exit     0x00000000       0x24 c:/renesas/ra/e2studio_v2023-07_fsp_v4.6.0/toolchains/gcc_arm/arm-gnu-toolchain-12.2.mpacbti-rel1-mingw-w64-i686-arm-none-eabi/bin/../lib/gcc/arm-none-eabi/12.2.1/thumb/v8-m.main+fp/hard\libg_nano.a(libc_a-exit.o)
 .debug_frame   0x00000000       0x28 c:/renesas/ra/e2studio_v2023-07_fsp_v4.6.0/toolchains/gcc_arm/arm-gnu-toolchain-12.2.mpacbti-rel1-mingw-w64-i686-arm-none-eabi/bin/../lib/gcc/arm-none-eabi/12.2.1/thumb/v8-m.main+fp/hard\libg_nano.a(libc_a-exit.o)
 .ARM.attributes
                0x00000000       0x38 c:/renesas/ra/e2studio_v2023-07_fsp_v4.6.0/toolchains/gcc_arm/arm-gnu-toolchain-12.2.mpacbti-rel1-mingw-w64-i686-arm-none-eabi/bin/../lib/gcc/arm-none-eabi/12.2.1/thumb/v8-m.main+fp/hard\libg_nano.a(libc_a-exit.o)
 .text          0x00000000        0x0 c:/renesas/ra/e2studio_v2023-07_fsp_v4.6.0/toolchains/gcc_arm/arm-gnu-toolchain-12.2.mpacbti-rel1-mingw-w64-i686-arm-none-eabi/bin/../lib/gcc/arm-none-eabi/12.2.1/thumb/v8-m.main+fp/hard\libg_nano.a(libc_a-itoa.o)
 .data          0x00000000        0x0 c:/renesas/ra/e2studio_v2023-07_fsp_v4.6.0/toolchains/gcc_arm/arm-gnu-toolchain-12.2.mpacbti-rel1-mingw-w64-i686-arm-none-eabi/bin/../lib/gcc/arm-none-eabi/12.2.1/thumb/v8-m.main+fp/hard\libg_nano.a(libc_a-itoa.o)
 .bss           0x00000000        0x0 c:/renesas/ra/e2studio_v2023-07_fsp_v4.6.0/toolchains/gcc_arm/arm-gnu-toolchain-12.2.mpacbti-rel1-mingw-w64-i686-arm-none-eabi/bin/../lib/gcc/arm-none-eabi/12.2.1/thumb/v8-m.main+fp/hard\libg_nano.a(libc_a-itoa.o)
 .text.itoa     0x00000000        0x4 c:/renesas/ra/e2studio_v2023-07_fsp_v4.6.0/toolchains/gcc_arm/arm-gnu-toolchain-12.2.mpacbti-rel1-mingw-w64-i686-arm-none-eabi/bin/../lib/gcc/arm-none-eabi/12.2.1/thumb/v8-m.main+fp/hard\libg_nano.a(libc_a-itoa.o)
 .text          0x00000000        0x0 c:/renesas/ra/e2studio_v2023-07_fsp_v4.6.0/toolchains/gcc_arm/arm-gnu-toolchain-12.2.mpacbti-rel1-mingw-w64-i686-arm-none-eabi/bin/../lib/gcc/arm-none-eabi/12.2.1/thumb/v8-m.main+fp/hard\libg_nano.a(libc_a-strtol.o)
 .data          0x00000000        0x0 c:/renesas/ra/e2studio_v2023-07_fsp_v4.6.0/toolchains/gcc_arm/arm-gnu-toolchain-12.2.mpacbti-rel1-mingw-w64-i686-arm-none-eabi/bin/../lib/gcc/arm-none-eabi/12.2.1/thumb/v8-m.main+fp/hard\libg_nano.a(libc_a-strtol.o)
 .bss           0x00000000        0x0 c:/renesas/ra/e2studio_v2023-07_fsp_v4.6.0/toolchains/gcc_arm/arm-gnu-toolchain-12.2.mpacbti-rel1-mingw-w64-i686-arm-none-eabi/bin/../lib/gcc/arm-none-eabi/12.2.1/thumb/v8-m.main+fp/hard\libg_nano.a(libc_a-strtol.o)
 .text._strtol_r
                0x00000000        0x4 c:/renesas/ra/e2studio_v2023-07_fsp_v4.6.0/toolchains/gcc_arm/arm-gnu-toolchain-12.2.mpacbti-rel1-mingw-w64-i686-arm-none-eabi/bin/../lib/gcc/arm-none-eabi/12.2.1/thumb/v8-m.main+fp/hard\libg_nano.a(libc_a-strtol.o)
 .text.strtol_l
                0x00000000       0x14 c:/renesas/ra/e2studio_v2023-07_fsp_v4.6.0/toolchains/gcc_arm/arm-gnu-toolchain-12.2.mpacbti-rel1-mingw-w64-i686-arm-none-eabi/bin/../lib/gcc/arm-none-eabi/12.2.1/thumb/v8-m.main+fp/hard\libg_nano.a(libc_a-strtol.o)
 .text          0x00000000        0x0 c:/renesas/ra/e2studio_v2023-07_fsp_v4.6.0/toolchains/gcc_arm/arm-gnu-toolchain-12.2.mpacbti-rel1-mingw-w64-i686-arm-none-eabi/bin/../lib/gcc/arm-none-eabi/12.2.1/thumb/v8-m.main+fp/hard\libg_nano.a(libc_a-utoa.o)
 .data          0x00000000        0x0 c:/renesas/ra/e2studio_v2023-07_fsp_v4.6.0/toolchains/gcc_arm/arm-gnu-toolchain-12.2.mpacbti-rel1-mingw-w64-i686-arm-none-eabi/bin/../lib/gcc/arm-none-eabi/12.2.1/thumb/v8-m.main+fp/hard\libg_nano.a(libc_a-utoa.o)
 .bss           0x00000000        0x0 c:/renesas/ra/e2studio_v2023-07_fsp_v4.6.0/toolchains/gcc_arm/arm-gnu-toolchain-12.2.mpacbti-rel1-mingw-w64-i686-arm-none-eabi/bin/../lib/gcc/arm-none-eabi/12.2.1/thumb/v8-m.main+fp/hard\libg_nano.a(libc_a-utoa.o)
 .text.utoa     0x00000000        0x4 c:/renesas/ra/e2studio_v2023-07_fsp_v4.6.0/toolchains/gcc_arm/arm-gnu-toolchain-12.2.mpacbti-rel1-mingw-w64-i686-arm-none-eabi/bin/../lib/gcc/arm-none-eabi/12.2.1/thumb/v8-m.main+fp/hard\libg_nano.a(libc_a-utoa.o)
 .text          0x00000000        0x0 c:/renesas/ra/e2studio_v2023-07_fsp_v4.6.0/toolchains/gcc_arm/arm-gnu-toolchain-12.2.mpacbti-rel1-mingw-w64-i686-arm-none-eabi/bin/../lib/gcc/arm-none-eabi/12.2.1/thumb/v8-m.main+fp/hard\libg_nano.a(libc_a-ctype_.o)
 .data          0x00000000        0x0 c:/renesas/ra/e2studio_v2023-07_fsp_v4.6.0/toolchains/gcc_arm/arm-gnu-toolchain-12.2.mpacbti-rel1-mingw-w64-i686-arm-none-eabi/bin/../lib/gcc/arm-none-eabi/12.2.1/thumb/v8-m.main+fp/hard\libg_nano.a(libc_a-ctype_.o)
 .bss           0x00000000        0x0 c:/renesas/ra/e2studio_v2023-07_fsp_v4.6.0/toolchains/gcc_arm/arm-gnu-toolchain-12.2.mpacbti-rel1-mingw-w64-i686-arm-none-eabi/bin/../lib/gcc/arm-none-eabi/12.2.1/thumb/v8-m.main+fp/hard\libg_nano.a(libc_a-ctype_.o)
 .text          0x00000000        0x0 c:/renesas/ra/e2studio_v2023-07_fsp_v4.6.0/toolchains/gcc_arm/arm-gnu-toolchain-12.2.mpacbti-rel1-mingw-w64-i686-arm-none-eabi/bin/../lib/gcc/arm-none-eabi/12.2.1/thumb/v8-m.main+fp/hard\libg_nano.a(libc_a-findfp.o)
 .data          0x00000000        0x0 c:/renesas/ra/e2studio_v2023-07_fsp_v4.6.0/toolchains/gcc_arm/arm-gnu-toolchain-12.2.mpacbti-rel1-mingw-w64-i686-arm-none-eabi/bin/../lib/gcc/arm-none-eabi/12.2.1/thumb/v8-m.main+fp/hard\libg_nano.a(libc_a-findfp.o)
 .bss           0x00000000        0x0 c:/renesas/ra/e2studio_v2023-07_fsp_v4.6.0/toolchains/gcc_arm/arm-gnu-toolchain-12.2.mpacbti-rel1-mingw-w64-i686-arm-none-eabi/bin/../lib/gcc/arm-none-eabi/12.2.1/thumb/v8-m.main+fp/hard\libg_nano.a(libc_a-findfp.o)
 .text.std      0x00000000       0x6c c:/renesas/ra/e2studio_v2023-07_fsp_v4.6.0/toolchains/gcc_arm/arm-gnu-toolchain-12.2.mpacbti-rel1-mingw-w64-i686-arm-none-eabi/bin/../lib/gcc/arm-none-eabi/12.2.1/thumb/v8-m.main+fp/hard\libg_nano.a(libc_a-findfp.o)
 .text.stdio_exit_handler
                0x00000000       0x18 c:/renesas/ra/e2studio_v2023-07_fsp_v4.6.0/toolchains/gcc_arm/arm-gnu-toolchain-12.2.mpacbti-rel1-mingw-w64-i686-arm-none-eabi/bin/../lib/gcc/arm-none-eabi/12.2.1/thumb/v8-m.main+fp/hard\libg_nano.a(libc_a-findfp.o)
 .text.cleanup_stdio
                0x00000000       0x40 c:/renesas/ra/e2studio_v2023-07_fsp_v4.6.0/toolchains/gcc_arm/arm-gnu-toolchain-12.2.mpacbti-rel1-mingw-w64-i686-arm-none-eabi/bin/../lib/gcc/arm-none-eabi/12.2.1/thumb/v8-m.main+fp/hard\libg_nano.a(libc_a-findfp.o)
 .text.__fp_lock
                0x00000000       0x18 c:/renesas/ra/e2studio_v2023-07_fsp_v4.6.0/toolchains/gcc_arm/arm-gnu-toolchain-12.2.mpacbti-rel1-mingw-w64-i686-arm-none-eabi/bin/../lib/gcc/arm-none-eabi/12.2.1/thumb/v8-m.main+fp/hard\libg_nano.a(libc_a-findfp.o)
 .text.__fp_unlock
                0x00000000       0x18 c:/renesas/ra/e2studio_v2023-07_fsp_v4.6.0/toolchains/gcc_arm/arm-gnu-toolchain-12.2.mpacbti-rel1-mingw-w64-i686-arm-none-eabi/bin/../lib/gcc/arm-none-eabi/12.2.1/thumb/v8-m.main+fp/hard\libg_nano.a(libc_a-findfp.o)
 .text.global_stdio_init.part.0
                0x00000000       0x3c c:/renesas/ra/e2studio_v2023-07_fsp_v4.6.0/toolchains/gcc_arm/arm-gnu-toolchain-12.2.mpacbti-rel1-mingw-w64-i686-arm-none-eabi/bin/../lib/gcc/arm-none-eabi/12.2.1/thumb/v8-m.main+fp/hard\libg_nano.a(libc_a-findfp.o)
 .text.__sfp_lock_acquire
                0x00000000        0xc c:/renesas/ra/e2studio_v2023-07_fsp_v4.6.0/toolchains/gcc_arm/arm-gnu-toolchain-12.2.mpacbti-rel1-mingw-w64-i686-arm-none-eabi/bin/../lib/gcc/arm-none-eabi/12.2.1/thumb/v8-m.main+fp/hard\libg_nano.a(libc_a-findfp.o)
 .text.__sfp_lock_release
                0x00000000        0xc c:/renesas/ra/e2studio_v2023-07_fsp_v4.6.0/toolchains/gcc_arm/arm-gnu-toolchain-12.2.mpacbti-rel1-mingw-w64-i686-arm-none-eabi/bin/../lib/gcc/arm-none-eabi/12.2.1/thumb/v8-m.main+fp/hard\libg_nano.a(libc_a-findfp.o)
 .text.__sfp    0x00000000       0xa4 c:/renesas/ra/e2studio_v2023-07_fsp_v4.6.0/toolchains/gcc_arm/arm-gnu-toolchain-12.2.mpacbti-rel1-mingw-w64-i686-arm-none-eabi/bin/../lib/gcc/arm-none-eabi/12.2.1/thumb/v8-m.main+fp/hard\libg_nano.a(libc_a-findfp.o)
 .text.__sinit  0x00000000       0x30 c:/renesas/ra/e2studio_v2023-07_fsp_v4.6.0/toolchains/gcc_arm/arm-gnu-toolchain-12.2.mpacbti-rel1-mingw-w64-i686-arm-none-eabi/bin/../lib/gcc/arm-none-eabi/12.2.1/thumb/v8-m.main+fp/hard\libg_nano.a(libc_a-findfp.o)
 .text.__fp_lock_all
                0x00000000       0x1c c:/renesas/ra/e2studio_v2023-07_fsp_v4.6.0/toolchains/gcc_arm/arm-gnu-toolchain-12.2.mpacbti-rel1-mingw-w64-i686-arm-none-eabi/bin/../lib/gcc/arm-none-eabi/12.2.1/thumb/v8-m.main+fp/hard\libg_nano.a(libc_a-findfp.o)
 .text.__fp_unlock_all
                0x00000000       0x1c c:/renesas/ra/e2studio_v2023-07_fsp_v4.6.0/toolchains/gcc_arm/arm-gnu-toolchain-12.2.mpacbti-rel1-mingw-w64-i686-arm-none-eabi/bin/../lib/gcc/arm-none-eabi/12.2.1/thumb/v8-m.main+fp/hard\libg_nano.a(libc_a-findfp.o)
 .data.__sglue  0x00000000        0xc c:/renesas/ra/e2studio_v2023-07_fsp_v4.6.0/toolchains/gcc_arm/arm-gnu-toolchain-12.2.mpacbti-rel1-mingw-w64-i686-arm-none-eabi/bin/../lib/gcc/arm-none-eabi/12.2.1/thumb/v8-m.main+fp/hard\libg_nano.a(libc_a-findfp.o)
 .bss.__stdio_exit_handler
                0x00000000        0x4 c:/renesas/ra/e2studio_v2023-07_fsp_v4.6.0/toolchains/gcc_arm/arm-gnu-toolchain-12.2.mpacbti-rel1-mingw-w64-i686-arm-none-eabi/bin/../lib/gcc/arm-none-eabi/12.2.1/thumb/v8-m.main+fp/hard\libg_nano.a(libc_a-findfp.o)
 .text          0x00000000        0x0 c:/renesas/ra/e2studio_v2023-07_fsp_v4.6.0/toolchains/gcc_arm/arm-gnu-toolchain-12.2.mpacbti-rel1-mingw-w64-i686-arm-none-eabi/bin/../lib/gcc/arm-none-eabi/12.2.1/thumb/v8-m.main+fp/hard\libg_nano.a(libc_a-fwalk.o)
 .data          0x00000000        0x0 c:/renesas/ra/e2studio_v2023-07_fsp_v4.6.0/toolchains/gcc_arm/arm-gnu-toolchain-12.2.mpacbti-rel1-mingw-w64-i686-arm-none-eabi/bin/../lib/gcc/arm-none-eabi/12.2.1/thumb/v8-m.main+fp/hard\libg_nano.a(libc_a-fwalk.o)
 .bss           0x00000000        0x0 c:/renesas/ra/e2studio_v2023-07_fsp_v4.6.0/toolchains/gcc_arm/arm-gnu-toolchain-12.2.mpacbti-rel1-mingw-w64-i686-arm-none-eabi/bin/../lib/gcc/arm-none-eabi/12.2.1/thumb/v8-m.main+fp/hard\libg_nano.a(libc_a-fwalk.o)
 .text._fwalk_sglue
                0x00000000       0x3c c:/renesas/ra/e2studio_v2023-07_fsp_v4.6.0/toolchains/gcc_arm/arm-gnu-toolchain-12.2.mpacbti-rel1-mingw-w64-i686-arm-none-eabi/bin/../lib/gcc/arm-none-eabi/12.2.1/thumb/v8-m.main+fp/hard\libg_nano.a(libc_a-fwalk.o)
 .debug_frame   0x00000000       0x34 c:/renesas/ra/e2studio_v2023-07_fsp_v4.6.0/toolchains/gcc_arm/arm-gnu-toolchain-12.2.mpacbti-rel1-mingw-w64-i686-arm-none-eabi/bin/../lib/gcc/arm-none-eabi/12.2.1/thumb/v8-m.main+fp/hard\libg_nano.a(libc_a-fwalk.o)
 .ARM.attributes
                0x00000000       0x38 c:/renesas/ra/e2studio_v2023-07_fsp_v4.6.0/toolchains/gcc_arm/arm-gnu-toolchain-12.2.mpacbti-rel1-mingw-w64-i686-arm-none-eabi/bin/../lib/gcc/arm-none-eabi/12.2.1/thumb/v8-m.main+fp/hard\libg_nano.a(libc_a-fwalk.o)
 .text          0x00000000        0x0 c:/renesas/ra/e2studio_v2023-07_fsp_v4.6.0/toolchains/gcc_arm/arm-gnu-toolchain-12.2.mpacbti-rel1-mingw-w64-i686-arm-none-eabi/bin/../lib/gcc/arm-none-eabi/12.2.1/thumb/v8-m.main+fp/hard\libg_nano.a(libc_a-stdio.o)
 .data          0x00000000        0x0 c:/renesas/ra/e2studio_v2023-07_fsp_v4.6.0/toolchains/gcc_arm/arm-gnu-toolchain-12.2.mpacbti-rel1-mingw-w64-i686-arm-none-eabi/bin/../lib/gcc/arm-none-eabi/12.2.1/thumb/v8-m.main+fp/hard\libg_nano.a(libc_a-stdio.o)
 .bss           0x00000000        0x0 c:/renesas/ra/e2studio_v2023-07_fsp_v4.6.0/toolchains/gcc_arm/arm-gnu-toolchain-12.2.mpacbti-rel1-mingw-w64-i686-arm-none-eabi/bin/../lib/gcc/arm-none-eabi/12.2.1/thumb/v8-m.main+fp/hard\libg_nano.a(libc_a-stdio.o)
 .text.__sread  0x00000000       0x22 c:/renesas/ra/e2studio_v2023-07_fsp_v4.6.0/toolchains/gcc_arm/arm-gnu-toolchain-12.2.mpacbti-rel1-mingw-w64-i686-arm-none-eabi/bin/../lib/gcc/arm-none-eabi/12.2.1/thumb/v8-m.main+fp/hard\libg_nano.a(libc_a-stdio.o)
 .text.__seofread
                0x00000000        0x4 c:/renesas/ra/e2studio_v2023-07_fsp_v4.6.0/toolchains/gcc_arm/arm-gnu-toolchain-12.2.mpacbti-rel1-mingw-w64-i686-arm-none-eabi/bin/../lib/gcc/arm-none-eabi/12.2.1/thumb/v8-m.main+fp/hard\libg_nano.a(libc_a-stdio.o)
 .text.__swrite
                0x00000000       0x38 c:/renesas/ra/e2studio_v2023-07_fsp_v4.6.0/toolchains/gcc_arm/arm-gnu-toolchain-12.2.mpacbti-rel1-mingw-w64-i686-arm-none-eabi/bin/../lib/gcc/arm-none-eabi/12.2.1/thumb/v8-m.main+fp/hard\libg_nano.a(libc_a-stdio.o)
 .text.__sseek  0x00000000       0x24 c:/renesas/ra/e2studio_v2023-07_fsp_v4.6.0/toolchains/gcc_arm/arm-gnu-toolchain-12.2.mpacbti-rel1-mingw-w64-i686-arm-none-eabi/bin/../lib/gcc/arm-none-eabi/12.2.1/thumb/v8-m.main+fp/hard\libg_nano.a(libc_a-stdio.o)
 .text.__sclose
                0x00000000        0x8 c:/renesas/ra/e2studio_v2023-07_fsp_v4.6.0/toolchains/gcc_arm/arm-gnu-toolchain-12.2.mpacbti-rel1-mingw-w64-i686-arm-none-eabi/bin/../lib/gcc/arm-none-eabi/12.2.1/thumb/v8-m.main+fp/hard\libg_nano.a(libc_a-stdio.o)
 .debug_frame   0x00000000       0x88 c:/renesas/ra/e2studio_v2023-07_fsp_v4.6.0/toolchains/gcc_arm/arm-gnu-toolchain-12.2.mpacbti-rel1-mingw-w64-i686-arm-none-eabi/bin/../lib/gcc/arm-none-eabi/12.2.1/thumb/v8-m.main+fp/hard\libg_nano.a(libc_a-stdio.o)
 .ARM.attributes
                0x00000000       0x38 c:/renesas/ra/e2studio_v2023-07_fsp_v4.6.0/toolchains/gcc_arm/arm-gnu-toolchain-12.2.mpacbti-rel1-mingw-w64-i686-arm-none-eabi/bin/../lib/gcc/arm-none-eabi/12.2.1/thumb/v8-m.main+fp/hard\libg_nano.a(libc_a-stdio.o)
 .text          0x00000000        0x0 c:/renesas/ra/e2studio_v2023-07_fsp_v4.6.0/toolchains/gcc_arm/arm-gnu-toolchain-12.2.mpacbti-rel1-mingw-w64-i686-arm-none-eabi/bin/../lib/gcc/arm-none-eabi/12.2.1/thumb/v8-m.main+fp/hard\libg_nano.a(libc_a-memset.o)
 .data          0x00000000        0x0 c:/renesas/ra/e2studio_v2023-07_fsp_v4.6.0/toolchains/gcc_arm/arm-gnu-toolchain-12.2.mpacbti-rel1-mingw-w64-i686-arm-none-eabi/bin/../lib/gcc/arm-none-eabi/12.2.1/thumb/v8-m.main+fp/hard\libg_nano.a(libc_a-memset.o)
 .bss           0x00000000        0x0 c:/renesas/ra/e2studio_v2023-07_fsp_v4.6.0/toolchains/gcc_arm/arm-gnu-toolchain-12.2.mpacbti-rel1-mingw-w64-i686-arm-none-eabi/bin/../lib/gcc/arm-none-eabi/12.2.1/thumb/v8-m.main+fp/hard\libg_nano.a(libc_a-memset.o)
 .text          0x00000000        0x0 c:/renesas/ra/e2studio_v2023-07_fsp_v4.6.0/toolchains/gcc_arm/arm-gnu-toolchain-12.2.mpacbti-rel1-mingw-w64-i686-arm-none-eabi/bin/../lib/gcc/arm-none-eabi/12.2.1/thumb/v8-m.main+fp/hard\libg_nano.a(libc_a-strncmp.o)
 .data          0x00000000        0x0 c:/renesas/ra/e2studio_v2023-07_fsp_v4.6.0/toolchains/gcc_arm/arm-gnu-toolchain-12.2.mpacbti-rel1-mingw-w64-i686-arm-none-eabi/bin/../lib/gcc/arm-none-eabi/12.2.1/thumb/v8-m.main+fp/hard\libg_nano.a(libc_a-strncmp.o)
 .bss           0x00000000        0x0 c:/renesas/ra/e2studio_v2023-07_fsp_v4.6.0/toolchains/gcc_arm/arm-gnu-toolchain-12.2.mpacbti-rel1-mingw-w64-i686-arm-none-eabi/bin/../lib/gcc/arm-none-eabi/12.2.1/thumb/v8-m.main+fp/hard\libg_nano.a(libc_a-strncmp.o)
 .text          0x00000000        0x0 c:/renesas/ra/e2studio_v2023-07_fsp_v4.6.0/toolchains/gcc_arm/arm-gnu-toolchain-12.2.mpacbti-rel1-mingw-w64-i686-arm-none-eabi/bin/../lib/gcc/arm-none-eabi/12.2.1/thumb/v8-m.main+fp/hard\libg_nano.a(libc_a-closer.o)
 .data          0x00000000        0x0 c:/renesas/ra/e2studio_v2023-07_fsp_v4.6.0/toolchains/gcc_arm/arm-gnu-toolchain-12.2.mpacbti-rel1-mingw-w64-i686-arm-none-eabi/bin/../lib/gcc/arm-none-eabi/12.2.1/thumb/v8-m.main+fp/hard\libg_nano.a(libc_a-closer.o)
 .bss           0x00000000        0x0 c:/renesas/ra/e2studio_v2023-07_fsp_v4.6.0/toolchains/gcc_arm/arm-gnu-toolchain-12.2.mpacbti-rel1-mingw-w64-i686-arm-none-eabi/bin/../lib/gcc/arm-none-eabi/12.2.1/thumb/v8-m.main+fp/hard\libg_nano.a(libc_a-closer.o)
 .text._close_r
                0x00000000       0x20 c:/renesas/ra/e2studio_v2023-07_fsp_v4.6.0/toolchains/gcc_arm/arm-gnu-toolchain-12.2.mpacbti-rel1-mingw-w64-i686-arm-none-eabi/bin/../lib/gcc/arm-none-eabi/12.2.1/thumb/v8-m.main+fp/hard\libg_nano.a(libc_a-closer.o)
 .debug_frame   0x00000000       0x2c c:/renesas/ra/e2studio_v2023-07_fsp_v4.6.0/toolchains/gcc_arm/arm-gnu-toolchain-12.2.mpacbti-rel1-mingw-w64-i686-arm-none-eabi/bin/../lib/gcc/arm-none-eabi/12.2.1/thumb/v8-m.main+fp/hard\libg_nano.a(libc_a-closer.o)
 .ARM.attributes
                0x00000000       0x38 c:/renesas/ra/e2studio_v2023-07_fsp_v4.6.0/toolchains/gcc_arm/arm-gnu-toolchain-12.2.mpacbti-rel1-mingw-w64-i686-arm-none-eabi/bin/../lib/gcc/arm-none-eabi/12.2.1/thumb/v8-m.main+fp/hard\libg_nano.a(libc_a-closer.o)
 .text          0x00000000        0x0 c:/renesas/ra/e2studio_v2023-07_fsp_v4.6.0/toolchains/gcc_arm/arm-gnu-toolchain-12.2.mpacbti-rel1-mingw-w64-i686-arm-none-eabi/bin/../lib/gcc/arm-none-eabi/12.2.1/thumb/v8-m.main+fp/hard\libg_nano.a(libc_a-reent.o)
 .data          0x00000000        0x0 c:/renesas/ra/e2studio_v2023-07_fsp_v4.6.0/toolchains/gcc_arm/arm-gnu-toolchain-12.2.mpacbti-rel1-mingw-w64-i686-arm-none-eabi/bin/../lib/gcc/arm-none-eabi/12.2.1/thumb/v8-m.main+fp/hard\libg_nano.a(libc_a-reent.o)
 .bss           0x00000000        0x0 c:/renesas/ra/e2studio_v2023-07_fsp_v4.6.0/toolchains/gcc_arm/arm-gnu-toolchain-12.2.mpacbti-rel1-mingw-w64-i686-arm-none-eabi/bin/../lib/gcc/arm-none-eabi/12.2.1/thumb/v8-m.main+fp/hard\libg_nano.a(libc_a-reent.o)
 .text._reclaim_reent
                0x00000000       0xac c:/renesas/ra/e2studio_v2023-07_fsp_v4.6.0/toolchains/gcc_arm/arm-gnu-toolchain-12.2.mpacbti-rel1-mingw-w64-i686-arm-none-eabi/bin/../lib/gcc/arm-none-eabi/12.2.1/thumb/v8-m.main+fp/hard\libg_nano.a(libc_a-reent.o)
 .bss.errno     0x00000000        0x4 c:/renesas/ra/e2studio_v2023-07_fsp_v4.6.0/toolchains/gcc_arm/arm-gnu-toolchain-12.2.mpacbti-rel1-mingw-w64-i686-arm-none-eabi/bin/../lib/gcc/arm-none-eabi/12.2.1/thumb/v8-m.main+fp/hard\libg_nano.a(libc_a-reent.o)
 .debug_frame   0x00000000       0x38 c:/renesas/ra/e2studio_v2023-07_fsp_v4.6.0/toolchains/gcc_arm/arm-gnu-toolchain-12.2.mpacbti-rel1-mingw-w64-i686-arm-none-eabi/bin/../lib/gcc/arm-none-eabi/12.2.1/thumb/v8-m.main+fp/hard\libg_nano.a(libc_a-reent.o)
 .ARM.attributes
                0x00000000       0x38 c:/renesas/ra/e2studio_v2023-07_fsp_v4.6.0/toolchains/gcc_arm/arm-gnu-toolchain-12.2.mpacbti-rel1-mingw-w64-i686-arm-none-eabi/bin/../lib/gcc/arm-none-eabi/12.2.1/thumb/v8-m.main+fp/hard\libg_nano.a(libc_a-reent.o)
 .text          0x00000000        0x0 c:/renesas/ra/e2studio_v2023-07_fsp_v4.6.0/toolchains/gcc_arm/arm-gnu-toolchain-12.2.mpacbti-rel1-mingw-w64-i686-arm-none-eabi/bin/../lib/gcc/arm-none-eabi/12.2.1/thumb/v8-m.main+fp/hard\libg_nano.a(libc_a-impure.o)
 .data          0x00000000        0x0 c:/renesas/ra/e2studio_v2023-07_fsp_v4.6.0/toolchains/gcc_arm/arm-gnu-toolchain-12.2.mpacbti-rel1-mingw-w64-i686-arm-none-eabi/bin/../lib/gcc/arm-none-eabi/12.2.1/thumb/v8-m.main+fp/hard\libg_nano.a(libc_a-impure.o)
 .bss           0x00000000        0x0 c:/renesas/ra/e2studio_v2023-07_fsp_v4.6.0/toolchains/gcc_arm/arm-gnu-toolchain-12.2.mpacbti-rel1-mingw-w64-i686-arm-none-eabi/bin/../lib/gcc/arm-none-eabi/12.2.1/thumb/v8-m.main+fp/hard\libg_nano.a(libc_a-impure.o)
 .text          0x00000000        0x0 c:/renesas/ra/e2studio_v2023-07_fsp_v4.6.0/toolchains/gcc_arm/arm-gnu-toolchain-12.2.mpacbti-rel1-mingw-w64-i686-arm-none-eabi/bin/../lib/gcc/arm-none-eabi/12.2.1/thumb/v8-m.main+fp/hard\libg_nano.a(libc_a-lseekr.o)
 .data          0x00000000        0x0 c:/renesas/ra/e2studio_v2023-07_fsp_v4.6.0/toolchains/gcc_arm/arm-gnu-toolchain-12.2.mpacbti-rel1-mingw-w64-i686-arm-none-eabi/bin/../lib/gcc/arm-none-eabi/12.2.1/thumb/v8-m.main+fp/hard\libg_nano.a(libc_a-lseekr.o)
 .bss           0x00000000        0x0 c:/renesas/ra/e2studio_v2023-07_fsp_v4.6.0/toolchains/gcc_arm/arm-gnu-toolchain-12.2.mpacbti-rel1-mingw-w64-i686-arm-none-eabi/bin/../lib/gcc/arm-none-eabi/12.2.1/thumb/v8-m.main+fp/hard\libg_nano.a(libc_a-lseekr.o)
 .text._lseek_r
                0x00000000       0x24 c:/renesas/ra/e2studio_v2023-07_fsp_v4.6.0/toolchains/gcc_arm/arm-gnu-toolchain-12.2.mpacbti-rel1-mingw-w64-i686-arm-none-eabi/bin/../lib/gcc/arm-none-eabi/12.2.1/thumb/v8-m.main+fp/hard\libg_nano.a(libc_a-lseekr.o)
 .debug_frame   0x00000000       0x2c c:/renesas/ra/e2studio_v2023-07_fsp_v4.6.0/toolchains/gcc_arm/arm-gnu-toolchain-12.2.mpacbti-rel1-mingw-w64-i686-arm-none-eabi/bin/../lib/gcc/arm-none-eabi/12.2.1/thumb/v8-m.main+fp/hard\libg_nano.a(libc_a-lseekr.o)
 .ARM.attributes
                0x00000000       0x38 c:/renesas/ra/e2studio_v2023-07_fsp_v4.6.0/toolchains/gcc_arm/arm-gnu-toolchain-12.2.mpacbti-rel1-mingw-w64-i686-arm-none-eabi/bin/../lib/gcc/arm-none-eabi/12.2.1/thumb/v8-m.main+fp/hard\libg_nano.a(libc_a-lseekr.o)
 .text          0x00000000        0x0 c:/renesas/ra/e2studio_v2023-07_fsp_v4.6.0/toolchains/gcc_arm/arm-gnu-toolchain-12.2.mpacbti-rel1-mingw-w64-i686-arm-none-eabi/bin/../lib/gcc/arm-none-eabi/12.2.1/thumb/v8-m.main+fp/hard\libg_nano.a(libc_a-readr.o)
 .data          0x00000000        0x0 c:/renesas/ra/e2studio_v2023-07_fsp_v4.6.0/toolchains/gcc_arm/arm-gnu-toolchain-12.2.mpacbti-rel1-mingw-w64-i686-arm-none-eabi/bin/../lib/gcc/arm-none-eabi/12.2.1/thumb/v8-m.main+fp/hard\libg_nano.a(libc_a-readr.o)
 .bss           0x00000000        0x0 c:/renesas/ra/e2studio_v2023-07_fsp_v4.6.0/toolchains/gcc_arm/arm-gnu-toolchain-12.2.mpacbti-rel1-mingw-w64-i686-arm-none-eabi/bin/../lib/gcc/arm-none-eabi/12.2.1/thumb/v8-m.main+fp/hard\libg_nano.a(libc_a-readr.o)
 .text._read_r  0x00000000       0x24 c:/renesas/ra/e2studio_v2023-07_fsp_v4.6.0/toolchains/gcc_arm/arm-gnu-toolchain-12.2.mpacbti-rel1-mingw-w64-i686-arm-none-eabi/bin/../lib/gcc/arm-none-eabi/12.2.1/thumb/v8-m.main+fp/hard\libg_nano.a(libc_a-readr.o)
 .debug_frame   0x00000000       0x2c c:/renesas/ra/e2studio_v2023-07_fsp_v4.6.0/toolchains/gcc_arm/arm-gnu-toolchain-12.2.mpacbti-rel1-mingw-w64-i686-arm-none-eabi/bin/../lib/gcc/arm-none-eabi/12.2.1/thumb/v8-m.main+fp/hard\libg_nano.a(libc_a-readr.o)
 .ARM.attributes
                0x00000000       0x38 c:/renesas/ra/e2studio_v2023-07_fsp_v4.6.0/toolchains/gcc_arm/arm-gnu-toolchain-12.2.mpacbti-rel1-mingw-w64-i686-arm-none-eabi/bin/../lib/gcc/arm-none-eabi/12.2.1/thumb/v8-m.main+fp/hard\libg_nano.a(libc_a-readr.o)
 .text          0x00000000        0x0 c:/renesas/ra/e2studio_v2023-07_fsp_v4.6.0/toolchains/gcc_arm/arm-gnu-toolchain-12.2.mpacbti-rel1-mingw-w64-i686-arm-none-eabi/bin/../lib/gcc/arm-none-eabi/12.2.1/thumb/v8-m.main+fp/hard\libg_nano.a(libc_a-writer.o)
 .data          0x00000000        0x0 c:/renesas/ra/e2studio_v2023-07_fsp_v4.6.0/toolchains/gcc_arm/arm-gnu-toolchain-12.2.mpacbti-rel1-mingw-w64-i686-arm-none-eabi/bin/../lib/gcc/arm-none-eabi/12.2.1/thumb/v8-m.main+fp/hard\libg_nano.a(libc_a-writer.o)
 .bss           0x00000000        0x0 c:/renesas/ra/e2studio_v2023-07_fsp_v4.6.0/toolchains/gcc_arm/arm-gnu-toolchain-12.2.mpacbti-rel1-mingw-w64-i686-arm-none-eabi/bin/../lib/gcc/arm-none-eabi/12.2.1/thumb/v8-m.main+fp/hard\libg_nano.a(libc_a-writer.o)
 .text._write_r
                0x00000000       0x24 c:/renesas/ra/e2studio_v2023-07_fsp_v4.6.0/toolchains/gcc_arm/arm-gnu-toolchain-12.2.mpacbti-rel1-mingw-w64-i686-arm-none-eabi/bin/../lib/gcc/arm-none-eabi/12.2.1/thumb/v8-m.main+fp/hard\libg_nano.a(libc_a-writer.o)
 .debug_frame   0x00000000       0x2c c:/renesas/ra/e2studio_v2023-07_fsp_v4.6.0/toolchains/gcc_arm/arm-gnu-toolchain-12.2.mpacbti-rel1-mingw-w64-i686-arm-none-eabi/bin/../lib/gcc/arm-none-eabi/12.2.1/thumb/v8-m.main+fp/hard\libg_nano.a(libc_a-writer.o)
 .ARM.attributes
                0x00000000       0x38 c:/renesas/ra/e2studio_v2023-07_fsp_v4.6.0/toolchains/gcc_arm/arm-gnu-toolchain-12.2.mpacbti-rel1-mingw-w64-i686-arm-none-eabi/bin/../lib/gcc/arm-none-eabi/12.2.1/thumb/v8-m.main+fp/hard\libg_nano.a(libc_a-writer.o)
 .text          0x00000000        0x0 c:/renesas/ra/e2studio_v2023-07_fsp_v4.6.0/toolchains/gcc_arm/arm-gnu-toolchain-12.2.mpacbti-rel1-mingw-w64-i686-arm-none-eabi/bin/../lib/gcc/arm-none-eabi/12.2.1/thumb/v8-m.main+fp/hard\libg_nano.a(libc_a-errno.o)
 .data          0x00000000        0x0 c:/renesas/ra/e2studio_v2023-07_fsp_v4.6.0/toolchains/gcc_arm/arm-gnu-toolchain-12.2.mpacbti-rel1-mingw-w64-i686-arm-none-eabi/bin/../lib/gcc/arm-none-eabi/12.2.1/thumb/v8-m.main+fp/hard\libg_nano.a(libc_a-errno.o)
 .bss           0x00000000        0x0 c:/renesas/ra/e2studio_v2023-07_fsp_v4.6.0/toolchains/gcc_arm/arm-gnu-toolchain-12.2.mpacbti-rel1-mingw-w64-i686-arm-none-eabi/bin/../lib/gcc/arm-none-eabi/12.2.1/thumb/v8-m.main+fp/hard\libg_nano.a(libc_a-errno.o)
 .text          0x00000000        0x0 c:/renesas/ra/e2studio_v2023-07_fsp_v4.6.0/toolchains/gcc_arm/arm-gnu-toolchain-12.2.mpacbti-rel1-mingw-w64-i686-arm-none-eabi/bin/../lib/gcc/arm-none-eabi/12.2.1/thumb/v8-m.main+fp/hard\libg_nano.a(libc_a-init.o)
 .data          0x00000000        0x0 c:/renesas/ra/e2studio_v2023-07_fsp_v4.6.0/toolchains/gcc_arm/arm-gnu-toolchain-12.2.mpacbti-rel1-mingw-w64-i686-arm-none-eabi/bin/../lib/gcc/arm-none-eabi/12.2.1/thumb/v8-m.main+fp/hard\libg_nano.a(libc_a-init.o)
 .bss           0x00000000        0x0 c:/renesas/ra/e2studio_v2023-07_fsp_v4.6.0/toolchains/gcc_arm/arm-gnu-toolchain-12.2.mpacbti-rel1-mingw-w64-i686-arm-none-eabi/bin/../lib/gcc/arm-none-eabi/12.2.1/thumb/v8-m.main+fp/hard\libg_nano.a(libc_a-init.o)
 .text.__libc_init_array
                0x00000000       0x48 c:/renesas/ra/e2studio_v2023-07_fsp_v4.6.0/toolchains/gcc_arm/arm-gnu-toolchain-12.2.mpacbti-rel1-mingw-w64-i686-arm-none-eabi/bin/../lib/gcc/arm-none-eabi/12.2.1/thumb/v8-m.main+fp/hard\libg_nano.a(libc_a-init.o)
 .debug_frame   0x00000000       0x2c c:/renesas/ra/e2studio_v2023-07_fsp_v4.6.0/toolchains/gcc_arm/arm-gnu-toolchain-12.2.mpacbti-rel1-mingw-w64-i686-arm-none-eabi/bin/../lib/gcc/arm-none-eabi/12.2.1/thumb/v8-m.main+fp/hard\libg_nano.a(libc_a-init.o)
 .ARM.attributes
                0x00000000       0x38 c:/renesas/ra/e2studio_v2023-07_fsp_v4.6.0/toolchains/gcc_arm/arm-gnu-toolchain-12.2.mpacbti-rel1-mingw-w64-i686-arm-none-eabi/bin/../lib/gcc/arm-none-eabi/12.2.1/thumb/v8-m.main+fp/hard\libg_nano.a(libc_a-init.o)
 .text          0x00000000        0x0 c:/renesas/ra/e2studio_v2023-07_fsp_v4.6.0/toolchains/gcc_arm/arm-gnu-toolchain-12.2.mpacbti-rel1-mingw-w64-i686-arm-none-eabi/bin/../lib/gcc/arm-none-eabi/12.2.1/thumb/v8-m.main+fp/hard\libg_nano.a(libc_a-lock.o)
 .data          0x00000000        0x0 c:/renesas/ra/e2studio_v2023-07_fsp_v4.6.0/toolchains/gcc_arm/arm-gnu-toolchain-12.2.mpacbti-rel1-mingw-w64-i686-arm-none-eabi/bin/../lib/gcc/arm-none-eabi/12.2.1/thumb/v8-m.main+fp/hard\libg_nano.a(libc_a-lock.o)
 .bss           0x00000000        0x0 c:/renesas/ra/e2studio_v2023-07_fsp_v4.6.0/toolchains/gcc_arm/arm-gnu-toolchain-12.2.mpacbti-rel1-mingw-w64-i686-arm-none-eabi/bin/../lib/gcc/arm-none-eabi/12.2.1/thumb/v8-m.main+fp/hard\libg_nano.a(libc_a-lock.o)
 .text.__retarget_lock_init
                0x00000000        0x2 c:/renesas/ra/e2studio_v2023-07_fsp_v4.6.0/toolchains/gcc_arm/arm-gnu-toolchain-12.2.mpacbti-rel1-mingw-w64-i686-arm-none-eabi/bin/../lib/gcc/arm-none-eabi/12.2.1/thumb/v8-m.main+fp/hard\libg_nano.a(libc_a-lock.o)
 .text.__retarget_lock_init_recursive
                0x00000000        0x2 c:/renesas/ra/e2studio_v2023-07_fsp_v4.6.0/toolchains/gcc_arm/arm-gnu-toolchain-12.2.mpacbti-rel1-mingw-w64-i686-arm-none-eabi/bin/../lib/gcc/arm-none-eabi/12.2.1/thumb/v8-m.main+fp/hard\libg_nano.a(libc_a-lock.o)
 .text.__retarget_lock_close
                0x00000000        0x2 c:/renesas/ra/e2studio_v2023-07_fsp_v4.6.0/toolchains/gcc_arm/arm-gnu-toolchain-12.2.mpacbti-rel1-mingw-w64-i686-arm-none-eabi/bin/../lib/gcc/arm-none-eabi/12.2.1/thumb/v8-m.main+fp/hard\libg_nano.a(libc_a-lock.o)
 .text.__retarget_lock_close_recursive
                0x00000000        0x2 c:/renesas/ra/e2studio_v2023-07_fsp_v4.6.0/toolchains/gcc_arm/arm-gnu-toolchain-12.2.mpacbti-rel1-mingw-w64-i686-arm-none-eabi/bin/../lib/gcc/arm-none-eabi/12.2.1/thumb/v8-m.main+fp/hard\libg_nano.a(libc_a-lock.o)
 .text.__retarget_lock_acquire
                0x00000000        0x2 c:/renesas/ra/e2studio_v2023-07_fsp_v4.6.0/toolchains/gcc_arm/arm-gnu-toolchain-12.2.mpacbti-rel1-mingw-w64-i686-arm-none-eabi/bin/../lib/gcc/arm-none-eabi/12.2.1/thumb/v8-m.main+fp/hard\libg_nano.a(libc_a-lock.o)
 .text.__retarget_lock_acquire_recursive
                0x00000000        0x2 c:/renesas/ra/e2studio_v2023-07_fsp_v4.6.0/toolchains/gcc_arm/arm-gnu-toolchain-12.2.mpacbti-rel1-mingw-w64-i686-arm-none-eabi/bin/../lib/gcc/arm-none-eabi/12.2.1/thumb/v8-m.main+fp/hard\libg_nano.a(libc_a-lock.o)
 .text.__retarget_lock_try_acquire
                0x00000000        0x4 c:/renesas/ra/e2studio_v2023-07_fsp_v4.6.0/toolchains/gcc_arm/arm-gnu-toolchain-12.2.mpacbti-rel1-mingw-w64-i686-arm-none-eabi/bin/../lib/gcc/arm-none-eabi/12.2.1/thumb/v8-m.main+fp/hard\libg_nano.a(libc_a-lock.o)
 .text.__retarget_lock_try_acquire_recursive
                0x00000000        0x4 c:/renesas/ra/e2studio_v2023-07_fsp_v4.6.0/toolchains/gcc_arm/arm-gnu-toolchain-12.2.mpacbti-rel1-mingw-w64-i686-arm-none-eabi/bin/../lib/gcc/arm-none-eabi/12.2.1/thumb/v8-m.main+fp/hard\libg_nano.a(libc_a-lock.o)
 .text.__retarget_lock_release
                0x00000000        0x2 c:/renesas/ra/e2studio_v2023-07_fsp_v4.6.0/toolchains/gcc_arm/arm-gnu-toolchain-12.2.mpacbti-rel1-mingw-w64-i686-arm-none-eabi/bin/../lib/gcc/arm-none-eabi/12.2.1/thumb/v8-m.main+fp/hard\libg_nano.a(libc_a-lock.o)
 .text.__retarget_lock_release_recursive
                0x00000000        0x2 c:/renesas/ra/e2studio_v2023-07_fsp_v4.6.0/toolchains/gcc_arm/arm-gnu-toolchain-12.2.mpacbti-rel1-mingw-w64-i686-arm-none-eabi/bin/../lib/gcc/arm-none-eabi/12.2.1/thumb/v8-m.main+fp/hard\libg_nano.a(libc_a-lock.o)
 .bss.__lock___arc4random_mutex
                0x00000000        0x1 c:/renesas/ra/e2studio_v2023-07_fsp_v4.6.0/toolchains/gcc_arm/arm-gnu-toolchain-12.2.mpacbti-rel1-mingw-w64-i686-arm-none-eabi/bin/../lib/gcc/arm-none-eabi/12.2.1/thumb/v8-m.main+fp/hard\libg_nano.a(libc_a-lock.o)
 .bss.__lock___dd_hash_mutex
                0x00000000        0x1 c:/renesas/ra/e2studio_v2023-07_fsp_v4.6.0/toolchains/gcc_arm/arm-gnu-toolchain-12.2.mpacbti-rel1-mingw-w64-i686-arm-none-eabi/bin/../lib/gcc/arm-none-eabi/12.2.1/thumb/v8-m.main+fp/hard\libg_nano.a(libc_a-lock.o)
 .bss.__lock___tz_mutex
                0x00000000        0x1 c:/renesas/ra/e2studio_v2023-07_fsp_v4.6.0/toolchains/gcc_arm/arm-gnu-toolchain-12.2.mpacbti-rel1-mingw-w64-i686-arm-none-eabi/bin/../lib/gcc/arm-none-eabi/12.2.1/thumb/v8-m.main+fp/hard\libg_nano.a(libc_a-lock.o)
 .bss.__lock___env_recursive_mutex
                0x00000000        0x1 c:/renesas/ra/e2studio_v2023-07_fsp_v4.6.0/toolchains/gcc_arm/arm-gnu-toolchain-12.2.mpacbti-rel1-mingw-w64-i686-arm-none-eabi/bin/../lib/gcc/arm-none-eabi/12.2.1/thumb/v8-m.main+fp/hard\libg_nano.a(libc_a-lock.o)
 .bss.__lock___malloc_recursive_mutex
                0x00000000        0x1 c:/renesas/ra/e2studio_v2023-07_fsp_v4.6.0/toolchains/gcc_arm/arm-gnu-toolchain-12.2.mpacbti-rel1-mingw-w64-i686-arm-none-eabi/bin/../lib/gcc/arm-none-eabi/12.2.1/thumb/v8-m.main+fp/hard\libg_nano.a(libc_a-lock.o)
 .bss.__lock___at_quick_exit_mutex
                0x00000000        0x1 c:/renesas/ra/e2studio_v2023-07_fsp_v4.6.0/toolchains/gcc_arm/arm-gnu-toolchain-12.2.mpacbti-rel1-mingw-w64-i686-arm-none-eabi/bin/../lib/gcc/arm-none-eabi/12.2.1/thumb/v8-m.main+fp/hard\libg_nano.a(libc_a-lock.o)
 .bss.__lock___atexit_recursive_mutex
                0x00000000        0x1 c:/renesas/ra/e2studio_v2023-07_fsp_v4.6.0/toolchains/gcc_arm/arm-gnu-toolchain-12.2.mpacbti-rel1-mingw-w64-i686-arm-none-eabi/bin/../lib/gcc/arm-none-eabi/12.2.1/thumb/v8-m.main+fp/hard\libg_nano.a(libc_a-lock.o)
 .bss.__lock___sfp_recursive_mutex
                0x00000000        0x1 c:/renesas/ra/e2studio_v2023-07_fsp_v4.6.0/toolchains/gcc_arm/arm-gnu-toolchain-12.2.mpacbti-rel1-mingw-w64-i686-arm-none-eabi/bin/../lib/gcc/arm-none-eabi/12.2.1/thumb/v8-m.main+fp/hard\libg_nano.a(libc_a-lock.o)
 .debug_frame   0x00000000       0xb0 c:/renesas/ra/e2studio_v2023-07_fsp_v4.6.0/toolchains/gcc_arm/arm-gnu-toolchain-12.2.mpacbti-rel1-mingw-w64-i686-arm-none-eabi/bin/../lib/gcc/arm-none-eabi/12.2.1/thumb/v8-m.main+fp/hard\libg_nano.a(libc_a-lock.o)
 .ARM.attributes
                0x00000000       0x38 c:/renesas/ra/e2studio_v2023-07_fsp_v4.6.0/toolchains/gcc_arm/arm-gnu-toolchain-12.2.mpacbti-rel1-mingw-w64-i686-arm-none-eabi/bin/../lib/gcc/arm-none-eabi/12.2.1/thumb/v8-m.main+fp/hard\libg_nano.a(libc_a-lock.o)
 .text          0x00000000        0x0 c:/renesas/ra/e2studio_v2023-07_fsp_v4.6.0/toolchains/gcc_arm/arm-gnu-toolchain-12.2.mpacbti-rel1-mingw-w64-i686-arm-none-eabi/bin/../lib/gcc/arm-none-eabi/12.2.1/thumb/v8-m.main+fp/hard\libg_nano.a(libc_a-strcpy.o)
 .data          0x00000000        0x0 c:/renesas/ra/e2studio_v2023-07_fsp_v4.6.0/toolchains/gcc_arm/arm-gnu-toolchain-12.2.mpacbti-rel1-mingw-w64-i686-arm-none-eabi/bin/../lib/gcc/arm-none-eabi/12.2.1/thumb/v8-m.main+fp/hard\libg_nano.a(libc_a-strcpy.o)
 .bss           0x00000000        0x0 c:/renesas/ra/e2studio_v2023-07_fsp_v4.6.0/toolchains/gcc_arm/arm-gnu-toolchain-12.2.mpacbti-rel1-mingw-w64-i686-arm-none-eabi/bin/../lib/gcc/arm-none-eabi/12.2.1/thumb/v8-m.main+fp/hard\libg_nano.a(libc_a-strcpy.o)
 .text          0x00000000        0x0 c:/renesas/ra/e2studio_v2023-07_fsp_v4.6.0/toolchains/gcc_arm/arm-gnu-toolchain-12.2.mpacbti-rel1-mingw-w64-i686-arm-none-eabi/bin/../lib/gcc/arm-none-eabi/12.2.1/thumb/v8-m.main+fp/hard\libg_nano.a(libc_a-aeabi_memcpy.o)
 .data          0x00000000        0x0 c:/renesas/ra/e2studio_v2023-07_fsp_v4.6.0/toolchains/gcc_arm/arm-gnu-toolchain-12.2.mpacbti-rel1-mingw-w64-i686-arm-none-eabi/bin/../lib/gcc/arm-none-eabi/12.2.1/thumb/v8-m.main+fp/hard\libg_nano.a(libc_a-aeabi_memcpy.o)
 .bss           0x00000000        0x0 c:/renesas/ra/e2studio_v2023-07_fsp_v4.6.0/toolchains/gcc_arm/arm-gnu-toolchain-12.2.mpacbti-rel1-mingw-w64-i686-arm-none-eabi/bin/../lib/gcc/arm-none-eabi/12.2.1/thumb/v8-m.main+fp/hard\libg_nano.a(libc_a-aeabi_memcpy.o)
 .text          0x00000000        0x0 c:/renesas/ra/e2studio_v2023-07_fsp_v4.6.0/toolchains/gcc_arm/arm-gnu-toolchain-12.2.mpacbti-rel1-mingw-w64-i686-arm-none-eabi/bin/../lib/gcc/arm-none-eabi/12.2.1/thumb/v8-m.main+fp/hard\libg_nano.a(libc_a-aeabi_memclr.o)
 .data          0x00000000        0x0 c:/renesas/ra/e2studio_v2023-07_fsp_v4.6.0/toolchains/gcc_arm/arm-gnu-toolchain-12.2.mpacbti-rel1-mingw-w64-i686-arm-none-eabi/bin/../lib/gcc/arm-none-eabi/12.2.1/thumb/v8-m.main+fp/hard\libg_nano.a(libc_a-aeabi_memclr.o)
 .bss           0x00000000        0x0 c:/renesas/ra/e2studio_v2023-07_fsp_v4.6.0/toolchains/gcc_arm/arm-gnu-toolchain-12.2.mpacbti-rel1-mingw-w64-i686-arm-none-eabi/bin/../lib/gcc/arm-none-eabi/12.2.1/thumb/v8-m.main+fp/hard\libg_nano.a(libc_a-aeabi_memclr.o)
 .text          0x00000000        0x0 c:/renesas/ra/e2studio_v2023-07_fsp_v4.6.0/toolchains/gcc_arm/arm-gnu-toolchain-12.2.mpacbti-rel1-mingw-w64-i686-arm-none-eabi/bin/../lib/gcc/arm-none-eabi/12.2.1/thumb/v8-m.main+fp/hard\libg_nano.a(libc_a-memcpy-stub.o)
 .data          0x00000000        0x0 c:/renesas/ra/e2studio_v2023-07_fsp_v4.6.0/toolchains/gcc_arm/arm-gnu-toolchain-12.2.mpacbti-rel1-mingw-w64-i686-arm-none-eabi/bin/../lib/gcc/arm-none-eabi/12.2.1/thumb/v8-m.main+fp/hard\libg_nano.a(libc_a-memcpy-stub.o)
 .bss           0x00000000        0x0 c:/renesas/ra/e2studio_v2023-07_fsp_v4.6.0/toolchains/gcc_arm/arm-gnu-toolchain-12.2.mpacbti-rel1-mingw-w64-i686-arm-none-eabi/bin/../lib/gcc/arm-none-eabi/12.2.1/thumb/v8-m.main+fp/hard\libg_nano.a(libc_a-memcpy-stub.o)
 .data          0x00000000        0x0 c:/renesas/ra/e2studio_v2023-07_fsp_v4.6.0/toolchains/gcc_arm/arm-gnu-toolchain-12.2.mpacbti-rel1-mingw-w64-i686-arm-none-eabi/bin/../lib/gcc/arm-none-eabi/12.2.1/thumb/v8-m.main+fp/hard\libg_nano.a(libc_a-strlen.o)
 .bss           0x00000000        0x0 c:/renesas/ra/e2studio_v2023-07_fsp_v4.6.0/toolchains/gcc_arm/arm-gnu-toolchain-12.2.mpacbti-rel1-mingw-w64-i686-arm-none-eabi/bin/../lib/gcc/arm-none-eabi/12.2.1/thumb/v8-m.main+fp/hard\libg_nano.a(libc_a-strlen.o)
 .ARM.extab     0x00000000        0x0 c:/renesas/ra/e2studio_v2023-07_fsp_v4.6.0/toolchains/gcc_arm/arm-gnu-toolchain-12.2.mpacbti-rel1-mingw-w64-i686-arm-none-eabi/bin/../lib/gcc/arm-none-eabi/12.2.1/thumb/v8-m.main+fp/hard\libg_nano.a(libc_a-strlen.o)
 .text          0x00000000        0x0 c:/renesas/ra/e2studio_v2023-07_fsp_v4.6.0/toolchains/gcc_arm/arm-gnu-toolchain-12.2.mpacbti-rel1-mingw-w64-i686-arm-none-eabi/bin/../lib/gcc/arm-none-eabi/12.2.1/thumb/v8-m.main+fp/hard\libg_nano.a(libc_a-freer.o)
 .data          0x00000000        0x0 c:/renesas/ra/e2studio_v2023-07_fsp_v4.6.0/toolchains/gcc_arm/arm-gnu-toolchain-12.2.mpacbti-rel1-mingw-w64-i686-arm-none-eabi/bin/../lib/gcc/arm-none-eabi/12.2.1/thumb/v8-m.main+fp/hard\libg_nano.a(libc_a-freer.o)
 .bss           0x00000000        0x0 c:/renesas/ra/e2studio_v2023-07_fsp_v4.6.0/toolchains/gcc_arm/arm-gnu-toolchain-12.2.mpacbti-rel1-mingw-w64-i686-arm-none-eabi/bin/../lib/gcc/arm-none-eabi/12.2.1/thumb/v8-m.main+fp/hard\libg_nano.a(libc_a-freer.o)
 .text._free_r  0x00000000       0x94 c:/renesas/ra/e2studio_v2023-07_fsp_v4.6.0/toolchains/gcc_arm/arm-gnu-toolchain-12.2.mpacbti-rel1-mingw-w64-i686-arm-none-eabi/bin/../lib/gcc/arm-none-eabi/12.2.1/thumb/v8-m.main+fp/hard\libg_nano.a(libc_a-freer.o)
 .debug_frame   0x00000000       0x38 c:/renesas/ra/e2studio_v2023-07_fsp_v4.6.0/toolchains/gcc_arm/arm-gnu-toolchain-12.2.mpacbti-rel1-mingw-w64-i686-arm-none-eabi/bin/../lib/gcc/arm-none-eabi/12.2.1/thumb/v8-m.main+fp/hard\libg_nano.a(libc_a-freer.o)
 .ARM.attributes
                0x00000000       0x38 c:/renesas/ra/e2studio_v2023-07_fsp_v4.6.0/toolchains/gcc_arm/arm-gnu-toolchain-12.2.mpacbti-rel1-mingw-w64-i686-arm-none-eabi/bin/../lib/gcc/arm-none-eabi/12.2.1/thumb/v8-m.main+fp/hard\libg_nano.a(libc_a-freer.o)
 .text          0x00000000        0x0 c:/renesas/ra/e2studio_v2023-07_fsp_v4.6.0/toolchains/gcc_arm/arm-gnu-toolchain-12.2.mpacbti-rel1-mingw-w64-i686-arm-none-eabi/bin/../lib/gcc/arm-none-eabi/12.2.1/thumb/v8-m.main+fp/hard\libg_nano.a(libc_a-mallocr.o)
 .data          0x00000000        0x0 c:/renesas/ra/e2studio_v2023-07_fsp_v4.6.0/toolchains/gcc_arm/arm-gnu-toolchain-12.2.mpacbti-rel1-mingw-w64-i686-arm-none-eabi/bin/../lib/gcc/arm-none-eabi/12.2.1/thumb/v8-m.main+fp/hard\libg_nano.a(libc_a-mallocr.o)
 .bss           0x00000000        0x0 c:/renesas/ra/e2studio_v2023-07_fsp_v4.6.0/toolchains/gcc_arm/arm-gnu-toolchain-12.2.mpacbti-rel1-mingw-w64-i686-arm-none-eabi/bin/../lib/gcc/arm-none-eabi/12.2.1/thumb/v8-m.main+fp/hard\libg_nano.a(libc_a-mallocr.o)
 .text.sbrk_aligned
                0x00000000       0x44 c:/renesas/ra/e2studio_v2023-07_fsp_v4.6.0/toolchains/gcc_arm/arm-gnu-toolchain-12.2.mpacbti-rel1-mingw-w64-i686-arm-none-eabi/bin/../lib/gcc/arm-none-eabi/12.2.1/thumb/v8-m.main+fp/hard\libg_nano.a(libc_a-mallocr.o)
 .text._malloc_r
                0x00000000      0x100 c:/renesas/ra/e2studio_v2023-07_fsp_v4.6.0/toolchains/gcc_arm/arm-gnu-toolchain-12.2.mpacbti-rel1-mingw-w64-i686-arm-none-eabi/bin/../lib/gcc/arm-none-eabi/12.2.1/thumb/v8-m.main+fp/hard\libg_nano.a(libc_a-mallocr.o)
 .bss.__malloc_sbrk_start
                0x00000000        0x4 c:/renesas/ra/e2studio_v2023-07_fsp_v4.6.0/toolchains/gcc_arm/arm-gnu-toolchain-12.2.mpacbti-rel1-mingw-w64-i686-arm-none-eabi/bin/../lib/gcc/arm-none-eabi/12.2.1/thumb/v8-m.main+fp/hard\libg_nano.a(libc_a-mallocr.o)
 .bss.__malloc_free_list
                0x00000000        0x4 c:/renesas/ra/e2studio_v2023-07_fsp_v4.6.0/toolchains/gcc_arm/arm-gnu-toolchain-12.2.mpacbti-rel1-mingw-w64-i686-arm-none-eabi/bin/../lib/gcc/arm-none-eabi/12.2.1/thumb/v8-m.main+fp/hard\libg_nano.a(libc_a-mallocr.o)
 .debug_frame   0x00000000       0x50 c:/renesas/ra/e2studio_v2023-07_fsp_v4.6.0/toolchains/gcc_arm/arm-gnu-toolchain-12.2.mpacbti-rel1-mingw-w64-i686-arm-none-eabi/bin/../lib/gcc/arm-none-eabi/12.2.1/thumb/v8-m.main+fp/hard\libg_nano.a(libc_a-mallocr.o)
 .ARM.attributes
                0x00000000       0x38 c:/renesas/ra/e2studio_v2023-07_fsp_v4.6.0/toolchains/gcc_arm/arm-gnu-toolchain-12.2.mpacbti-rel1-mingw-w64-i686-arm-none-eabi/bin/../lib/gcc/arm-none-eabi/12.2.1/thumb/v8-m.main+fp/hard\libg_nano.a(libc_a-mallocr.o)
 .text          0x00000000        0x0 c:/renesas/ra/e2studio_v2023-07_fsp_v4.6.0/toolchains/gcc_arm/arm-gnu-toolchain-12.2.mpacbti-rel1-mingw-w64-i686-arm-none-eabi/bin/../lib/gcc/arm-none-eabi/12.2.1/thumb/v8-m.main+fp/hard\libg_nano.a(libc_a-mlock.o)
 .data          0x00000000        0x0 c:/renesas/ra/e2studio_v2023-07_fsp_v4.6.0/toolchains/gcc_arm/arm-gnu-toolchain-12.2.mpacbti-rel1-mingw-w64-i686-arm-none-eabi/bin/../lib/gcc/arm-none-eabi/12.2.1/thumb/v8-m.main+fp/hard\libg_nano.a(libc_a-mlock.o)
 .bss           0x00000000        0x0 c:/renesas/ra/e2studio_v2023-07_fsp_v4.6.0/toolchains/gcc_arm/arm-gnu-toolchain-12.2.mpacbti-rel1-mingw-w64-i686-arm-none-eabi/bin/../lib/gcc/arm-none-eabi/12.2.1/thumb/v8-m.main+fp/hard\libg_nano.a(libc_a-mlock.o)
 .text.__malloc_lock
                0x00000000        0xc c:/renesas/ra/e2studio_v2023-07_fsp_v4.6.0/toolchains/gcc_arm/arm-gnu-toolchain-12.2.mpacbti-rel1-mingw-w64-i686-arm-none-eabi/bin/../lib/gcc/arm-none-eabi/12.2.1/thumb/v8-m.main+fp/hard\libg_nano.a(libc_a-mlock.o)
 .text.__malloc_unlock
                0x00000000        0xc c:/renesas/ra/e2studio_v2023-07_fsp_v4.6.0/toolchains/gcc_arm/arm-gnu-toolchain-12.2.mpacbti-rel1-mingw-w64-i686-arm-none-eabi/bin/../lib/gcc/arm-none-eabi/12.2.1/thumb/v8-m.main+fp/hard\libg_nano.a(libc_a-mlock.o)
 .debug_frame   0x00000000       0x30 c:/renesas/ra/e2studio_v2023-07_fsp_v4.6.0/toolchains/gcc_arm/arm-gnu-toolchain-12.2.mpacbti-rel1-mingw-w64-i686-arm-none-eabi/bin/../lib/gcc/arm-none-eabi/12.2.1/thumb/v8-m.main+fp/hard\libg_nano.a(libc_a-mlock.o)
 .ARM.attributes
                0x00000000       0x38 c:/renesas/ra/e2studio_v2023-07_fsp_v4.6.0/toolchains/gcc_arm/arm-gnu-toolchain-12.2.mpacbti-rel1-mingw-w64-i686-arm-none-eabi/bin/../lib/gcc/arm-none-eabi/12.2.1/thumb/v8-m.main+fp/hard\libg_nano.a(libc_a-mlock.o)
 .text          0x00000000        0x0 c:/renesas/ra/e2studio_v2023-07_fsp_v4.6.0/toolchains/gcc_arm/arm-gnu-toolchain-12.2.mpacbti-rel1-mingw-w64-i686-arm-none-eabi/bin/../lib/gcc/arm-none-eabi/12.2.1/thumb/v8-m.main+fp/hard\libg_nano.a(libc_a-fflush.o)
 .data          0x00000000        0x0 c:/renesas/ra/e2studio_v2023-07_fsp_v4.6.0/toolchains/gcc_arm/arm-gnu-toolchain-12.2.mpacbti-rel1-mingw-w64-i686-arm-none-eabi/bin/../lib/gcc/arm-none-eabi/12.2.1/thumb/v8-m.main+fp/hard\libg_nano.a(libc_a-fflush.o)
 .bss           0x00000000        0x0 c:/renesas/ra/e2studio_v2023-07_fsp_v4.6.0/toolchains/gcc_arm/arm-gnu-toolchain-12.2.mpacbti-rel1-mingw-w64-i686-arm-none-eabi/bin/../lib/gcc/arm-none-eabi/12.2.1/thumb/v8-m.main+fp/hard\libg_nano.a(libc_a-fflush.o)
 .text.__sflush_r
                0x00000000      0x106 c:/renesas/ra/e2studio_v2023-07_fsp_v4.6.0/toolchains/gcc_arm/arm-gnu-toolchain-12.2.mpacbti-rel1-mingw-w64-i686-arm-none-eabi/bin/../lib/gcc/arm-none-eabi/12.2.1/thumb/v8-m.main+fp/hard\libg_nano.a(libc_a-fflush.o)
 .text._fflush_r
                0x00000000       0x50 c:/renesas/ra/e2studio_v2023-07_fsp_v4.6.0/toolchains/gcc_arm/arm-gnu-toolchain-12.2.mpacbti-rel1-mingw-w64-i686-arm-none-eabi/bin/../lib/gcc/arm-none-eabi/12.2.1/thumb/v8-m.main+fp/hard\libg_nano.a(libc_a-fflush.o)
 .text.fflush   0x00000000       0x28 c:/renesas/ra/e2studio_v2023-07_fsp_v4.6.0/toolchains/gcc_arm/arm-gnu-toolchain-12.2.mpacbti-rel1-mingw-w64-i686-arm-none-eabi/bin/../lib/gcc/arm-none-eabi/12.2.1/thumb/v8-m.main+fp/hard\libg_nano.a(libc_a-fflush.o)
 .debug_frame   0x00000000       0x5c c:/renesas/ra/e2studio_v2023-07_fsp_v4.6.0/toolchains/gcc_arm/arm-gnu-toolchain-12.2.mpacbti-rel1-mingw-w64-i686-arm-none-eabi/bin/../lib/gcc/arm-none-eabi/12.2.1/thumb/v8-m.main+fp/hard\libg_nano.a(libc_a-fflush.o)
 .ARM.attributes
                0x00000000       0x38 c:/renesas/ra/e2studio_v2023-07_fsp_v4.6.0/toolchains/gcc_arm/arm-gnu-toolchain-12.2.mpacbti-rel1-mingw-w64-i686-arm-none-eabi/bin/../lib/gcc/arm-none-eabi/12.2.1/thumb/v8-m.main+fp/hard\libg_nano.a(libc_a-fflush.o)
 .text          0x00000000        0x0 c:/renesas/ra/e2studio_v2023-07_fsp_v4.6.0/toolchains/gcc_arm/arm-gnu-toolchain-12.2.mpacbti-rel1-mingw-w64-i686-arm-none-eabi/bin/../lib/gcc/arm-none-eabi/12.2.1/thumb/v8-m.main+fp/hard\libg_nano.a(libc_a-sbrkr.o)
 .data          0x00000000        0x0 c:/renesas/ra/e2studio_v2023-07_fsp_v4.6.0/toolchains/gcc_arm/arm-gnu-toolchain-12.2.mpacbti-rel1-mingw-w64-i686-arm-none-eabi/bin/../lib/gcc/arm-none-eabi/12.2.1/thumb/v8-m.main+fp/hard\libg_nano.a(libc_a-sbrkr.o)
 .bss           0x00000000        0x0 c:/renesas/ra/e2studio_v2023-07_fsp_v4.6.0/toolchains/gcc_arm/arm-gnu-toolchain-12.2.mpacbti-rel1-mingw-w64-i686-arm-none-eabi/bin/../lib/gcc/arm-none-eabi/12.2.1/thumb/v8-m.main+fp/hard\libg_nano.a(libc_a-sbrkr.o)
 .text._sbrk_r  0x00000000       0x20 c:/renesas/ra/e2studio_v2023-07_fsp_v4.6.0/toolchains/gcc_arm/arm-gnu-toolchain-12.2.mpacbti-rel1-mingw-w64-i686-arm-none-eabi/bin/../lib/gcc/arm-none-eabi/12.2.1/thumb/v8-m.main+fp/hard\libg_nano.a(libc_a-sbrkr.o)
 .debug_frame   0x00000000       0x2c c:/renesas/ra/e2studio_v2023-07_fsp_v4.6.0/toolchains/gcc_arm/arm-gnu-toolchain-12.2.mpacbti-rel1-mingw-w64-i686-arm-none-eabi/bin/../lib/gcc/arm-none-eabi/12.2.1/thumb/v8-m.main+fp/hard\libg_nano.a(libc_a-sbrkr.o)
 .ARM.attributes
                0x00000000       0x38 c:/renesas/ra/e2studio_v2023-07_fsp_v4.6.0/toolchains/gcc_arm/arm-gnu-toolchain-12.2.mpacbti-rel1-mingw-w64-i686-arm-none-eabi/bin/../lib/gcc/arm-none-eabi/12.2.1/thumb/v8-m.main+fp/hard\libg_nano.a(libc_a-sbrkr.o)
 .data          0x00000000        0x0 c:/renesas/ra/e2studio_v2023-07_fsp_v4.6.0/toolchains/gcc_arm/arm-gnu-toolchain-12.2.mpacbti-rel1-mingw-w64-i686-arm-none-eabi/bin/../lib/gcc/arm-none-eabi/12.2.1/thumb/v8-m.main+fp/hard\libg_nano.a(libc_a-aeabi_memset-soft.o)
 .bss           0x00000000        0x0 c:/renesas/ra/e2studio_v2023-07_fsp_v4.6.0/toolchains/gcc_arm/arm-gnu-toolchain-12.2.mpacbti-rel1-mingw-w64-i686-arm-none-eabi/bin/../lib/gcc/arm-none-eabi/12.2.1/thumb/v8-m.main+fp/hard\libg_nano.a(libc_a-aeabi_memset-soft.o)
 .ARM.extab     0x00000000        0x0 c:/renesas/ra/e2studio_v2023-07_fsp_v4.6.0/toolchains/gcc_arm/arm-gnu-toolchain-12.2.mpacbti-rel1-mingw-w64-i686-arm-none-eabi/bin/../lib/gcc/arm-none-eabi/12.2.1/thumb/v8-m.main+fp/hard\libg_nano.a(libc_a-aeabi_memset-soft.o)
 .text          0x00000000        0x0 c:/renesas/ra/e2studio_v2023-07_fsp_v4.6.0/toolchains/gcc_arm/arm-gnu-toolchain-12.2.mpacbti-rel1-mingw-w64-i686-arm-none-eabi/bin/../lib/gcc/arm-none-eabi/12.2.1/thumb/v8-m.main+fp/hard\librdimon_nano.a(arm_librdimon_a-_exit.o)
 .data          0x00000000        0x0 c:/renesas/ra/e2studio_v2023-07_fsp_v4.6.0/toolchains/gcc_arm/arm-gnu-toolchain-12.2.mpacbti-rel1-mingw-w64-i686-arm-none-eabi/bin/../lib/gcc/arm-none-eabi/12.2.1/thumb/v8-m.main+fp/hard\librdimon_nano.a(arm_librdimon_a-_exit.o)
 .bss           0x00000000        0x0 c:/renesas/ra/e2studio_v2023-07_fsp_v4.6.0/toolchains/gcc_arm/arm-gnu-toolchain-12.2.mpacbti-rel1-mingw-w64-i686-arm-none-eabi/bin/../lib/gcc/arm-none-eabi/12.2.1/thumb/v8-m.main+fp/hard\librdimon_nano.a(arm_librdimon_a-_exit.o)
 .text._exit    0x00000000       0x14 c:/renesas/ra/e2studio_v2023-07_fsp_v4.6.0/toolchains/gcc_arm/arm-gnu-toolchain-12.2.mpacbti-rel1-mingw-w64-i686-arm-none-eabi/bin/../lib/gcc/arm-none-eabi/12.2.1/thumb/v8-m.main+fp/hard\librdimon_nano.a(arm_librdimon_a-_exit.o)
 .debug_frame   0x00000000       0x28 c:/renesas/ra/e2studio_v2023-07_fsp_v4.6.0/toolchains/gcc_arm/arm-gnu-toolchain-12.2.mpacbti-rel1-mingw-w64-i686-arm-none-eabi/bin/../lib/gcc/arm-none-eabi/12.2.1/thumb/v8-m.main+fp/hard\librdimon_nano.a(arm_librdimon_a-_exit.o)
 .ARM.attributes
                0x00000000       0x38 c:/renesas/ra/e2studio_v2023-07_fsp_v4.6.0/toolchains/gcc_arm/arm-gnu-toolchain-12.2.mpacbti-rel1-mingw-w64-i686-arm-none-eabi/bin/../lib/gcc/arm-none-eabi/12.2.1/thumb/v8-m.main+fp/hard\librdimon_nano.a(arm_librdimon_a-_exit.o)
 .text          0x00000000        0x0 c:/renesas/ra/e2studio_v2023-07_fsp_v4.6.0/toolchains/gcc_arm/arm-gnu-toolchain-12.2.mpacbti-rel1-mingw-w64-i686-arm-none-eabi/bin/../lib/gcc/arm-none-eabi/12.2.1/thumb/v8-m.main+fp/hard\librdimon_nano.a(arm_librdimon_a-_kill.o)
 .data          0x00000000        0x0 c:/renesas/ra/e2studio_v2023-07_fsp_v4.6.0/toolchains/gcc_arm/arm-gnu-toolchain-12.2.mpacbti-rel1-mingw-w64-i686-arm-none-eabi/bin/../lib/gcc/arm-none-eabi/12.2.1/thumb/v8-m.main+fp/hard\librdimon_nano.a(arm_librdimon_a-_kill.o)
 .bss           0x00000000        0x0 c:/renesas/ra/e2studio_v2023-07_fsp_v4.6.0/toolchains/gcc_arm/arm-gnu-toolchain-12.2.mpacbti-rel1-mingw-w64-i686-arm-none-eabi/bin/../lib/gcc/arm-none-eabi/12.2.1/thumb/v8-m.main+fp/hard\librdimon_nano.a(arm_librdimon_a-_kill.o)
 .text._kill_shared
                0x00000000       0x26 c:/renesas/ra/e2studio_v2023-07_fsp_v4.6.0/toolchains/gcc_arm/arm-gnu-toolchain-12.2.mpacbti-rel1-mingw-w64-i686-arm-none-eabi/bin/../lib/gcc/arm-none-eabi/12.2.1/thumb/v8-m.main+fp/hard\librdimon_nano.a(arm_librdimon_a-_kill.o)
 .text._kill    0x00000000       0x18 c:/renesas/ra/e2studio_v2023-07_fsp_v4.6.0/toolchains/gcc_arm/arm-gnu-toolchain-12.2.mpacbti-rel1-mingw-w64-i686-arm-none-eabi/bin/../lib/gcc/arm-none-eabi/12.2.1/thumb/v8-m.main+fp/hard\librdimon_nano.a(arm_librdimon_a-_kill.o)
 .debug_frame   0x00000000       0x40 c:/renesas/ra/e2studio_v2023-07_fsp_v4.6.0/toolchains/gcc_arm/arm-gnu-toolchain-12.2.mpacbti-rel1-mingw-w64-i686-arm-none-eabi/bin/../lib/gcc/arm-none-eabi/12.2.1/thumb/v8-m.main+fp/hard\librdimon_nano.a(arm_librdimon_a-_kill.o)
 .ARM.attributes
                0x00000000       0x38 c:/renesas/ra/e2studio_v2023-07_fsp_v4.6.0/toolchains/gcc_arm/arm-gnu-toolchain-12.2.mpacbti-rel1-mingw-w64-i686-arm-none-eabi/bin/../lib/gcc/arm-none-eabi/12.2.1/thumb/v8-m.main+fp/hard\librdimon_nano.a(arm_librdimon_a-_kill.o)
 .text          0x00000000        0x0 c:/renesas/ra/e2studio_v2023-07_fsp_v4.6.0/toolchains/gcc_arm/arm-gnu-toolchain-12.2.mpacbti-rel1-mingw-w64-i686-arm-none-eabi/bin/../lib/gcc/arm-none-eabi/12.2.1/thumb/v8-m.main+fp/hard\librdimon_nano.a(arm_librdimon_a-syscalls.o)
 .data          0x00000000        0x0 c:/renesas/ra/e2studio_v2023-07_fsp_v4.6.0/toolchains/gcc_arm/arm-gnu-toolchain-12.2.mpacbti-rel1-mingw-w64-i686-arm-none-eabi/bin/../lib/gcc/arm-none-eabi/12.2.1/thumb/v8-m.main+fp/hard\librdimon_nano.a(arm_librdimon_a-syscalls.o)
 .bss           0x00000000        0x0 c:/renesas/ra/e2studio_v2023-07_fsp_v4.6.0/toolchains/gcc_arm/arm-gnu-toolchain-12.2.mpacbti-rel1-mingw-w64-i686-arm-none-eabi/bin/../lib/gcc/arm-none-eabi/12.2.1/thumb/v8-m.main+fp/hard\librdimon_nano.a(arm_librdimon_a-syscalls.o)
 .text.findslot
                0x00000000       0x34 c:/renesas/ra/e2studio_v2023-07_fsp_v4.6.0/toolchains/gcc_arm/arm-gnu-toolchain-12.2.mpacbti-rel1-mingw-w64-i686-arm-none-eabi/bin/../lib/gcc/arm-none-eabi/12.2.1/thumb/v8-m.main+fp/hard\librdimon_nano.a(arm_librdimon_a-syscalls.o)
 .text.error    0x00000000       0x1c c:/renesas/ra/e2studio_v2023-07_fsp_v4.6.0/toolchains/gcc_arm/arm-gnu-toolchain-12.2.mpacbti-rel1-mingw-w64-i686-arm-none-eabi/bin/../lib/gcc/arm-none-eabi/12.2.1/thumb/v8-m.main+fp/hard\librdimon_nano.a(arm_librdimon_a-syscalls.o)
 .text.checkerror
                0x00000000        0xa c:/renesas/ra/e2studio_v2023-07_fsp_v4.6.0/toolchains/gcc_arm/arm-gnu-toolchain-12.2.mpacbti-rel1-mingw-w64-i686-arm-none-eabi/bin/../lib/gcc/arm-none-eabi/12.2.1/thumb/v8-m.main+fp/hard\librdimon_nano.a(arm_librdimon_a-syscalls.o)
 .text._swiread
                0x00000000       0x20 c:/renesas/ra/e2studio_v2023-07_fsp_v4.6.0/toolchains/gcc_arm/arm-gnu-toolchain-12.2.mpacbti-rel1-mingw-w64-i686-arm-none-eabi/bin/../lib/gcc/arm-none-eabi/12.2.1/thumb/v8-m.main+fp/hard\librdimon_nano.a(arm_librdimon_a-syscalls.o)
 .text._read    0x00000000       0x34 c:/renesas/ra/e2studio_v2023-07_fsp_v4.6.0/toolchains/gcc_arm/arm-gnu-toolchain-12.2.mpacbti-rel1-mingw-w64-i686-arm-none-eabi/bin/../lib/gcc/arm-none-eabi/12.2.1/thumb/v8-m.main+fp/hard\librdimon_nano.a(arm_librdimon_a-syscalls.o)
 .text._swilseek
                0x00000000       0x78 c:/renesas/ra/e2studio_v2023-07_fsp_v4.6.0/toolchains/gcc_arm/arm-gnu-toolchain-12.2.mpacbti-rel1-mingw-w64-i686-arm-none-eabi/bin/../lib/gcc/arm-none-eabi/12.2.1/thumb/v8-m.main+fp/hard\librdimon_nano.a(arm_librdimon_a-syscalls.o)
 .text._lseek   0x00000000        0x4 c:/renesas/ra/e2studio_v2023-07_fsp_v4.6.0/toolchains/gcc_arm/arm-gnu-toolchain-12.2.mpacbti-rel1-mingw-w64-i686-arm-none-eabi/bin/../lib/gcc/arm-none-eabi/12.2.1/thumb/v8-m.main+fp/hard\librdimon_nano.a(arm_librdimon_a-syscalls.o)
 .text._swiwrite
                0x00000000       0x20 c:/renesas/ra/e2studio_v2023-07_fsp_v4.6.0/toolchains/gcc_arm/arm-gnu-toolchain-12.2.mpacbti-rel1-mingw-w64-i686-arm-none-eabi/bin/../lib/gcc/arm-none-eabi/12.2.1/thumb/v8-m.main+fp/hard\librdimon_nano.a(arm_librdimon_a-syscalls.o)
 .text._write   0x00000000       0x40 c:/renesas/ra/e2studio_v2023-07_fsp_v4.6.0/toolchains/gcc_arm/arm-gnu-toolchain-12.2.mpacbti-rel1-mingw-w64-i686-arm-none-eabi/bin/../lib/gcc/arm-none-eabi/12.2.1/thumb/v8-m.main+fp/hard\librdimon_nano.a(arm_librdimon_a-syscalls.o)
 .text._swiclose
                0x00000000       0x1a c:/renesas/ra/e2studio_v2023-07_fsp_v4.6.0/toolchains/gcc_arm/arm-gnu-toolchain-12.2.mpacbti-rel1-mingw-w64-i686-arm-none-eabi/bin/../lib/gcc/arm-none-eabi/12.2.1/thumb/v8-m.main+fp/hard\librdimon_nano.a(arm_librdimon_a-syscalls.o)
 .text._close   0x00000000       0x44 c:/renesas/ra/e2studio_v2023-07_fsp_v4.6.0/toolchains/gcc_arm/arm-gnu-toolchain-12.2.mpacbti-rel1-mingw-w64-i686-arm-none-eabi/bin/../lib/gcc/arm-none-eabi/12.2.1/thumb/v8-m.main+fp/hard\librdimon_nano.a(arm_librdimon_a-syscalls.o)
 .text._getpid  0x00000000        0x4 c:/renesas/ra/e2studio_v2023-07_fsp_v4.6.0/toolchains/gcc_arm/arm-gnu-toolchain-12.2.mpacbti-rel1-mingw-w64-i686-arm-none-eabi/bin/../lib/gcc/arm-none-eabi/12.2.1/thumb/v8-m.main+fp/hard\librdimon_nano.a(arm_librdimon_a-syscalls.o)
 .text._sbrk    0x00000000       0x48 c:/renesas/ra/e2studio_v2023-07_fsp_v4.6.0/toolchains/gcc_arm/arm-gnu-toolchain-12.2.mpacbti-rel1-mingw-w64-i686-arm-none-eabi/bin/../lib/gcc/arm-none-eabi/12.2.1/thumb/v8-m.main+fp/hard\librdimon_nano.a(arm_librdimon_a-syscalls.o)
 .text._swistat
                0x00000000       0x42 c:/renesas/ra/e2studio_v2023-07_fsp_v4.6.0/toolchains/gcc_arm/arm-gnu-toolchain-12.2.mpacbti-rel1-mingw-w64-i686-arm-none-eabi/bin/../lib/gcc/arm-none-eabi/12.2.1/thumb/v8-m.main+fp/hard\librdimon_nano.a(arm_librdimon_a-syscalls.o)
 .text._fstat   0x00000000       0x1c c:/renesas/ra/e2studio_v2023-07_fsp_v4.6.0/toolchains/gcc_arm/arm-gnu-toolchain-12.2.mpacbti-rel1-mingw-w64-i686-arm-none-eabi/bin/../lib/gcc/arm-none-eabi/12.2.1/thumb/v8-m.main+fp/hard\librdimon_nano.a(arm_librdimon_a-syscalls.o)
 .text._stat    0x00000000       0x3a c:/renesas/ra/e2studio_v2023-07_fsp_v4.6.0/toolchains/gcc_arm/arm-gnu-toolchain-12.2.mpacbti-rel1-mingw-w64-i686-arm-none-eabi/bin/../lib/gcc/arm-none-eabi/12.2.1/thumb/v8-m.main+fp/hard\librdimon_nano.a(arm_librdimon_a-syscalls.o)
 .text._swiopen
                0x00000000       0xb0 c:/renesas/ra/e2studio_v2023-07_fsp_v4.6.0/toolchains/gcc_arm/arm-gnu-toolchain-12.2.mpacbti-rel1-mingw-w64-i686-arm-none-eabi/bin/../lib/gcc/arm-none-eabi/12.2.1/thumb/v8-m.main+fp/hard\librdimon_nano.a(arm_librdimon_a-syscalls.o)
 .text._open    0x00000000       0x12 c:/renesas/ra/e2studio_v2023-07_fsp_v4.6.0/toolchains/gcc_arm/arm-gnu-toolchain-12.2.mpacbti-rel1-mingw-w64-i686-arm-none-eabi/bin/../lib/gcc/arm-none-eabi/12.2.1/thumb/v8-m.main+fp/hard\librdimon_nano.a(arm_librdimon_a-syscalls.o)
 .rodata._get_semihosting_exts.str1.1
                0x00000000       0x16 c:/renesas/ra/e2studio_v2023-07_fsp_v4.6.0/toolchains/gcc_arm/arm-gnu-toolchain-12.2.mpacbti-rel1-mingw-w64-i686-arm-none-eabi/bin/../lib/gcc/arm-none-eabi/12.2.1/thumb/v8-m.main+fp/hard\librdimon_nano.a(arm_librdimon_a-syscalls.o)
 .text._get_semihosting_exts
                0x00000000       0xb4 c:/renesas/ra/e2studio_v2023-07_fsp_v4.6.0/toolchains/gcc_arm/arm-gnu-toolchain-12.2.mpacbti-rel1-mingw-w64-i686-arm-none-eabi/bin/../lib/gcc/arm-none-eabi/12.2.1/thumb/v8-m.main+fp/hard\librdimon_nano.a(arm_librdimon_a-syscalls.o)
 .text.initialise_semihosting_exts
                0x00000000       0x34 c:/renesas/ra/e2studio_v2023-07_fsp_v4.6.0/toolchains/gcc_arm/arm-gnu-toolchain-12.2.mpacbti-rel1-mingw-w64-i686-arm-none-eabi/bin/../lib/gcc/arm-none-eabi/12.2.1/thumb/v8-m.main+fp/hard\librdimon_nano.a(arm_librdimon_a-syscalls.o)
 .text._has_ext_exit_extended
                0x00000000       0x18 c:/renesas/ra/e2studio_v2023-07_fsp_v4.6.0/toolchains/gcc_arm/arm-gnu-toolchain-12.2.mpacbti-rel1-mingw-w64-i686-arm-none-eabi/bin/../lib/gcc/arm-none-eabi/12.2.1/thumb/v8-m.main+fp/hard\librdimon_nano.a(arm_librdimon_a-syscalls.o)
 .text._has_ext_stdout_stderr
                0x00000000       0x18 c:/renesas/ra/e2studio_v2023-07_fsp_v4.6.0/toolchains/gcc_arm/arm-gnu-toolchain-12.2.mpacbti-rel1-mingw-w64-i686-arm-none-eabi/bin/../lib/gcc/arm-none-eabi/12.2.1/thumb/v8-m.main+fp/hard\librdimon_nano.a(arm_librdimon_a-syscalls.o)
 .rodata.initialise_monitor_handles.str1.1
                0x00000000        0x4 c:/renesas/ra/e2studio_v2023-07_fsp_v4.6.0/toolchains/gcc_arm/arm-gnu-toolchain-12.2.mpacbti-rel1-mingw-w64-i686-arm-none-eabi/bin/../lib/gcc/arm-none-eabi/12.2.1/thumb/v8-m.main+fp/hard\librdimon_nano.a(arm_librdimon_a-syscalls.o)
 .text.initialise_monitor_handles
                0x00000000       0xc0 c:/renesas/ra/e2studio_v2023-07_fsp_v4.6.0/toolchains/gcc_arm/arm-gnu-toolchain-12.2.mpacbti-rel1-mingw-w64-i686-arm-none-eabi/bin/../lib/gcc/arm-none-eabi/12.2.1/thumb/v8-m.main+fp/hard\librdimon_nano.a(arm_librdimon_a-syscalls.o)
 .text._link    0x00000000       0x10 c:/renesas/ra/e2studio_v2023-07_fsp_v4.6.0/toolchains/gcc_arm/arm-gnu-toolchain-12.2.mpacbti-rel1-mingw-w64-i686-arm-none-eabi/bin/../lib/gcc/arm-none-eabi/12.2.1/thumb/v8-m.main+fp/hard\librdimon_nano.a(arm_librdimon_a-syscalls.o)
 .text._unlink  0x00000000       0x28 c:/renesas/ra/e2studio_v2023-07_fsp_v4.6.0/toolchains/gcc_arm/arm-gnu-toolchain-12.2.mpacbti-rel1-mingw-w64-i686-arm-none-eabi/bin/../lib/gcc/arm-none-eabi/12.2.1/thumb/v8-m.main+fp/hard\librdimon_nano.a(arm_librdimon_a-syscalls.o)
 .text._gettimeofday
                0x00000000       0x28 c:/renesas/ra/e2studio_v2023-07_fsp_v4.6.0/toolchains/gcc_arm/arm-gnu-toolchain-12.2.mpacbti-rel1-mingw-w64-i686-arm-none-eabi/bin/../lib/gcc/arm-none-eabi/12.2.1/thumb/v8-m.main+fp/hard\librdimon_nano.a(arm_librdimon_a-syscalls.o)
 .text._clock   0x00000000       0x12 c:/renesas/ra/e2studio_v2023-07_fsp_v4.6.0/toolchains/gcc_arm/arm-gnu-toolchain-12.2.mpacbti-rel1-mingw-w64-i686-arm-none-eabi/bin/../lib/gcc/arm-none-eabi/12.2.1/thumb/v8-m.main+fp/hard\librdimon_nano.a(arm_librdimon_a-syscalls.o)
 .text._times   0x00000000       0x16 c:/renesas/ra/e2studio_v2023-07_fsp_v4.6.0/toolchains/gcc_arm/arm-gnu-toolchain-12.2.mpacbti-rel1-mingw-w64-i686-arm-none-eabi/bin/../lib/gcc/arm-none-eabi/12.2.1/thumb/v8-m.main+fp/hard\librdimon_nano.a(arm_librdimon_a-syscalls.o)
 .text._isatty  0x00000000       0x3a c:/renesas/ra/e2studio_v2023-07_fsp_v4.6.0/toolchains/gcc_arm/arm-gnu-toolchain-12.2.mpacbti-rel1-mingw-w64-i686-arm-none-eabi/bin/../lib/gcc/arm-none-eabi/12.2.1/thumb/v8-m.main+fp/hard\librdimon_nano.a(arm_librdimon_a-syscalls.o)
 .text._system  0x00000000       0x3c c:/renesas/ra/e2studio_v2023-07_fsp_v4.6.0/toolchains/gcc_arm/arm-gnu-toolchain-12.2.mpacbti-rel1-mingw-w64-i686-arm-none-eabi/bin/../lib/gcc/arm-none-eabi/12.2.1/thumb/v8-m.main+fp/hard\librdimon_nano.a(arm_librdimon_a-syscalls.o)
 .text._rename  0x00000000       0x36 c:/renesas/ra/e2studio_v2023-07_fsp_v4.6.0/toolchains/gcc_arm/arm-gnu-toolchain-12.2.mpacbti-rel1-mingw-w64-i686-arm-none-eabi/bin/../lib/gcc/arm-none-eabi/12.2.1/thumb/v8-m.main+fp/hard\librdimon_nano.a(arm_librdimon_a-syscalls.o)
 .bss.heap_end.0
                0x00000000        0x4 c:/renesas/ra/e2studio_v2023-07_fsp_v4.6.0/toolchains/gcc_arm/arm-gnu-toolchain-12.2.mpacbti-rel1-mingw-w64-i686-arm-none-eabi/bin/../lib/gcc/arm-none-eabi/12.2.1/thumb/v8-m.main+fp/hard\librdimon_nano.a(arm_librdimon_a-syscalls.o)
 .data.__heap_limit
                0x00000000        0x4 c:/renesas/ra/e2studio_v2023-07_fsp_v4.6.0/toolchains/gcc_arm/arm-gnu-toolchain-12.2.mpacbti-rel1-mingw-w64-i686-arm-none-eabi/bin/../lib/gcc/arm-none-eabi/12.2.1/thumb/v8-m.main+fp/hard\librdimon_nano.a(arm_librdimon_a-syscalls.o)
 .data.supports_ext_stdout_stderr
                0x00000000        0x4 c:/renesas/ra/e2studio_v2023-07_fsp_v4.6.0/toolchains/gcc_arm/arm-gnu-toolchain-12.2.mpacbti-rel1-mingw-w64-i686-arm-none-eabi/bin/../lib/gcc/arm-none-eabi/12.2.1/thumb/v8-m.main+fp/hard\librdimon_nano.a(arm_librdimon_a-syscalls.o)
 .data.supports_ext_exit_extended
                0x00000000        0x4 c:/renesas/ra/e2studio_v2023-07_fsp_v4.6.0/toolchains/gcc_arm/arm-gnu-toolchain-12.2.mpacbti-rel1-mingw-w64-i686-arm-none-eabi/bin/../lib/gcc/arm-none-eabi/12.2.1/thumb/v8-m.main+fp/hard\librdimon_nano.a(arm_librdimon_a-syscalls.o)
 .bss.monitor_stderr
                0x00000000        0x4 c:/renesas/ra/e2studio_v2023-07_fsp_v4.6.0/toolchains/gcc_arm/arm-gnu-toolchain-12.2.mpacbti-rel1-mingw-w64-i686-arm-none-eabi/bin/../lib/gcc/arm-none-eabi/12.2.1/thumb/v8-m.main+fp/hard\librdimon_nano.a(arm_librdimon_a-syscalls.o)
 .bss.monitor_stdout
                0x00000000        0x4 c:/renesas/ra/e2studio_v2023-07_fsp_v4.6.0/toolchains/gcc_arm/arm-gnu-toolchain-12.2.mpacbti-rel1-mingw-w64-i686-arm-none-eabi/bin/../lib/gcc/arm-none-eabi/12.2.1/thumb/v8-m.main+fp/hard\librdimon_nano.a(arm_librdimon_a-syscalls.o)
 .bss.monitor_stdin
                0x00000000        0x4 c:/renesas/ra/e2studio_v2023-07_fsp_v4.6.0/toolchains/gcc_arm/arm-gnu-toolchain-12.2.mpacbti-rel1-mingw-w64-i686-arm-none-eabi/bin/../lib/gcc/arm-none-eabi/12.2.1/thumb/v8-m.main+fp/hard\librdimon_nano.a(arm_librdimon_a-syscalls.o)
 .bss.openfiles
                0x00000000       0xa0 c:/renesas/ra/e2studio_v2023-07_fsp_v4.6.0/toolchains/gcc_arm/arm-gnu-toolchain-12.2.mpacbti-rel1-mingw-w64-i686-arm-none-eabi/bin/../lib/gcc/arm-none-eabi/12.2.1/thumb/v8-m.main+fp/hard\librdimon_nano.a(arm_librdimon_a-syscalls.o)
 .debug_frame   0x00000000      0x39c c:/renesas/ra/e2studio_v2023-07_fsp_v4.6.0/toolchains/gcc_arm/arm-gnu-toolchain-12.2.mpacbti-rel1-mingw-w64-i686-arm-none-eabi/bin/../lib/gcc/arm-none-eabi/12.2.1/thumb/v8-m.main+fp/hard\librdimon_nano.a(arm_librdimon_a-syscalls.o)
 .ARM.attributes
                0x00000000       0x38 c:/renesas/ra/e2studio_v2023-07_fsp_v4.6.0/toolchains/gcc_arm/arm-gnu-toolchain-12.2.mpacbti-rel1-mingw-w64-i686-arm-none-eabi/bin/../lib/gcc/arm-none-eabi/12.2.1/thumb/v8-m.main+fp/hard\librdimon_nano.a(arm_librdimon_a-syscalls.o)
 .text          0x00000000        0x0 c:/renesas/ra/e2studio_v2023-07_fsp_v4.6.0/toolchains/gcc_arm/arm-gnu-toolchain-12.2.mpacbti-rel1-mingw-w64-i686-arm-none-eabi/bin/../lib/gcc/arm-none-eabi/12.2.1/thumb/v8-m.main+fp/hard/crtend.o
 .data          0x00000000        0x0 c:/renesas/ra/e2studio_v2023-07_fsp_v4.6.0/toolchains/gcc_arm/arm-gnu-toolchain-12.2.mpacbti-rel1-mingw-w64-i686-arm-none-eabi/bin/../lib/gcc/arm-none-eabi/12.2.1/thumb/v8-m.main+fp/hard/crtend.o
 .bss           0x00000000        0x0 c:/renesas/ra/e2studio_v2023-07_fsp_v4.6.0/toolchains/gcc_arm/arm-gnu-toolchain-12.2.mpacbti-rel1-mingw-w64-i686-arm-none-eabi/bin/../lib/gcc/arm-none-eabi/12.2.1/thumb/v8-m.main+fp/hard/crtend.o
 .rodata.all_implied_fbits
                0x00000000       0x24 c:/renesas/ra/e2studio_v2023-07_fsp_v4.6.0/toolchains/gcc_arm/arm-gnu-toolchain-12.2.mpacbti-rel1-mingw-w64-i686-arm-none-eabi/bin/../lib/gcc/arm-none-eabi/12.2.1/thumb/v8-m.main+fp/hard/crtend.o
 .text          0x00000000        0x0 c:/renesas/ra/e2studio_v2023-07_fsp_v4.6.0/toolchains/gcc_arm/arm-gnu-toolchain-12.2.mpacbti-rel1-mingw-w64-i686-arm-none-eabi/bin/../lib/gcc/arm-none-eabi/12.2.1/thumb/v8-m.main+fp/hard/crtn.o
 .data          0x00000000        0x0 c:/renesas/ra/e2studio_v2023-07_fsp_v4.6.0/toolchains/gcc_arm/arm-gnu-toolchain-12.2.mpacbti-rel1-mingw-w64-i686-arm-none-eabi/bin/../lib/gcc/arm-none-eabi/12.2.1/thumb/v8-m.main+fp/hard/crtn.o
 .bss           0x00000000        0x0 c:/renesas/ra/e2studio_v2023-07_fsp_v4.6.0/toolchains/gcc_arm/arm-gnu-toolchain-12.2.mpacbti-rel1-mingw-w64-i686-arm-none-eabi/bin/../lib/gcc/arm-none-eabi/12.2.1/thumb/v8-m.main+fp/hard/crtn.o

Memory Configuration

Name             Origin             Length             Attributes
FLASH            0x00010000         0x00050000         xr
RAM              0x20000000         0x00020000         xrw
DATA_FLASH       0x08000000         0x00002000         xr
QSPI_FLASH       0x60000000         0x04000000         xr
OSPI_DEVICE_0    0x80020000         0x00000000         xr
OSPI_DEVICE_1    0x80030000         0x00000000         xr
OSPI_DEVICE_0_RAM 0x80020000         0x00000000         xrw
OSPI_DEVICE_1_RAM 0x80030000         0x00000000         xrw
SDRAM            0x80010000         0x00000000         xrw
OPTION_SETTING   0x0100a100         0x00000100         r
OPTION_SETTING_S 0x0100a200         0x00000100         r
ID_CODE          0x00000000         0x00000000         xr
*default*        0x00000000         0xffffffff

Linker script and memory map

LOAD c:/renesas/ra/e2studio_v2023-07_fsp_v4.6.0/toolchains/gcc_arm/arm-gnu-toolchain-12.2.mpacbti-rel1-mingw-w64-i686-arm-none-eabi/bin/../lib/gcc/arm-none-eabi/12.2.1/thumb/v8-m.main+fp/hard/crti.o
LOAD c:/renesas/ra/e2studio_v2023-07_fsp_v4.6.0/toolchains/gcc_arm/arm-gnu-toolchain-12.2.mpacbti-rel1-mingw-w64-i686-arm-none-eabi/bin/../lib/gcc/arm-none-eabi/12.2.1/thumb/v8-m.main+fp/hard/crtbegin.o
LOAD c:/renesas/ra/e2studio_v2023-07_fsp_v4.6.0/toolchains/gcc_arm/arm-gnu-toolchain-12.2.mpacbti-rel1-mingw-w64-i686-arm-none-eabi/bin/../lib/gcc/arm-none-eabi/12.2.1/thumb/v8-m.main+fp/hard/rdimon-crt0.o
                0x00010000                        FLASH_IMAGE_START = 0x10000
                0x00050000                        FLASH_IMAGE_LENGTH = 0x50000
START GROUP
LOAD ./src/adc_temp.o
LOAD ./src/angle.o
LOAD ./src/control_table.o
LOAD ./src/global_variables.o
LOAD ./src/hal_entry.o
LOAD ./src/interpolation.o
LOAD ./src/monitor.o
LOAD ./src/packet.o
LOAD ./src/pid.o
LOAD ./src/power_monitor.o
LOAD ./src/sintable.o
LOAD ./src/usart.o
LOAD ./ra_gen/common_data.o
LOAD ./ra_gen/hal_data.o
LOAD ./ra_gen/main.o
LOAD ./ra_gen/pin_data.o
LOAD ./ra_gen/vector_data.o
LOAD ./ra/fsp/src/r_sci_uart/r_sci_uart.o
LOAD ./ra/fsp/src/r_sci_spi/r_sci_spi.o
LOAD ./ra/fsp/src/r_sci_i2c/r_sci_i2c.o
LOAD ./ra/fsp/src/r_rtc/r_rtc.o
LOAD ./ra/fsp/src/r_ioport/r_ioport.o
LOAD ./ra/fsp/src/r_gpt/r_gpt.o
LOAD ./ra/fsp/src/r_flash_hp/r_flash_hp.o
LOAD ./ra/fsp/src/r_dtc/r_dtc.o
LOAD ./ra/fsp/src/r_crc/r_crc.o
LOAD ./ra/fsp/src/r_agt/r_agt.o
LOAD ./ra/fsp/src/r_adc/r_adc.o
LOAD ./ra/fsp/src/bsp/mcu/all/bsp_clocks.o
LOAD ./ra/fsp/src/bsp/mcu/all/bsp_common.o
LOAD ./ra/fsp/src/bsp/mcu/all/bsp_delay.o
LOAD ./ra/fsp/src/bsp/mcu/all/bsp_group_irq.o
LOAD ./ra/fsp/src/bsp/mcu/all/bsp_guard.o
LOAD ./ra/fsp/src/bsp/mcu/all/bsp_io.o
LOAD ./ra/fsp/src/bsp/mcu/all/bsp_irq.o
LOAD ./ra/fsp/src/bsp/mcu/all/bsp_register_protection.o
LOAD ./ra/fsp/src/bsp/mcu/all/bsp_rom_registers.o
LOAD ./ra/fsp/src/bsp/mcu/all/bsp_sbrk.o
LOAD ./ra/fsp/src/bsp/mcu/all/bsp_security.o
LOAD ./ra/fsp/src/bsp/cmsis/Device/RENESAS/Source/startup.o
LOAD ./ra/fsp/src/bsp/cmsis/Device/RENESAS/Source/system.o
END GROUP
START GROUP
LOAD c:/renesas/ra/e2studio_v2023-07_fsp_v4.6.0/toolchains/gcc_arm/arm-gnu-toolchain-12.2.mpacbti-rel1-mingw-w64-i686-arm-none-eabi/bin/../lib/gcc/arm-none-eabi/12.2.1/thumb/v8-m.main+fp/hard\libgcc.a
LOAD c:/renesas/ra/e2studio_v2023-07_fsp_v4.6.0/toolchains/gcc_arm/arm-gnu-toolchain-12.2.mpacbti-rel1-mingw-w64-i686-arm-none-eabi/bin/../lib/gcc/arm-none-eabi/12.2.1/thumb/v8-m.main+fp/hard\libg_nano.a
LOAD c:/renesas/ra/e2studio_v2023-07_fsp_v4.6.0/toolchains/gcc_arm/arm-gnu-toolchain-12.2.mpacbti-rel1-mingw-w64-i686-arm-none-eabi/bin/../lib/gcc/arm-none-eabi/12.2.1/thumb/v8-m.main+fp/hard\libc_nano.a
END GROUP
START GROUP
LOAD c:/renesas/ra/e2studio_v2023-07_fsp_v4.6.0/toolchains/gcc_arm/arm-gnu-toolchain-12.2.mpacbti-rel1-mingw-w64-i686-arm-none-eabi/bin/../lib/gcc/arm-none-eabi/12.2.1/thumb/v8-m.main+fp/hard\libgcc.a
LOAD c:/renesas/ra/e2studio_v2023-07_fsp_v4.6.0/toolchains/gcc_arm/arm-gnu-toolchain-12.2.mpacbti-rel1-mingw-w64-i686-arm-none-eabi/bin/../lib/gcc/arm-none-eabi/12.2.1/thumb/v8-m.main+fp/hard\libc_nano.a
LOAD c:/renesas/ra/e2studio_v2023-07_fsp_v4.6.0/toolchains/gcc_arm/arm-gnu-toolchain-12.2.mpacbti-rel1-mingw-w64-i686-arm-none-eabi/bin/../lib/gcc/arm-none-eabi/12.2.1/thumb/v8-m.main+fp/hard\librdimon_nano.a
END GROUP
START GROUP
LOAD c:/renesas/ra/e2studio_v2023-07_fsp_v4.6.0/toolchains/gcc_arm/arm-gnu-toolchain-12.2.mpacbti-rel1-mingw-w64-i686-arm-none-eabi/bin/../lib/gcc/arm-none-eabi/12.2.1/thumb/v8-m.main+fp/hard\libgcc.a
LOAD c:/renesas/ra/e2studio_v2023-07_fsp_v4.6.0/toolchains/gcc_arm/arm-gnu-toolchain-12.2.mpacbti-rel1-mingw-w64-i686-arm-none-eabi/bin/../lib/gcc/arm-none-eabi/12.2.1/thumb/v8-m.main+fp/hard\libc_nano.a
LOAD c:/renesas/ra/e2studio_v2023-07_fsp_v4.6.0/toolchains/gcc_arm/arm-gnu-toolchain-12.2.mpacbti-rel1-mingw-w64-i686-arm-none-eabi/bin/../lib/gcc/arm-none-eabi/12.2.1/thumb/v8-m.main+fp/hard\librdimon_nano.a
END GROUP
LOAD c:/renesas/ra/e2studio_v2023-07_fsp_v4.6.0/toolchains/gcc_arm/arm-gnu-toolchain-12.2.mpacbti-rel1-mingw-w64-i686-arm-none-eabi/bin/../lib/gcc/arm-none-eabi/12.2.1/thumb/v8-m.main+fp/hard/crtend.o
LOAD c:/renesas/ra/e2studio_v2023-07_fsp_v4.6.0/toolchains/gcc_arm/arm-gnu-toolchain-12.2.mpacbti-rel1-mingw-w64-i686-arm-none-eabi/bin/../lib/gcc/arm-none-eabi/12.2.1/thumb/v8-m.main+fp/hard/crtn.o
                0x20000000                        RAM_START = 0x20000000
                0x00020000                        RAM_LENGTH = 0x20000
                0x00000000                        FLASH_START = 0x0
                0x00060000                        FLASH_LENGTH = 0x60000
                0x08000000                        DATA_FLASH_START = 0x8000000
                0x00002000                        DATA_FLASH_LENGTH = 0x2000
                0x0100a100                        OPTION_SETTING_START = 0x100a100
                0x00000100                        OPTION_SETTING_LENGTH = 0x100
                0x0100a200                        OPTION_SETTING_S_START = 0x100a200
                0x00000100                        OPTION_SETTING_S_LENGTH = 0x100
                0x00000000                        ID_CODE_START = 0x0
                0x00000000                        ID_CODE_LENGTH = 0x0
                0x80010000                        SDRAM_START = 0x80010000
                0x00000000                        SDRAM_LENGTH = 0x0
                0x60000000                        QSPI_FLASH_START = 0x60000000
                0x04000000                        QSPI_FLASH_LENGTH = 0x4000000
                0x80020000                        OSPI_DEVICE_0_START = 0x80020000
                0x00000000                        OSPI_DEVICE_0_LENGTH = 0x0
                0x80030000                        OSPI_DEVICE_1_START = 0x80030000
                0x00000000                        OSPI_DEVICE_1_LENGTH = 0x0
                0x04000000                        QSPI_FLASH_PRV_LENGTH = DEFINED (QSPI_FLASH_SIZE)?ABSOLUTE (QSPI_FLASH_SIZE):ABSOLUTE (QSPI_FLASH_LENGTH)
                0x00000000                        OSPI_DEVICE_0_PRV_LENGTH = DEFINED (OSPI_DEVICE_0_SIZE)?ABSOLUTE (OSPI_DEVICE_0_SIZE):ABSOLUTE (OSPI_DEVICE_0_LENGTH)
                0x00000000                        OSPI_DEVICE_1_PRV_LENGTH = DEFINED (OSPI_DEVICE_1_SIZE)?ABSOLUTE (OSPI_DEVICE_1_SIZE):ABSOLUTE (OSPI_DEVICE_1_LENGTH)
                0x00000000                        __RESERVE_NS_RAM = ((! (DEFINED (PROJECT_NONSECURE)) && DEFINED (RAM_NS_BUFFER_LENGTH)) && (OPTION_SETTING_S_LENGTH != 0x0))
                0x00000000                        RAM_NS_BUFFER_BLOCK_LENGTH = DEFINED (RAM_NS_BUFFER_LENGTH)?ALIGN (RAM_NS_BUFFER_LENGTH, 0x2000):0x0
                0x00000000                        RAM_NS_BUFFER_LENGTH = DEFINED (RAM_NS_BUFFER_LENGTH)?RAM_NS_BUFFER_LENGTH:0x0
                0x20020000                        RAM_NS_BUFFER_START = ((RAM_START + RAM_LENGTH) - RAM_NS_BUFFER_LENGTH)
                0x20020000                        RAM_NS_BUFFER_BLOCK_START = ((RAM_START + RAM_LENGTH) - RAM_NS_BUFFER_BLOCK_LENGTH)
                0x0100a180                        OPTION_SETTING_START_NS = 0x100a180
                0x00000001                        __bl_FSP_BOOTABLE_IMAGE = 0x1
                0x00000001                        __bln_FSP_BOOTABLE_IMAGE = 0x1
                0x00000001                        PROJECT_SECURE_OR_FLAT = ((! (DEFINED (PROJECT_NONSECURE)) && OPTION_SETTING_LENGTH) && ! (DEFINED (FSP_BOOTABLE_IMAGE)))
                0x00000000                        USE_OPTION_SETTING_NS = (DEFINED (PROJECT_NONSECURE) && ! (DEFINED (FSP_BOOTABLE_IMAGE)))
                0x00000000                        __bl_FLASH_IMAGE_START = ! (DEFINED (FLASH_BOOTLOADER_LENGTH))?0x0:(FLASH_APPLICATION_IMAGE_NUMBER == 0x1)?(FLASH_BOOTLOADER_LENGTH + FLASH_BOOTLOADER_HEADER_LENGTH):(((FLASH_BOOTLOADER_LENGTH + FLASH_BOOTLOADER_SCRATCH_LENGTH) + FLASH_APPLICATION_S_LENGTH) + FLASH_BOOTLOADER_HEADER_LENGTH)
                0x00000000                        __bl_FLASH_IMAGE_LENGTH = ! (DEFINED (FLASH_BOOTLOADER_LENGTH))?0x0:(FLASH_APPLICATION_S_LENGTH - FLASH_BOOTLOADER_HEADER_LENGTH)
                0x00000000                        __bl_FLASH_IMAGE_END = (__bl_FLASH_IMAGE_START + __bl_FLASH_IMAGE_LENGTH)
                0x00000000                        __bl_FLASH_NS_START = ! (DEFINED (FLASH_BOOTLOADER_LENGTH))?0x0:(FLASH_APPLICATION_NS_LENGTH == 0x0)?__bl_FLASH_IMAGE_END:((__bl_FLASH_IMAGE_START - FLASH_BOOTLOADER_HEADER_LENGTH) + FLASH_APPLICATION_S_LENGTH)
                0x00000000                        __bl_FLASH_NSC_START = ! (DEFINED (FLASH_BOOTLOADER_LENGTH))?0x0:(FLASH_APPLICATION_NS_LENGTH == 0x0)?__bl_FLASH_IMAGE_END:(__bl_FLASH_NS_START - FLASH_APPLICATION_NSC_LENGTH)
                0x00000000                        __bl_RAM_NS_START = ! (DEFINED (FLASH_BOOTLOADER_LENGTH))?0x0:(FLASH_APPLICATION_NS_LENGTH == 0x0)?(RAM_START + RAM_LENGTH):((RAM_START + RAM_LENGTH) - RAM_APPLICATION_NS_LENGTH)
                0x00000000                        __bl_RAM_NSC_START = ! (DEFINED (FLASH_BOOTLOADER_LENGTH))?0x0:(FLASH_APPLICATION_NS_LENGTH == 0x0)?(RAM_START + RAM_LENGTH):(__bl_RAM_NS_START - RAM_APPLICATION_NSC_LENGTH)
                0x00000000                        __bl_FLASH_NS_IMAGE_START = ! (DEFINED (FLASH_BOOTLOADER_LENGTH))?0x0:(FLASH_APPLICATION_NS_LENGTH == 0x0)?__bl_FLASH_IMAGE_END:(__bl_FLASH_NS_START + FLASH_BOOTLOADER_HEADER_LENGTH_2)
                0x00000000                        __bln_FLASH_IMAGE_START = __bl_FLASH_NS_IMAGE_START
                0x00000000                        __bln_FLASH_IMAGE_LENGTH = ! (DEFINED (FLASH_BOOTLOADER_LENGTH))?0x0:(FLASH_APPLICATION_NS_LENGTH == 0x0)?__bl_FLASH_IMAGE_END:(FLASH_APPLICATION_NS_LENGTH - FLASH_BOOTLOADER_HEADER_LENGTH_2)
                0x00010000                        FLASH_ORIGIN = DEFINED (FLASH_IMAGE_START)?FLASH_IMAGE_START:FLASH_START
                0x00050000                        LIMITED_FLASH_LENGTH = DEFINED (FLASH_IMAGE_LENGTH)?FLASH_IMAGE_LENGTH:DEFINED (FLASH_BOOTLOADER_LENGTH)?FLASH_BOOTLOADER_LENGTH:FLASH_LENGTH
START GROUP
LOAD c:/renesas/ra/e2studio_v2023-07_fsp_v4.6.0/toolchains/gcc_arm/arm-gnu-toolchain-12.2.mpacbti-rel1-mingw-w64-i686-arm-none-eabi/bin/../lib/gcc/arm-none-eabi/12.2.1/thumb/v8-m.main+fp/hard\libgcc.a
LOAD c:/renesas/ra/e2studio_v2023-07_fsp_v4.6.0/toolchains/gcc_arm/arm-gnu-toolchain-12.2.mpacbti-rel1-mingw-w64-i686-arm-none-eabi/bin/../lib/gcc/arm-none-eabi/12.2.1/thumb/v8-m.main+fp/hard\libc.a
LOAD c:/renesas/ra/e2studio_v2023-07_fsp_v4.6.0/toolchains/gcc_arm/arm-gnu-toolchain-12.2.mpacbti-rel1-mingw-w64-i686-arm-none-eabi/bin/../lib/gcc/arm-none-eabi/12.2.1/thumb/v8-m.main+fp/hard\libm.a
LOAD c:/renesas/ra/e2studio_v2023-07_fsp_v4.6.0/toolchains/gcc_arm/arm-gnu-toolchain-12.2.mpacbti-rel1-mingw-w64-i686-arm-none-eabi/bin/../lib/gcc/arm-none-eabi/12.2.1/thumb/v8-m.main+fp/hard\libnosys.a
END GROUP

.text           0x00010000     0x9edc
                0x00000000                        __tz_FLASH_S = ABSOLUTE (FLASH_START)
                0x00010000                        __ROM_Start = .
 *(.fixed_vectors*)
 .fixed_vectors
                0x00010000       0x40 ./ra/fsp/src/bsp/cmsis/Device/RENESAS/Source/startup.o
                0x00010000                __Vectors
 *(.application_vectors*)
 .application_vectors
                0x00010040      0x180 ./ra_gen/vector_data.o
                0x00010040                g_vector_table
                0x000101c0                        __Vectors_End = .
                0x000101c0                        . = (OPTION_SETTING_LENGTH > 0x0)?.:(__ROM_Start + 0x400)
 *(.rom_registers*)
                0x000101c0                        . = (OPTION_SETTING_LENGTH > 0x0)?.:(__ROM_Start + 0x500)
                0x00010200                        . = ALIGN (0x80)
 *fill*         0x000101c0       0x40 ff
 *(.mcuboot_sce9_key*)
 *(.text*)
 .text.deregister_tm_clones
                0x00010200       0x1c c:/renesas/ra/e2studio_v2023-07_fsp_v4.6.0/toolchains/gcc_arm/arm-gnu-toolchain-12.2.mpacbti-rel1-mingw-w64-i686-arm-none-eabi/bin/../lib/gcc/arm-none-eabi/12.2.1/thumb/v8-m.main+fp/hard/crtbegin.o
 .text.register_tm_clones
                0x0001021c       0x28 c:/renesas/ra/e2studio_v2023-07_fsp_v4.6.0/toolchains/gcc_arm/arm-gnu-toolchain-12.2.mpacbti-rel1-mingw-w64-i686-arm-none-eabi/bin/../lib/gcc/arm-none-eabi/12.2.1/thumb/v8-m.main+fp/hard/crtbegin.o
 .text.__do_global_dtors_aux
                0x00010244       0x28 c:/renesas/ra/e2studio_v2023-07_fsp_v4.6.0/toolchains/gcc_arm/arm-gnu-toolchain-12.2.mpacbti-rel1-mingw-w64-i686-arm-none-eabi/bin/../lib/gcc/arm-none-eabi/12.2.1/thumb/v8-m.main+fp/hard/crtbegin.o
 .text.frame_dummy
                0x0001026c       0x24 c:/renesas/ra/e2studio_v2023-07_fsp_v4.6.0/toolchains/gcc_arm/arm-gnu-toolchain-12.2.mpacbti-rel1-mingw-w64-i686-arm-none-eabi/bin/../lib/gcc/arm-none-eabi/12.2.1/thumb/v8-m.main+fp/hard/crtbegin.o
 .text.movingmean
                0x00010290       0x80 ./src/adc_temp.o
 .text.get_motor_temp
                0x00010310       0x38 ./src/adc_temp.o
                0x00010310                get_motor_temp
 .text.get_hvamp_temp
                0x00010348       0x3c ./src/adc_temp.o
                0x00010348                get_hvamp_temp
 *fill*         0x00010384        0x4 ff
 .text.get_cpu_temp
                0x00010388       0x68 ./src/adc_temp.o
                0x00010388                get_cpu_temp
 .text.update_adcvalue
                0x000103f0       0x90 ./src/adc_temp.o
                0x000103f0                update_adcvalue
 .text.GetCRC8.constprop.0
                0x00010480       0x38 ./src/angle.o
 .text.sci_spi_callback
                0x000104b8       0x18 ./src/angle.o
                0x000104b8                sci_spi_callback
 .text.tad2141_readstream
                0x000104d0       0xa8 ./src/angle.o
                0x000104d0                tad2141_readstream
 .text.tad2141_init
                0x00010578       0xdc ./src/angle.o
                0x00010578                tad2141_init
 .text.RestoreControlTable2FactoryDefaults
                0x00010654       0xd4 ./src/control_table.o
                0x00010654                RestoreControlTable2FactoryDefaults
 .text.write_item
                0x00010728       0xd4 ./src/control_table.o
                0x00010728                write_item
 .text.read_item
                0x000107fc       0x60 ./src/control_table.o
                0x000107fc                read_item
 .text.SaveCcontroltableToNVM
                0x0001085c       0xc0 ./src/control_table.o
                0x0001085c                SaveCcontroltableToNVM
 *fill*         0x0001091c        0x4 ff
 .text.LoadCcontroltableFromNVM
                0x00010920       0xb4 ./src/control_table.o
                0x00010920                LoadCcontroltableFromNVM
 .text.__NVIC_SystemReset
                0x000109d4       0x24 ./src/hal_entry.o
 .text.CurveInterpolation
                0x000109f8      0x150 ./src/hal_entry.o
 .text.ReqNumConversionItems
                0x00010b48       0xf8 ./src/hal_entry.o
 .text.led_on   0x00010c40       0x18 ./src/hal_entry.o
                0x00010c40                led_on
 .text.led_off  0x00010c58       0x18 ./src/hal_entry.o
                0x00010c58                led_off
 .text.rgt0_callback
                0x00010c70     0x1320 ./src/hal_entry.o
                0x00010c70                rgt0_callback
 .text.hal_entry
                0x00011f90      0x1a0 ./src/hal_entry.o
                0x00011f90                hal_entry
 .text.R_BSP_WarmStart
                0x00012130       0x18 ./src/hal_entry.o
                0x00012130                R_BSP_WarmStart
 .text.interp1dim
                0x00012148       0x8c ./src/interpolation.o
                0x00012148                interp1dim
 .text.MonConditions
                0x000121d4      0x128 ./src/monitor.o
                0x000121d4                MonConditions
 *fill*         0x000122fc        0x4 ff
 .text.write_item_callback
                0x00012300      0x1cc ./src/packet.o
                0x00012300                write_item_callback
 .text.concack.part.0
                0x000124cc       0x90 ./src/packet.o
 .text.cmd_rb   0x0001255c       0x58 ./src/packet.o
 .text.concdec.part.0
                0x000125b4       0xc0 ./src/packet.o
 .text.cmd_cb   0x00012674       0x44 ./src/packet.o
 .text.cmd_cp   0x000126b8       0x44 ./src/packet.o
 .text.cmd_cc   0x000126fc       0x44 ./src/packet.o
 .text.cmd_cv   0x00012740       0x44 ./src/packet.o
 .text.cmd_ca   0x00012784       0x44 ./src/packet.o
 .text.cmd_sg2  0x000127c8       0xe4 ./src/packet.o
 .text.cmd_sg1  0x000128ac       0xe4 ./src/packet.o
 .text.cmd_sg0  0x00012990       0xe4 ./src/packet.o
 .text.cmd_ex   0x00012a74       0x74 ./src/packet.o
 .text.cmd_tp   0x00012ae8       0x74 ./src/packet.o
 .text.cmd_tc   0x00012b5c       0xc8 ./src/packet.o
 .text.cmd_tv   0x00012c24       0xc8 ./src/packet.o
 .text.cmd_ta   0x00012cec       0xc8 ./src/packet.o
 .text.cmd_wr   0x00012db4       0xd4 ./src/packet.o
 .text.cmd_st   0x00012e88       0xdc ./src/packet.o
 .text.cmd_ct   0x00012f64       0xe0 ./src/packet.o
 .text.cmd_wd   0x00013044       0x48 ./src/packet.o
 .text.cmd_id   0x0001308c       0xe8 ./src/packet.o
 .text.cmd_ini  0x00013174       0xbc ./src/packet.o
 .text.cmd_rr   0x00013230      0x43c ./src/packet.o
 .text.packet_receive
                0x0001366c      0x114 ./src/packet.o
                0x0001366c                packet_receive
 .text.packet_handling
                0x00013780      0x2b4 ./src/packet.o
                0x00013780                packet_handling
 .text.PIDReset_real
                0x00013a34       0x14 ./src/pid.o
                0x00013a34                PIDReset_real
 .text.PIDUpdate_real
                0x00013a48       0xf0 ./src/pid.o
                0x00013a48                PIDUpdate_real
 .text.sci_i2c_master_callback
                0x00013b38       0xe8 ./src/power_monitor.o
                0x00013b38                sci_i2c_master_callback
 .text.isl28022_write
                0x00013c20       0xcc ./src/power_monitor.o
                0x00013c20                isl28022_write
 .text.isl28022_read
                0x00013cec       0x58 ./src/power_monitor.o
                0x00013cec                isl28022_read
 .text.isl28022_read_ex
                0x00013d44       0x80 ./src/power_monitor.o
                0x00013d44                isl28022_read_ex
 .text.isl28022_comp_stat
                0x00013dc4       0x18 ./src/power_monitor.o
                0x00013dc4                isl28022_comp_stat
 .text.isl28022_force_reset_stat
                0x00013ddc       0x24 ./src/power_monitor.o
                0x00013ddc                isl28022_force_reset_stat
 .text.isl28022_init
                0x00013e00      0x11c ./src/power_monitor.o
                0x00013e00                isl28022_init
 .text.my_cos1000
                0x00013f1c       0x88 ./src/sintable.o
                0x00013f1c                my_cos1000
 .text.user_uart_callback
                0x00013fa4       0x6c ./src/usart.o
                0x00013fa4                user_uart_callback
 .text.us_tx_buff
                0x00014010       0x10 ./src/usart.o
                0x00014010                us_tx_buff
 .text.us_rx_buff
                0x00014020       0x1c ./src/usart.o
                0x00014020                us_rx_buff
 .text.us_putsb
                0x0001403c       0x9c ./src/usart.o
                0x0001403c                us_putsb
 .text.us_getc  0x000140d8       0x30 ./src/usart.o
                0x000140d8                us_getc
 .text.us_setbaudrate
                0x00014108       0x30 ./src/usart.o
                0x00014108                us_setbaudrate
 .text.us_init  0x00014138       0x78 ./src/usart.o
                0x00014138                us_init
 .text.startup.main
                0x000141b0        0xc ./ra_gen/main.o
                0x000141b0                main
 .text.R_SCI_UART_Write
                0x000141bc       0xac ./ra/fsp/src/r_sci_uart/r_sci_uart.o
                0x000141bc                R_SCI_UART_Write
 .text.R_SCI_UART_BaudSet
                0x00014268       0x4c ./ra/fsp/src/r_sci_uart/r_sci_uart.o
                0x00014268                R_SCI_UART_BaudSet
 .text.R_SCI_UART_Open
                0x000142b4      0x42c ./ra/fsp/src/r_sci_uart/r_sci_uart.o
                0x000142b4                R_SCI_UART_Open
 .text.R_SCI_UART_BaudCalculate
                0x000146e0      0x1d0 ./ra/fsp/src/r_sci_uart/r_sci_uart.o
                0x000146e0                R_SCI_UART_BaudCalculate
 .text.sci_uart_txi_isr
                0x000148b0      0x160 ./ra/fsp/src/r_sci_uart/r_sci_uart.o
                0x000148b0                sci_uart_txi_isr
 .text.sci_uart_rxi_isr
                0x00014a10      0x16c ./ra/fsp/src/r_sci_uart/r_sci_uart.o
                0x00014a10                sci_uart_rxi_isr
 .text.sci_uart_tei_isr
                0x00014b7c       0x80 ./ra/fsp/src/r_sci_uart/r_sci_uart.o
                0x00014b7c                sci_uart_tei_isr
 .text.sci_uart_eri_isr
                0x00014bfc       0xb8 ./ra/fsp/src/r_sci_uart/r_sci_uart.o
                0x00014bfc                sci_uart_eri_isr
 .text.R_SCI_SPI_WriteRead
                0x00014cb4      0x124 ./ra/fsp/src/r_sci_spi/r_sci_spi.o
                0x00014cb4                R_SCI_SPI_WriteRead
 .text.R_SCI_SPI_Open
                0x00014dd8      0x2d4 ./ra/fsp/src/r_sci_spi/r_sci_spi.o
                0x00014dd8                R_SCI_SPI_Open
 .text.sci_spi_txi_isr
                0x000150ac       0x6c ./ra/fsp/src/r_sci_spi/r_sci_spi.o
                0x000150ac                sci_spi_txi_isr
 .text.sci_spi_rxi_isr
                0x00015118       0x78 ./ra/fsp/src/r_sci_spi/r_sci_spi.o
                0x00015118                sci_spi_rxi_isr
 .text.sci_spi_tei_isr
                0x00015190       0x70 ./ra/fsp/src/r_sci_spi/r_sci_spi.o
                0x00015190                sci_spi_tei_isr
 .text.sci_spi_eri_isr
                0x00015200       0x78 ./ra/fsp/src/r_sci_spi/r_sci_spi.o
                0x00015200                sci_spi_eri_isr
 .text.R_SCI_I2C_SlaveAddressSet
                0x00015278        0xc ./ra/fsp/src/r_sci_i2c/r_sci_i2c.o
                0x00015278                R_SCI_I2C_SlaveAddressSet
 .text.R_SCI_I2C_Read
                0x00015284       0x94 ./ra/fsp/src/r_sci_i2c/r_sci_i2c.o
                0x00015284                R_SCI_I2C_Read
 .text.R_SCI_I2C_Write
                0x00015318       0x90 ./ra/fsp/src/r_sci_i2c/r_sci_i2c.o
                0x00015318                R_SCI_I2C_Write
 .text.R_SCI_I2C_Open
                0x000153a8      0x170 ./ra/fsp/src/r_sci_i2c/r_sci_i2c.o
                0x000153a8                R_SCI_I2C_Open
 .text.sci_i2c_txi_isr
                0x00015518      0x144 ./ra/fsp/src/r_sci_i2c/r_sci_i2c.o
                0x00015518                sci_i2c_txi_isr
 .text.sci_i2c_tei_isr
                0x0001565c      0x120 ./ra/fsp/src/r_sci_i2c/r_sci_i2c.o
                0x0001565c                sci_i2c_tei_isr
 .text.rtc_carry_isr
                0x0001577c       0x30 ./ra/fsp/src/r_rtc/r_rtc.o
                0x0001577c                rtc_carry_isr
 .text.R_IOPORT_Close
                0x000157ac        0xc ./ra/fsp/src/r_ioport/r_ioport.o
                0x000157ac                R_IOPORT_Close
 .text.R_IOPORT_PinRead
                0x000157b8       0x24 ./ra/fsp/src/r_ioport/r_ioport.o
                0x000157b8                R_IOPORT_PinRead
 .text.R_IOPORT_PortRead
                0x000157dc       0x14 ./ra/fsp/src/r_ioport/r_ioport.o
                0x000157dc                R_IOPORT_PortRead
 .text.R_IOPORT_PortWrite
                0x000157f0       0x1c ./ra/fsp/src/r_ioport/r_ioport.o
                0x000157f0                R_IOPORT_PortWrite
 .text.R_IOPORT_PinWrite
                0x0001580c       0x20 ./ra/fsp/src/r_ioport/r_ioport.o
                0x0001580c                R_IOPORT_PinWrite
 .text.R_IOPORT_PortDirectionSet
                0x0001582c       0x2c ./ra/fsp/src/r_ioport/r_ioport.o
                0x0001582c                R_IOPORT_PortDirectionSet
 .text.R_IOPORT_PortEventInputRead
                0x00015858       0x18 ./ra/fsp/src/r_ioport/r_ioport.o
                0x00015858                R_IOPORT_PortEventInputRead
 .text.R_IOPORT_PinEventInputRead
                0x00015870       0x34 ./ra/fsp/src/r_ioport/r_ioport.o
                0x00015870                R_IOPORT_PinEventInputRead
 .text.R_IOPORT_PortEventOutputWrite
                0x000158a4       0x1c ./ra/fsp/src/r_ioport/r_ioport.o
                0x000158a4                R_IOPORT_PortEventOutputWrite
 .text.R_IOPORT_PinEventOutputWrite
                0x000158c0       0x34 ./ra/fsp/src/r_ioport/r_ioport.o
                0x000158c0                R_IOPORT_PinEventOutputWrite
 .text.bsp_vbatt_init
                0x000158f4      0x128 ./ra/fsp/src/r_ioport/r_ioport.o
 .text.r_ioport_pins_config
                0x00015a1c       0xa8 ./ra/fsp/src/r_ioport/r_ioport.o
 .text.R_IOPORT_Open
                0x00015ac4       0x14 ./ra/fsp/src/r_ioport/r_ioport.o
                0x00015ac4                R_IOPORT_Open
 .text.R_IOPORT_PinsCfg
                0x00015ad8        0xc ./ra/fsp/src/r_ioport/r_ioport.o
                0x00015ad8                R_IOPORT_PinsCfg
 .text.R_IOPORT_PinCfg
                0x00015ae4       0xa8 ./ra/fsp/src/r_ioport/r_ioport.o
                0x00015ae4                R_IOPORT_PinCfg
 .text.R_GPT_Start
                0x00015b8c        0xc ./ra/fsp/src/r_gpt/r_gpt.o
                0x00015b8c                R_GPT_Start
 .text.r_gpt_enable_irq
                0x00015b98       0x60 ./ra/fsp/src/r_gpt/r_gpt.o
 .text.R_GPT_DutyCycleSet
                0x00015bf8      0x188 ./ra/fsp/src/r_gpt/r_gpt.o
                0x00015bf8                R_GPT_DutyCycleSet
 .text.R_GPT_Open
                0x00015d80      0x298 ./ra/fsp/src/r_gpt/r_gpt.o
                0x00015d80                R_GPT_Open
 .text.R_FLASH_HP_Close
                0x00016018       0x6c ./ra/fsp/src/r_flash_hp/r_flash_hp.o
                0x00016018                R_FLASH_HP_Close
 .text.flash_hp_enter_pe_df_mode
                0x00016084       0xd0 ./ra/fsp/src/r_flash_hp/r_flash_hp.o
 .text.R_FLASH_HP_Open
                0x00016154      0x1e0 ./ra/fsp/src/r_flash_hp/r_flash_hp.o
                0x00016154                R_FLASH_HP_Open
 .text.R_FLASH_HP_Erase
                0x00016334      0x18c ./ra/fsp/src/r_flash_hp/r_flash_hp.o
                0x00016334                R_FLASH_HP_Erase
 .text.R_FLASH_HP_Write
                0x000164c0      0x224 ./ra/fsp/src/r_flash_hp/r_flash_hp.o
                0x000164c0                R_FLASH_HP_Write
 .text.R_DTC_Reset
                0x000166e4       0x98 ./ra/fsp/src/r_dtc/r_dtc.o
                0x000166e4                R_DTC_Reset
 .text.R_DTC_SoftwareStart
                0x0001677c        0x4 ./ra/fsp/src/r_dtc/r_dtc.o
                0x0001677c                R_DTC_SoftwareStart
 .text.R_DTC_SoftwareStop
                0x00016780        0x4 ./ra/fsp/src/r_dtc/r_dtc.o
                0x00016780                R_DTC_SoftwareStop
 .text.R_DTC_Enable
                0x00016784       0x20 ./ra/fsp/src/r_dtc/r_dtc.o
                0x00016784                R_DTC_Enable
 .text.R_DTC_Disable
                0x000167a4       0x20 ./ra/fsp/src/r_dtc/r_dtc.o
                0x000167a4                R_DTC_Disable
 .text.R_DTC_InfoGet
                0x000167c4       0x5c ./ra/fsp/src/r_dtc/r_dtc.o
                0x000167c4                R_DTC_InfoGet
 .text.R_DTC_Close
                0x00016820       0x34 ./ra/fsp/src/r_dtc/r_dtc.o
                0x00016820                R_DTC_Close
 .text.R_DTC_Open
                0x00016854       0xbc ./ra/fsp/src/r_dtc/r_dtc.o
                0x00016854                R_DTC_Open
 .text.R_DTC_Reconfigure
                0x00016910       0x84 ./ra/fsp/src/r_dtc/r_dtc.o
                0x00016910                R_DTC_Reconfigure
 .text.R_CRC_Open
                0x00016994       0x44 ./ra/fsp/src/r_crc/r_crc.o
                0x00016994                R_CRC_Open
 .text.R_CRC_Close
                0x000169d8       0x28 ./ra/fsp/src/r_crc/r_crc.o
                0x000169d8                R_CRC_Close
 .text.R_CRC_Calculate
                0x00016a00       0x88 ./ra/fsp/src/r_crc/r_crc.o
                0x00016a00                R_CRC_Calculate
 .text.R_AGT_Enable
                0x00016a88       0x24 ./ra/fsp/src/r_agt/r_agt.o
                0x00016a88                R_AGT_Enable
 .text.R_AGT_Open
                0x00016aac      0x150 ./ra/fsp/src/r_agt/r_agt.o
                0x00016aac                R_AGT_Open
 .text.agt_int_isr
                0x00016bfc       0x9c ./ra/fsp/src/r_agt/r_agt.o
                0x00016bfc                agt_int_isr
 .text.R_ADC_ScanStart
                0x00016c98        0xc ./ra/fsp/src/r_adc/r_adc.o
                0x00016c98                R_ADC_ScanStart
 .text.R_ADC_Read
                0x00016ca4       0x10 ./ra/fsp/src/r_adc/r_adc.o
                0x00016ca4                R_ADC_Read
 .text.R_ADC_ScanCfg
                0x00016cb4      0x1e8 ./ra/fsp/src/r_adc/r_adc.o
                0x00016cb4                R_ADC_ScanCfg
 .text.R_ADC_Open
                0x00016e9c      0x23c ./ra/fsp/src/r_adc/r_adc.o
                0x00016e9c                R_ADC_Open
 .text.SystemCoreClockUpdate
                0x000170d8       0x28 ./ra/fsp/src/bsp/mcu/all/bsp_clocks.o
                0x000170d8                SystemCoreClockUpdate
 .text.R_BSP_SubClockStabilizeWaitAfterReset
                0x00017100        0x4 ./ra/fsp/src/bsp/mcu/all/bsp_clocks.o
                0x00017100                R_BSP_SubClockStabilizeWaitAfterReset
 .text.bsp_clock_init
                0x00017104      0x174 ./ra/fsp/src/bsp/mcu/all/bsp_clocks.o
                0x00017104                bsp_clock_init
 .text.R_BSP_Init_RTC
                0x00017278       0x28 ./ra/fsp/src/bsp/mcu/all/bsp_clocks.o
                0x00017278                R_BSP_Init_RTC
 .text.bsp_init_internal
                0x000172a0        0x4 ./ra/fsp/src/bsp/mcu/all/bsp_common.o
                0x000172a0                bsp_init_internal
                0x000172a0                bsp_init
 .text.bsp_prv_software_delay_loop
                0x000172a4        0xc ./ra/fsp/src/bsp/mcu/all/bsp_delay.o
                0x000172a4                bsp_prv_software_delay_loop
 .text.R_BSP_SoftwareDelay
                0x000172b0       0x58 ./ra/fsp/src/bsp/mcu/all/bsp_delay.o
                0x000172b0                R_BSP_SoftwareDelay
 .text.NMI_Handler
                0x00017308       0x38 ./ra/fsp/src/bsp/mcu/all/bsp_group_irq.o
                0x00017308                NMI_Handler
 .text.bsp_irq_cfg
                0x00017340       0xa0 ./ra/fsp/src/bsp/mcu/all/bsp_irq.o
                0x00017340                bsp_irq_cfg
 .text.R_BSP_RegisterProtectEnable
                0x000173e0       0x60 ./ra/fsp/src/bsp/mcu/all/bsp_register_protection.o
                0x000173e0                R_BSP_RegisterProtectEnable
 .text.R_BSP_RegisterProtectDisable
                0x00017440       0x54 ./ra/fsp/src/bsp/mcu/all/bsp_register_protection.o
                0x00017440                R_BSP_RegisterProtectDisable
 .text.Default_Handler
                0x00017494        0x4 ./ra/fsp/src/bsp/cmsis/Device/RENESAS/Source/startup.o
                0x00017494                DebugMon_Handler
                0x00017494                HardFault_Handler
                0x00017494                SysTick_Handler
                0x00017494                PendSV_Handler
                0x00017494                UsageFault_Handler
                0x00017494                SecureFault_Handler
                0x00017494                Default_Handler
                0x00017494                MemManage_Handler
                0x00017494                SVC_Handler
                0x00017494                BusFault_Handler
 .text.Reset_Handler
                0x00017498        0xc ./ra/fsp/src/bsp/cmsis/Device/RENESAS/Source/startup.o
                0x00017498                Reset_Handler
 .text.SystemInit
                0x000174a4       0xc4 ./ra/fsp/src/bsp/cmsis/Device/RENESAS/Source/system.o
                0x000174a4                SystemInit
 .text          0x00017568      0x378 c:/renesas/ra/e2studio_v2023-07_fsp_v4.6.0/toolchains/gcc_arm/arm-gnu-toolchain-12.2.mpacbti-rel1-mingw-w64-i686-arm-none-eabi/bin/../lib/gcc/arm-none-eabi/12.2.1/thumb/v8-m.main+fp/hard\libgcc.a(_arm_addsubdf3.o)
                0x00017568                __aeabi_drsub
                0x00017570                __aeabi_dsub
                0x00017570                __subdf3
                0x00017574                __aeabi_dadd
                0x00017574                __adddf3
                0x000177ec                __floatunsidf
                0x000177ec                __aeabi_ui2d
                0x0001780c                __floatsidf
                0x0001780c                __aeabi_i2d
                0x00017830                __aeabi_f2d
                0x00017830                __extendsfdf2
                0x00017874                __floatundidf
                0x00017874                __aeabi_ul2d
                0x00017884                __floatdidf
                0x00017884                __aeabi_l2d
 .text          0x000178e0      0x424 c:/renesas/ra/e2studio_v2023-07_fsp_v4.6.0/toolchains/gcc_arm/arm-gnu-toolchain-12.2.mpacbti-rel1-mingw-w64-i686-arm-none-eabi/bin/../lib/gcc/arm-none-eabi/12.2.1/thumb/v8-m.main+fp/hard\libgcc.a(_arm_muldivdf3.o)
                0x000178e0                __aeabi_dmul
                0x000178e0                __muldf3
                0x00017b34                __divdf3
                0x00017b34                __aeabi_ddiv
 .text          0x00017d04      0x110 c:/renesas/ra/e2studio_v2023-07_fsp_v4.6.0/toolchains/gcc_arm/arm-gnu-toolchain-12.2.mpacbti-rel1-mingw-w64-i686-arm-none-eabi/bin/../lib/gcc/arm-none-eabi/12.2.1/thumb/v8-m.main+fp/hard\libgcc.a(_arm_cmpdf2.o)
                0x00017d04                __gtdf2
                0x00017d04                __gedf2
                0x00017d0c                __ltdf2
                0x00017d0c                __ledf2
                0x00017d14                __nedf2
                0x00017d14                __eqdf2
                0x00017d14                __cmpdf2
                0x00017d90                __aeabi_cdrcmple
                0x00017da0                __aeabi_cdcmpeq
                0x00017da0                __aeabi_cdcmple
                0x00017db0                __aeabi_dcmpeq
                0x00017dc4                __aeabi_dcmplt
                0x00017dd8                __aeabi_dcmple
                0x00017dec                __aeabi_dcmpge
                0x00017e00                __aeabi_dcmpgt
 .text          0x00017e14       0x50 c:/renesas/ra/e2studio_v2023-07_fsp_v4.6.0/toolchains/gcc_arm/arm-gnu-toolchain-12.2.mpacbti-rel1-mingw-w64-i686-arm-none-eabi/bin/../lib/gcc/arm-none-eabi/12.2.1/thumb/v8-m.main+fp/hard\libgcc.a(_arm_fixdfsi.o)
                0x00017e14                __aeabi_d2iz
                0x00017e14                __fixdfsi
 .text          0x00017e64       0x40 c:/renesas/ra/e2studio_v2023-07_fsp_v4.6.0/toolchains/gcc_arm/arm-gnu-toolchain-12.2.mpacbti-rel1-mingw-w64-i686-arm-none-eabi/bin/../lib/gcc/arm-none-eabi/12.2.1/thumb/v8-m.main+fp/hard\libgcc.a(_arm_fixunsdfsi.o)
                0x00017e64                __aeabi_d2uiz
                0x00017e64                __fixunsdfsi
 .text          0x00017ea4       0xa0 c:/renesas/ra/e2studio_v2023-07_fsp_v4.6.0/toolchains/gcc_arm/arm-gnu-toolchain-12.2.mpacbti-rel1-mingw-w64-i686-arm-none-eabi/bin/../lib/gcc/arm-none-eabi/12.2.1/thumb/v8-m.main+fp/hard\libgcc.a(_aeabi_ldivmod.o)
                0x00017ea4                __aeabi_ldivmod
 .text.__udivmoddi4
                0x00017f44      0x2e4 c:/renesas/ra/e2studio_v2023-07_fsp_v4.6.0/toolchains/gcc_arm/arm-gnu-toolchain-12.2.mpacbti-rel1-mingw-w64-i686-arm-none-eabi/bin/../lib/gcc/arm-none-eabi/12.2.1/thumb/v8-m.main+fp/hard\libgcc.a(_udivmoddi4.o)
                0x00017f44                __udivmoddi4
 .text          0x00018228        0x4 c:/renesas/ra/e2studio_v2023-07_fsp_v4.6.0/toolchains/gcc_arm/arm-gnu-toolchain-12.2.mpacbti-rel1-mingw-w64-i686-arm-none-eabi/bin/../lib/gcc/arm-none-eabi/12.2.1/thumb/v8-m.main+fp/hard\libgcc.a(_dvmd_tls.o)
                0x00018228                __aeabi_idiv0
                0x00018228                __aeabi_ldiv0
 .text.__itoa   0x0001822c       0x30 c:/renesas/ra/e2studio_v2023-07_fsp_v4.6.0/toolchains/gcc_arm/arm-gnu-toolchain-12.2.mpacbti-rel1-mingw-w64-i686-arm-none-eabi/bin/../lib/gcc/arm-none-eabi/12.2.1/thumb/v8-m.main+fp/hard\libg_nano.a(libc_a-itoa.o)
                0x0001822c                __itoa
 .text._strtol_l.constprop.0
                0x0001825c       0xfc c:/renesas/ra/e2studio_v2023-07_fsp_v4.6.0/toolchains/gcc_arm/arm-gnu-toolchain-12.2.mpacbti-rel1-mingw-w64-i686-arm-none-eabi/bin/../lib/gcc/arm-none-eabi/12.2.1/thumb/v8-m.main+fp/hard\libg_nano.a(libc_a-strtol.o)
 .text.strtol   0x00018358       0x14 c:/renesas/ra/e2studio_v2023-07_fsp_v4.6.0/toolchains/gcc_arm/arm-gnu-toolchain-12.2.mpacbti-rel1-mingw-w64-i686-arm-none-eabi/bin/../lib/gcc/arm-none-eabi/12.2.1/thumb/v8-m.main+fp/hard\libg_nano.a(libc_a-strtol.o)
                0x00018358                strtol
 .text.__utoa   0x0001836c       0x84 c:/renesas/ra/e2studio_v2023-07_fsp_v4.6.0/toolchains/gcc_arm/arm-gnu-toolchain-12.2.mpacbti-rel1-mingw-w64-i686-arm-none-eabi/bin/../lib/gcc/arm-none-eabi/12.2.1/thumb/v8-m.main+fp/hard\libg_nano.a(libc_a-utoa.o)
                0x0001836c                __utoa
 .text.memset   0x000183f0       0x10 c:/renesas/ra/e2studio_v2023-07_fsp_v4.6.0/toolchains/gcc_arm/arm-gnu-toolchain-12.2.mpacbti-rel1-mingw-w64-i686-arm-none-eabi/bin/../lib/gcc/arm-none-eabi/12.2.1/thumb/v8-m.main+fp/hard\libg_nano.a(libc_a-memset.o)
                0x000183f0                memset
 .text.strncmp  0x00018400       0x24 c:/renesas/ra/e2studio_v2023-07_fsp_v4.6.0/toolchains/gcc_arm/arm-gnu-toolchain-12.2.mpacbti-rel1-mingw-w64-i686-arm-none-eabi/bin/../lib/gcc/arm-none-eabi/12.2.1/thumb/v8-m.main+fp/hard\libg_nano.a(libc_a-strncmp.o)
                0x00018400                strncmp
 .text.__errno  0x00018424        0xc c:/renesas/ra/e2studio_v2023-07_fsp_v4.6.0/toolchains/gcc_arm/arm-gnu-toolchain-12.2.mpacbti-rel1-mingw-w64-i686-arm-none-eabi/bin/../lib/gcc/arm-none-eabi/12.2.1/thumb/v8-m.main+fp/hard\libg_nano.a(libc_a-errno.o)
                0x00018424                __errno
 .text.strcpy   0x00018430       0x10 c:/renesas/ra/e2studio_v2023-07_fsp_v4.6.0/toolchains/gcc_arm/arm-gnu-toolchain-12.2.mpacbti-rel1-mingw-w64-i686-arm-none-eabi/bin/../lib/gcc/arm-none-eabi/12.2.1/thumb/v8-m.main+fp/hard\libg_nano.a(libc_a-strcpy.o)
                0x00018430                strcpy
 .text.__aeabi_memcpy
                0x00018440        0x4 c:/renesas/ra/e2studio_v2023-07_fsp_v4.6.0/toolchains/gcc_arm/arm-gnu-toolchain-12.2.mpacbti-rel1-mingw-w64-i686-arm-none-eabi/bin/../lib/gcc/arm-none-eabi/12.2.1/thumb/v8-m.main+fp/hard\libg_nano.a(libc_a-aeabi_memcpy.o)
                0x00018440                __aeabi_memcpy4
                0x00018440                __aeabi_memcpy8
                0x00018440                __aeabi_memcpy
 .text.__aeabi_memclr
                0x00018444        0x6 c:/renesas/ra/e2studio_v2023-07_fsp_v4.6.0/toolchains/gcc_arm/arm-gnu-toolchain-12.2.mpacbti-rel1-mingw-w64-i686-arm-none-eabi/bin/../lib/gcc/arm-none-eabi/12.2.1/thumb/v8-m.main+fp/hard\libg_nano.a(libc_a-aeabi_memclr.o)
                0x00018444                __aeabi_memclr
                0x00018444                __aeabi_memclr4
                0x00018444                __aeabi_memclr8
 .text.memcpy   0x0001844a       0x1a c:/renesas/ra/e2studio_v2023-07_fsp_v4.6.0/toolchains/gcc_arm/arm-gnu-toolchain-12.2.mpacbti-rel1-mingw-w64-i686-arm-none-eabi/bin/../lib/gcc/arm-none-eabi/12.2.1/thumb/v8-m.main+fp/hard\libg_nano.a(libc_a-memcpy-stub.o)
                0x0001844a                memcpy
 .text          0x00018464       0x10 c:/renesas/ra/e2studio_v2023-07_fsp_v4.6.0/toolchains/gcc_arm/arm-gnu-toolchain-12.2.mpacbti-rel1-mingw-w64-i686-arm-none-eabi/bin/../lib/gcc/arm-none-eabi/12.2.1/thumb/v8-m.main+fp/hard\libg_nano.a(libc_a-strlen.o)
                0x00018464                strlen
 .text          0x00018474       0x9a c:/renesas/ra/e2studio_v2023-07_fsp_v4.6.0/toolchains/gcc_arm/arm-gnu-toolchain-12.2.mpacbti-rel1-mingw-w64-i686-arm-none-eabi/bin/../lib/gcc/arm-none-eabi/12.2.1/thumb/v8-m.main+fp/hard\libg_nano.a(libc_a-aeabi_memset-soft.o)
                0x00018474                __aeabi_memset8
                0x00018474                __aeabi_memset4
                0x00018474                __aeabi_memset
 *(.version)
 *fill*         0x0001850e        0x2 ff
 .version       0x00018510       0x50 ./ra/fsp/src/bsp/mcu/all/bsp_common.o
 *(.init)
 .init          0x00018560        0x4 c:/renesas/ra/e2studio_v2023-07_fsp_v4.6.0/toolchains/gcc_arm/arm-gnu-toolchain-12.2.mpacbti-rel1-mingw-w64-i686-arm-none-eabi/bin/../lib/gcc/arm-none-eabi/12.2.1/thumb/v8-m.main+fp/hard/crti.o
                0x00018560                _init
 .init          0x00018564        0x8 c:/renesas/ra/e2studio_v2023-07_fsp_v4.6.0/toolchains/gcc_arm/arm-gnu-toolchain-12.2.mpacbti-rel1-mingw-w64-i686-arm-none-eabi/bin/../lib/gcc/arm-none-eabi/12.2.1/thumb/v8-m.main+fp/hard/crtn.o
 *(.fini)
 .fini          0x0001856c        0x4 c:/renesas/ra/e2studio_v2023-07_fsp_v4.6.0/toolchains/gcc_arm/arm-gnu-toolchain-12.2.mpacbti-rel1-mingw-w64-i686-arm-none-eabi/bin/../lib/gcc/arm-none-eabi/12.2.1/thumb/v8-m.main+fp/hard/crti.o
                0x0001856c                _fini
 .fini          0x00018570        0x8 c:/renesas/ra/e2studio_v2023-07_fsp_v4.6.0/toolchains/gcc_arm/arm-gnu-toolchain-12.2.mpacbti-rel1-mingw-w64-i686-arm-none-eabi/bin/../lib/gcc/arm-none-eabi/12.2.1/thumb/v8-m.main+fp/hard/crtn.o
 *crtbegin.o(.ctors)
 *crtbegin?.o(.ctors)
 *(EXCLUDE_FILE(*crtend.o *crtend?.o) .ctors)
 *(SORT_BY_NAME(.ctors.*))
 *(.ctors)
 *crtbegin.o(.dtors)
 *crtbegin?.o(.dtors)
 *(EXCLUDE_FILE(*crtend.o *crtend?.o) .dtors)
 *(SORT_BY_NAME(.dtors.*))
 *(.dtors)
 *(.rodata*)
 .rodata.interp_hvamp_1d
                0x00018578       0x90 ./src/adc_temp.o
 .rodata.interp_ntc_1d
                0x00018608       0x58 ./src/adc_temp.o
 .rodata        0x00018660      0x105 ./src/angle.o
 *fill*         0x00018765        0x3 ff
 .rodata.ItemInfo
                0x00018768      0x7f0 ./src/control_table.o
                0x00018768                ItemInfo
 .rodata.Default_ControlTable
                0x00018f58      0x188 ./src/control_table.o
                0x00018f58                Default_ControlTable
 .rodata.interp_current_compliance_ar_w
                0x000190e0        0x4 ./src/global_variables.o
                0x000190e0                interp_current_compliance_ar_w
 .rodata.interp_angle_compliance_ar_w
                0x000190e4        0x4 ./src/global_variables.o
                0x000190e4                interp_angle_compliance_ar_w
 .rodata.interp_tad2141_ar_w
                0x000190e8        0x4 ./src/global_variables.o
                0x000190e8                interp_tad2141_ar_w
 .rodata.pwm_gain.2
                0x000190ec       0x14 ./src/hal_entry.o
 .rodata.baudrate_list
                0x00019100       0x3c ./src/hal_entry.o
                0x00019100                baudrate_list
 .rodata.concack.part.0.str1.4
                0x0001913c       0x10 ./src/packet.o
 .rodata.concdec.part.0.str1.4
                0x0001914c        0x2 ./src/packet.o
 *fill*         0x0001914e        0x2 ff
 .rodata.cmd_ct.str1.4
                0x00019150        0xc ./src/packet.o
 .rodata.cmd_rr.str1.4
                0x0001915c        0x2 ./src/packet.o
 *fill*         0x0001915e        0x2 ff
 .rodata.packet_handling.str1.4
                0x00019160        0x2 ./src/packet.o
 *fill*         0x00019162        0x2 ff
 .rodata.CmdInfo
                0x00019164      0x150 ./src/packet.o
 .rodata.SindegTable
                0x000192b4      0x70a ./src/sintable.o
 *fill*         0x000199be        0x2 ff
 .rodata.g_ioport
                0x000199c0        0xc ./ra_gen/common_data.o
                0x000199c0                g_ioport
 .rodata.g_uart4_cfg
                0x000199cc       0x20 ./ra_gen/hal_data.o
                0x000199cc                g_uart4_cfg
 .rodata.g_uart4_cfg_extend
                0x000199ec       0x14 ./ra_gen/hal_data.o
                0x000199ec                g_uart4_cfg_extend
 .rodata.g_i2c3_cfg
                0x00019a00       0x28 ./ra_gen/hal_data.o
                0x00019a00                g_i2c3_cfg
 .rodata.g_i2c3_cfg_extend
                0x00019a28        0x6 ./ra_gen/hal_data.o
                0x00019a28                g_i2c3_cfg_extend
 *fill*         0x00019a2e        0x2 ff
 .rodata.g_spi2_cfg
                0x00019a30       0x24 ./ra_gen/hal_data.o
                0x00019a30                g_spi2_cfg
 .rodata.g_spi2_cfg_extend
                0x00019a54        0x3 ./ra_gen/hal_data.o
                0x00019a54                g_spi2_cfg_extend
 *fill*         0x00019a57        0x1 ff
 .rodata.g_transfer0
                0x00019a58        0xc ./ra_gen/hal_data.o
                0x00019a58                g_transfer0
 .rodata.g_transfer0_cfg
                0x00019a64        0x8 ./ra_gen/hal_data.o
                0x00019a64                g_transfer0_cfg
 .rodata.g_transfer0_cfg_extend
                0x00019a6c        0x1 ./ra_gen/hal_data.o
                0x00019a6c                g_transfer0_cfg_extend
 *fill*         0x00019a6d        0x3 ff
 .rodata.g_transfer1
                0x00019a70        0xc ./ra_gen/hal_data.o
                0x00019a70                g_transfer1
 .rodata.g_transfer1_cfg
                0x00019a7c        0x8 ./ra_gen/hal_data.o
                0x00019a7c                g_transfer1_cfg
 .rodata.g_transfer1_cfg_extend
                0x00019a84        0x1 ./ra_gen/hal_data.o
                0x00019a84                g_transfer1_cfg_extend
 *fill*         0x00019a85        0x3 ff
 .rodata.g_timer5_cfg
                0x00019a88       0x20 ./ra_gen/hal_data.o
                0x00019a88                g_timer5_cfg
 .rodata.g_timer5_extend
                0x00019aa8       0x30 ./ra_gen/hal_data.o
                0x00019aa8                g_timer5_extend
 .rodata.g_timer0_cfg
                0x00019ad8       0x20 ./ra_gen/hal_data.o
                0x00019ad8                g_timer0_cfg
 .rodata.g_timer0_extend
                0x00019af8        0x8 ./ra_gen/hal_data.o
                0x00019af8                g_timer0_extend
 .rodata.g_adc0_channel_cfg
                0x00019b00       0x14 ./ra_gen/hal_data.o
                0x00019b00                g_adc0_channel_cfg
 .rodata.g_adc0_cfg
                0x00019b14       0x18 ./ra_gen/hal_data.o
                0x00019b14                g_adc0_cfg
 .rodata.g_adc0_cfg_extend
                0x00019b2c        0xa ./ra_gen/hal_data.o
                0x00019b2c                g_adc0_cfg_extend
 *fill*         0x00019b36        0x2 ff
 .rodata.g_flash0_cfg
                0x00019b38       0x14 ./ra_gen/hal_data.o
                0x00019b38                g_flash0_cfg
 .rodata.g_crc0_cfg
                0x00019b4c        0xc ./ra_gen/hal_data.o
                0x00019b4c                g_crc0_cfg
 .rodata.g_bsp_pin_cfg
                0x00019b58        0x8 ./ra_gen/pin_data.o
                0x00019b58                g_bsp_pin_cfg
 .rodata.g_bsp_pin_cfg_data
                0x00019b60       0x98 ./ra_gen/pin_data.o
                0x00019b60                g_bsp_pin_cfg_data
 .rodata.g_interrupt_event_link_select
                0x00019bf8       0xc0 ./ra_gen/vector_data.o
                0x00019bf8                g_interrupt_event_link_select
 .rodata.g_div_coefficient
                0x00019cb8       0x1a ./ra/fsp/src/r_sci_uart/r_sci_uart.o
 *fill*         0x00019cd2        0x2 ff
 .rodata.g_async_baud
                0x00019cd4        0xd ./ra/fsp/src/r_sci_uart/r_sci_uart.o
 *fill*         0x00019ce1        0x3 ff
 .rodata.g_ioport_on_ioport
                0x00019ce4       0x34 ./ra/fsp/src/r_ioport/r_ioport.o
                0x00019ce4                g_ioport_on_ioport
 .rodata.g_transfer_on_dtc
                0x00019d18       0x24 ./ra/fsp/src/r_dtc/r_dtc.o
                0x00019d18                g_transfer_on_dtc
 .rodata.adc_elc_trigger_lut
                0x00019d3c        0xc ./ra/fsp/src/r_adc/r_adc.o
 .rodata.g_prcr_masks
                0x00019d48        0x8 ./ra/fsp/src/bsp/mcu/all/bsp_register_protection.o
 .rodata.__utoa.str1.1
                0x00019d50       0x25 c:/renesas/ra/e2studio_v2023-07_fsp_v4.6.0/toolchains/gcc_arm/arm-gnu-toolchain-12.2.mpacbti-rel1-mingw-w64-i686-arm-none-eabi/bin/../lib/gcc/arm-none-eabi/12.2.1/thumb/v8-m.main+fp/hard\libg_nano.a(libc_a-utoa.o)
 .rodata._ctype_
                0x00019d75      0x101 c:/renesas/ra/e2studio_v2023-07_fsp_v4.6.0/toolchains/gcc_arm/arm-gnu-toolchain-12.2.mpacbti-rel1-mingw-w64-i686-arm-none-eabi/bin/../lib/gcc/arm-none-eabi/12.2.1/thumb/v8-m.main+fp/hard\libg_nano.a(libc_a-ctype_.o)
                0x00019d75                _ctype_
                0x00019e76                        __usb_dev_descriptor_start_fs = .
 *(.usb_device_desc_fs*)
                0x00019e76                        __usb_cfg_descriptor_start_fs = .
 *(.usb_config_desc_fs*)
                0x00019e76                        __usb_interface_descriptor_start_fs = .
 *(.usb_interface_desc_fs*)
                0x00019e76                        __usb_descriptor_end_fs = .
                0x00019e76                        __usb_dev_descriptor_start_hs = .
 *(.usb_device_desc_hs*)
                0x00019e76                        __usb_cfg_descriptor_start_hs = .
 *(.usb_config_desc_hs*)
                0x00019e76                        __usb_interface_descriptor_start_hs = .
 *(.usb_interface_desc_hs*)
                0x00019e76                        __usb_descriptor_end_hs = .
 *(.eh_frame*)
 *fill*         0x00019e76        0x2 ff
 .eh_frame      0x00019e78        0x0 c:/renesas/ra/e2studio_v2023-07_fsp_v4.6.0/toolchains/gcc_arm/arm-gnu-toolchain-12.2.mpacbti-rel1-mingw-w64-i686-arm-none-eabi/bin/../lib/gcc/arm-none-eabi/12.2.1/thumb/v8-m.main+fp/hard/crtbegin.o
 .eh_frame      0x00019e78       0x28 c:/renesas/ra/e2studio_v2023-07_fsp_v4.6.0/toolchains/gcc_arm/arm-gnu-toolchain-12.2.mpacbti-rel1-mingw-w64-i686-arm-none-eabi/bin/../lib/gcc/arm-none-eabi/12.2.1/thumb/v8-m.main+fp/hard\libg_nano.a(libc_a-strlen.o)
 .eh_frame      0x00019ea0       0x38 c:/renesas/ra/e2studio_v2023-07_fsp_v4.6.0/toolchains/gcc_arm/arm-gnu-toolchain-12.2.mpacbti-rel1-mingw-w64-i686-arm-none-eabi/bin/../lib/gcc/arm-none-eabi/12.2.1/thumb/v8-m.main+fp/hard\libg_nano.a(libc_a-aeabi_memset-soft.o)
 .eh_frame      0x00019ed8        0x4 c:/renesas/ra/e2studio_v2023-07_fsp_v4.6.0/toolchains/gcc_arm/arm-gnu-toolchain-12.2.mpacbti-rel1-mingw-w64-i686-arm-none-eabi/bin/../lib/gcc/arm-none-eabi/12.2.1/thumb/v8-m.main+fp/hard/crtend.o
                0x00019edc                        __ROM_End = .
                0x000001c0                        __Vectors_Size = (__Vectors_End - __Vectors)

.glue_7         0x00019edc        0x0
 .glue_7        0x00019edc        0x0 linker stubs

.glue_7t        0x00019edc        0x0
 .glue_7t       0x00019edc        0x0 linker stubs

.vfp11_veneer   0x00019edc        0x0
 .vfp11_veneer  0x00019edc        0x0 linker stubs

.v4_bx          0x00019edc        0x0
 .v4_bx         0x00019edc        0x0 linker stubs

.iplt           0x00019edc        0x0
 .iplt          0x00019edc        0x0 c:/renesas/ra/e2studio_v2023-07_fsp_v4.6.0/toolchains/gcc_arm/arm-gnu-toolchain-12.2.mpacbti-rel1-mingw-w64-i686-arm-none-eabi/bin/../lib/gcc/arm-none-eabi/12.2.1/thumb/v8-m.main+fp/hard/crtbegin.o

.ARM.extab
 *(.ARM.extab* .gnu.linkonce.armextab.*)
                0x00019edc                        __exidx_start = .

.ARM.exidx      0x00019edc        0x8
 *(.ARM.exidx* .gnu.linkonce.armexidx.*)
 .ARM.exidx.text.__udivmoddi4
                0x00019edc        0x8 c:/renesas/ra/e2studio_v2023-07_fsp_v4.6.0/toolchains/gcc_arm/arm-gnu-toolchain-12.2.mpacbti-rel1-mingw-w64-i686-arm-none-eabi/bin/../lib/gcc/arm-none-eabi/12.2.1/thumb/v8-m.main+fp/hard\libgcc.a(_udivmoddi4.o)
 .ARM.exidx     0x00019ee4        0x0 c:/renesas/ra/e2studio_v2023-07_fsp_v4.6.0/toolchains/gcc_arm/arm-gnu-toolchain-12.2.mpacbti-rel1-mingw-w64-i686-arm-none-eabi/bin/../lib/gcc/arm-none-eabi/12.2.1/thumb/v8-m.main+fp/hard\libg_nano.a(libc_a-strlen.o)
                                  0x8 (size before relaxing)
 .ARM.exidx     0x00019ee4        0x0 c:/renesas/ra/e2studio_v2023-07_fsp_v4.6.0/toolchains/gcc_arm/arm-gnu-toolchain-12.2.mpacbti-rel1-mingw-w64-i686-arm-none-eabi/bin/../lib/gcc/arm-none-eabi/12.2.1/thumb/v8-m.main+fp/hard\libg_nano.a(libc_a-aeabi_memset-soft.o)
                                  0x8 (size before relaxing)
                0x00019ee4                        __exidx_end = .
                0x00019ee4                        __etext = .
                0x20000000                        __tz_RAM_S = ORIGIN (RAM)

.fsp_dtc_vector_table
                0x20000000      0x180
                0x20000000                        . = ORIGIN (RAM)
 *(.fsp_dtc_vector_table)
 .fsp_dtc_vector_table
                0x20000000      0x180 ./ra/fsp/src/r_dtc/r_dtc.o

.data           0x20000180      0x2d0 load address 0x00019ee4
                0x20000180                        __data_start__ = .
                0x20000180                        . = ALIGN (0x4)
                0x20000180                        __Code_In_RAM_Start = .
 *(.code_in_ram*)
                0x20000180                        __Code_In_RAM_End = .
 *(vtable)
 *(.data.*)
 .data.g_wait_count
                0x20000180        0x4 ./src/angle.o
 *fill*         0x20000184        0x4 
 .data.pidparam_cur
                0x20000188       0x48 ./src/global_variables.o
                0x20000188                pidparam_cur
 .data.pidparam_velo
                0x200001d0       0x48 ./src/global_variables.o
                0x200001d0                pidparam_velo
 .data.pidparam_ang
                0x20000218       0x48 ./src/global_variables.o
                0x20000218                pidparam_ang
 .data.interp_current_compliance_1d
                0x20000260       0x20 ./src/global_variables.o
                0x20000260                interp_current_compliance_1d
 .data.interp_angle_compliance_1d
                0x20000280       0x20 ./src/global_variables.o
                0x20000280                interp_angle_compliance_1d
 .data.interp_tad2141_1d
                0x200002a0      0x128 ./src/global_variables.o
                0x200002a0                interp_tad2141_1d
 .data.prev_moncon.1
                0x200003c8        0x1 ./src/hal_entry.o
 .data.isl28022_targetreg.22
                0x200003c9        0x1 ./src/hal_entry.o
 *fill*         0x200003ca        0x2 
 .data.PreviousID
                0x200003cc        0x4 ./src/packet.o
 .data.txcomp   0x200003d0        0x1 ./src/usart.o
 *fill*         0x200003d1        0x3 
 .data.g_uart4_baud_setting
                0x200003d4        0x4 ./ra_gen/hal_data.o
                0x200003d4                g_uart4_baud_setting
 .data.g_transfer0_info
                0x200003d8       0x10 ./ra_gen/hal_data.o
                0x200003d8                g_transfer0_info
 .data.g_transfer1_info
                0x200003e8       0x10 ./ra_gen/hal_data.o
                0x200003e8                g_transfer1_info
 .data._impure_ptr
                0x200003f8        0x4 c:/renesas/ra/e2studio_v2023-07_fsp_v4.6.0/toolchains/gcc_arm/arm-gnu-toolchain-12.2.mpacbti-rel1-mingw-w64-i686-arm-none-eabi/bin/../lib/gcc/arm-none-eabi/12.2.1/thumb/v8-m.main+fp/hard\libg_nano.a(libc_a-impure.o)
                0x200003f8                _impure_ptr
 .data._impure_data
                0x200003fc       0x4c c:/renesas/ra/e2studio_v2023-07_fsp_v4.6.0/toolchains/gcc_arm/arm-gnu-toolchain-12.2.mpacbti-rel1-mingw-w64-i686-arm-none-eabi/bin/../lib/gcc/arm-none-eabi/12.2.1/thumb/v8-m.main+fp/hard\libg_nano.a(libc_a-impure.o)
                0x200003fc                _impure_data
 *(.data)
                0x20000448                        . = ALIGN (0x4)
                0x20000448                        PROVIDE (__preinit_array_start = .)
 *(.preinit_array)
                0x20000448                        PROVIDE (__preinit_array_end = .)
                0x20000448                        . = ALIGN (0x4)
                0x20000448                        PROVIDE (__init_array_start = .)
 *(SORT_BY_NAME(.init_array.*))
 *(.init_array)
 .init_array    0x20000448        0x4 c:/renesas/ra/e2studio_v2023-07_fsp_v4.6.0/toolchains/gcc_arm/arm-gnu-toolchain-12.2.mpacbti-rel1-mingw-w64-i686-arm-none-eabi/bin/../lib/gcc/arm-none-eabi/12.2.1/thumb/v8-m.main+fp/hard/crtbegin.o
                0x2000044c                        PROVIDE (__init_array_end = .)
                0x2000044c                        . = ALIGN (0x4)
                [!provide]                        PROVIDE (__fini_array_start = .)
 *(SORT_BY_NAME(.fini_array.*))
 *(.fini_array)
 .fini_array    0x2000044c        0x4 c:/renesas/ra/e2studio_v2023-07_fsp_v4.6.0/toolchains/gcc_arm/arm-gnu-toolchain-12.2.mpacbti-rel1-mingw-w64-i686-arm-none-eabi/bin/../lib/gcc/arm-none-eabi/12.2.1/thumb/v8-m.main+fp/hard/crtbegin.o
                [!provide]                        PROVIDE (__fini_array_end = .)
 *(.jcr*)
                0x20000450                        . = ALIGN (0x4)
                0x20000450                        __data_end__ = .

.tm_clone_table
                0x20000450        0x0 load address 0x0001a1b4
 .tm_clone_table
                0x20000450        0x0 c:/renesas/ra/e2studio_v2023-07_fsp_v4.6.0/toolchains/gcc_arm/arm-gnu-toolchain-12.2.mpacbti-rel1-mingw-w64-i686-arm-none-eabi/bin/../lib/gcc/arm-none-eabi/12.2.1/thumb/v8-m.main+fp/hard/crtbegin.o
 .tm_clone_table
                0x20000450        0x0 c:/renesas/ra/e2studio_v2023-07_fsp_v4.6.0/toolchains/gcc_arm/arm-gnu-toolchain-12.2.mpacbti-rel1-mingw-w64-i686-arm-none-eabi/bin/../lib/gcc/arm-none-eabi/12.2.1/thumb/v8-m.main+fp/hard/crtend.o

.igot.plt       0x20000450        0x0 load address 0x0001a1b4
 .igot.plt      0x20000450        0x0 c:/renesas/ra/e2studio_v2023-07_fsp_v4.6.0/toolchains/gcc_arm/arm-gnu-toolchain-12.2.mpacbti-rel1-mingw-w64-i686-arm-none-eabi/bin/../lib/gcc/arm-none-eabi/12.2.1/thumb/v8-m.main+fp/hard/crtbegin.o

.gnu.sgstubs    0x0001a400        0x0
                0x0001a400                        . = (DEFINED (PROJECT_SECURE) && DEFINED (FLASH_NSC_START))?ABSOLUTE (FLASH_NSC_START):ALIGN (0x400)
                0x0001a400                        __tz_FLASH_C = DEFINED (FLASH_NSC_START)?ABSOLUTE (FLASH_NSC_START):__RESERVE_NS_RAM?ABSOLUTE ((FLASH_START + FLASH_LENGTH)):ALIGN (0x400)
                0x0001a400                        _start_sg = .
 *(.gnu.sgstubs*)
                0x0001a400                        . = ALIGN (0x20)
                0x0001a400                        _end_sg = .
                0x00020000                        __tz_FLASH_N = DEFINED (FLASH_NS_START)?ABSOLUTE (FLASH_NS_START):__RESERVE_NS_RAM?ABSOLUTE ((FLASH_START + FLASH_LENGTH)):(FLASH_LENGTH < 0x8000)?FLASH_LENGTH:ALIGN (0x8000)
                0x00020000                        FLASH_NS_IMAGE_START = DEFINED (FLASH_NS_IMAGE_START)?FLASH_NS_IMAGE_START:__tz_FLASH_N
                0x60000000                        __tz_QSPI_FLASH_S = ORIGIN (QSPI_FLASH)

.qspi_flash     0x60000000        0x0
                0x60000000                        __qspi_flash_start__ = .
 *(.qspi_flash*)
 *(.code_in_qspi*)
                0x60000000                        __qspi_flash_end__ = .
                0x00000000                        __qspi_flash_code_size__ = (__qspi_flash_end__ - __qspi_flash_start__)
                0x0001a1b4                        __qspi_flash_code_addr__ = (__etext + (__data_end__ - __data_start__))

.qspi_non_retentive
                0x60000000        0x0 load address 0x0001a1b4
                0x60000000                        __qspi_non_retentive_start__ = .
 *(.qspi_non_retentive*)
                0x60000000                        __qspi_non_retentive_end__ = .
                0x00000000                        __qspi_non_retentive_size__ = (__qspi_non_retentive_end__ - __qspi_non_retentive_start__)
                0x04000000                        __qspi_region_max_size__ = 0x4000000
                0x60000000                        __qspi_region_start_address__ = __qspi_flash_start__
                0x64000000                        __qspi_region_end_address__ = (__qspi_flash_start__ + __qspi_region_max_size__)
                0x60000000                        __tz_QSPI_FLASH_N = __qspi_non_retentive_end__

.OSPI_DEVICE_0_NO_LOAD
                0x80020000        0x0
                0x80020000                        . = ALIGN (0x4)
                0x80020000                        __ospi_device_0_start__ = .
 *(.ospi_device_0_no_load*)
                0x80020000                        . = ALIGN (0x4)
                0x80020000                        __ospi_device_0_end__ = .

.OSPI_DEVICE_1_NO_LOAD
                0x80030000        0x0
                0x80030000                        . = ALIGN (0x4)
                0x80030000                        __ospi_device_1_start__ = .
 *(.ospi_device_1_no_load*)
                0x80030000                        . = ALIGN (0x4)
                0x80030000                        __ospi_device_1_end__ = .
                0x80020000                        __tz_OSPI_DEVICE_0_S = ORIGIN (OSPI_DEVICE_0)

.OSPI_DEVICE_0  0x80020000        0x0
                0x80020000                        __ospi_device_0_start__ = .
 *(.ospi_device_0*)
 *(.code_in_ospi_device_0*)
                0x80020000                        __ospi_device_0_end__ = .
                0x00000000                        __ospi_device_0_code_size__ = (__ospi_device_0_end__ - __ospi_device_0_start__)
                0x0001a1b4                        __ospi_device_0_code_addr__ = (__etext + (__data_end__ - __data_start__))

.ospi_device_0_non_retentive
                0x80020000        0x0 load address 0x0001a1b4
                0x80020000                        __ospi_device_0_non_retentive_start__ = .
 *(.ospi_device_0_non_retentive*)
                0x80020000                        __ospi_device_0_non_retentive_end__ = .
                0x00000000                        __ospi_device_0_non_retentive_size__ = (__ospi_device_0_non_retentive_end__ - __ospi_device_0_non_retentive_start__)
                0x08000000                        __ospi_device_0_region_max_size__ = 0x8000000
                0x80020000                        __ospi_device_0_region_start_address__ = __ospi_device_0_start__
                0x88020000                        __ospi_device_0_region_end_address__ = (__ospi_device_0_start__ + __ospi_device_0_region_max_size__)
                0x80020000                        __tz_OSPI_DEVICE_0_N = __ospi_device_0_non_retentive_end__
                0x80030000                        __tz_OSPI_DEVICE_1_S = ORIGIN (OSPI_DEVICE_1)

.OSPI_DEVICE_1  0x80030000        0x0
                0x80030000                        __ospi_device_1_start__ = .
 *(.ospi_device_1*)
 *(.code_in_ospi_device_1*)
                0x80030000                        __ospi_device_1_end__ = .
                0x00000000                        __ospi_device_1_code_size__ = (__ospi_device_1_end__ - __ospi_device_1_start__)
                0x0001a1b4                        __ospi_device_1_code_addr__ = (__etext + (__data_end__ - __data_start__))

.ospi_device_1_non_retentive
                0x80030000        0x0 load address 0x0001a1b4
                0x80030000                        __ospi_device_1_non_retentive_start__ = .
 *(.ospi_device_1_non_retentive*)
                0x80030000                        __ospi_device_1_non_retentive_end__ = .
                0x00000000                        __ospi_device_1_non_retentive_size__ = (__ospi_device_1_non_retentive_end__ - __ospi_device_1_non_retentive_start__)
                0x10000000                        __ospi_device_1_region_max_size__ = 0x10000000
                0x80030000                        __ospi_device_1_region_start_address__ = __ospi_device_1_start__
                0x90030000                        __ospi_device_1_region_end_address__ = (__ospi_device_1_start__ + __ospi_device_1_region_max_size__)
                0x80030000                        __tz_OSPI_DEVICE_1_N = __ospi_device_1_non_retentive_end__

.noinit         0x20000450       0x20
                0x20000450                        . = ALIGN (0x4)
                0x20000450                        __noinit_start = .
 *(.noinit*)
 .noinit        0x20000450       0x1c ./ra/fsp/src/bsp/mcu/all/bsp_clocks.o
                0x20000470                        . = ALIGN (0x8)
 *fill*         0x2000046c        0x4 
 *(.heap.*)
                0x20000470                        __noinit_end = .

.bss            0x20000470     0x3b2c
                0x20000470                        . = ALIGN (0x4)
                0x20000470                        __bss_start__ = .
 *(.bss*)
 .bss.completed.1
                0x20000470        0x1 c:/renesas/ra/e2studio_v2023-07_fsp_v4.6.0/toolchains/gcc_arm/arm-gnu-toolchain-12.2.mpacbti-rel1-mingw-w64-i686-arm-none-eabi/bin/../lib/gcc/arm-none-eabi/12.2.1/thumb/v8-m.main+fp/hard/crtbegin.o
 *fill*         0x20000471        0x3 
 .bss.object.0  0x20000474       0x18 c:/renesas/ra/e2studio_v2023-07_fsp_v4.6.0/toolchains/gcc_arm/arm-gnu-toolchain-12.2.mpacbti-rel1-mingw-w64-i686-arm-none-eabi/bin/../lib/gcc/arm-none-eabi/12.2.1/thumb/v8-m.main+fp/hard/crtbegin.o
 *fill*         0x2000048c        0x4 
 .bss.adc_value
                0x20000490       0x18 ./src/adc_temp.o
 .bss.spi_master_event
                0x200004a8        0x1 ./src/angle.o
 *fill*         0x200004a9        0x3 
 .bss.ControlTable
                0x200004ac      0x188 ./src/control_table.o
                0x200004ac                ControlTable
 .bss.UpdateTargetValue
                0x20000634        0x1 ./src/global_variables.o
                0x20000634                UpdateTargetValue
 *fill*         0x20000635        0x3 
 .bss.packet.0  0x20000638      0x7d0 ./src/hal_entry.o
 .bss.MonCount.3
                0x20000e08        0x2 ./src/hal_entry.o
 *fill*         0x20000e0a        0x2 
 .bss.StartCurrent.4
                0x20000e0c        0x4 ./src/hal_entry.o
 .bss.prev_targetcurrent.5
                0x20000e10        0x4 ./src/hal_entry.o
 .bss.StartVelocity.6
                0x20000e14        0x4 ./src/hal_entry.o
 .bss.prev_targetvelocity.7
                0x20000e18        0x4 ./src/hal_entry.o
 .bss.LimitedTargetAngle.8
                0x20000e1c        0x4 ./src/hal_entry.o
 .bss.StartAngle.9
                0x20000e20        0x4 ./src/hal_entry.o
 .bss.TransitionTime.10
                0x20000e24        0x4 ./src/hal_entry.o
 .bss.prev_set_transition_mode.11
                0x20000e28        0x1 ./src/hal_entry.o
 *fill*         0x20000e29        0x3 
 .bss.prev_set_transition_time.12
                0x20000e2c        0x4 ./src/hal_entry.o
 .bss.prev_targetangle.13
                0x20000e30        0x4 ./src/hal_entry.o
 .bss.TargetCurrent.14
                0x20000e34        0x4 ./src/hal_entry.o
 .bss.TargetVelocity.15
                0x20000e38        0x4 ./src/hal_entry.o
 .bss.TargetAngle.16
                0x20000e3c        0x4 ./src/hal_entry.o
 .bss.stall.17  0x20000e40        0x1 ./src/hal_entry.o
 .bss.prevmode.18
                0x20000e41        0x1 ./src/hal_entry.o
 *fill*         0x20000e42        0x6 
 .bss.current.19
                0x20000e48        0x8 ./src/hal_entry.o
 .bss.stat_cur.20
                0x20000e50        0x8 ./src/hal_entry.o
 .bss.isl28022_read_data.21
                0x20000e58        0x2 ./src/hal_entry.o
 .bss.angle_depth.23
                0x20000e5a        0x1 ./src/hal_entry.o
 .bss.led_stat  0x20000e5b        0x1 ./src/hal_entry.o
 .bss.ang_history
                0x20000e5c       0x80 ./src/hal_entry.o
 .bss.ang_ex    0x20000edc        0x4 ./src/hal_entry.o
 .bss.now_ang   0x20000ee0        0x4 ./src/hal_entry.o
 .bss.prev_ang  0x20000ee4        0x4 ./src/hal_entry.o
 .bss.rxb       0x20000ee8      0xfa0 ./src/hal_entry.o
 .bss.txb       0x20001e88      0xfa0 ./src/hal_entry.o
 .bss.cmd_r.0   0x20002e28      0x3e8 ./src/packet.o
 .bss.MakeAck   0x20003210        0x1 ./src/packet.o
 .bss.AckSend   0x20003211        0x1 ./src/packet.o
 *fill*         0x20003212        0x2 
 .bss.Ack       0x20003214      0x7d0 ./src/packet.o
 .bss.MachedID  0x200039e4        0x1 ./src/packet.o
 *fill*         0x200039e5        0x3 
 .bss.FlagOfIDs
                0x200039e8      0x100 ./src/packet.o
 .bss.packet_req_init_id_baud
                0x20003ae8        0x1 ./src/packet.o
                0x20003ae8                packet_req_init_id_baud
 .bss.packet_req_initalize
                0x20003ae9        0x1 ./src/packet.o
                0x20003ae9                packet_req_initalize
 *fill*         0x20003aea        0x2 
 .bss.rreg.1    0x20003aec        0x4 ./src/power_monitor.o
 .bss.dat.0     0x20003af0        0x3 ./src/power_monitor.o
 .bss.i2c_stat  0x20003af3        0x1 ./src/power_monitor.o
 .bss.iic_pstat
                0x20003af4        0x1 ./src/power_monitor.o
 *fill*         0x20003af5        0x3 
 .bss.isl28022_destreaddata
                0x20003af8        0x4 ./src/power_monitor.o
 .bss.FIFO      0x20003afc       0x18 ./src/usart.o
 .bss.g_ioport_ctrl
                0x20003b14        0x8 ./ra_gen/common_data.o
                0x20003b14                g_ioport_ctrl
 .bss.g_uart4_ctrl
                0x20003b1c       0x30 ./ra_gen/hal_data.o
                0x20003b1c                g_uart4_ctrl
 .bss.g_i2c3_ctrl
                0x20003b4c       0x40 ./ra_gen/hal_data.o
                0x20003b4c                g_i2c3_ctrl
 .bss.g_spi2_ctrl
                0x20003b8c       0x2c ./ra_gen/hal_data.o
                0x20003b8c                g_spi2_ctrl
 .bss.g_transfer0_ctrl
                0x20003bb8        0x8 ./ra_gen/hal_data.o
                0x20003bb8                g_transfer0_ctrl
 .bss.g_transfer1_ctrl
                0x20003bc0        0x8 ./ra_gen/hal_data.o
                0x20003bc0                g_transfer1_ctrl
 .bss.g_timer5_ctrl
                0x20003bc8       0x20 ./ra_gen/hal_data.o
                0x20003bc8                g_timer5_ctrl
 .bss.g_timer0_ctrl
                0x20003be8       0x20 ./ra_gen/hal_data.o
                0x20003be8                g_timer0_ctrl
 .bss.g_adc0_ctrl
                0x20003c08       0x24 ./ra_gen/hal_data.o
                0x20003c08                g_adc0_ctrl
 .bss.g_flash0_ctrl
                0x20003c2c       0x44 ./ra_gen/hal_data.o
                0x20003c2c                g_flash0_ctrl
 .bss.g_crc0_ctrl
                0x20003c70        0x8 ./ra_gen/hal_data.o
                0x20003c70                g_crc0_ctrl
 .bss.tx_dummy.0
                0x20003c78        0x1 ./ra/fsp/src/r_sci_spi/r_sci_spi.o
 .bss.g_dtc_state_initialized.0
                0x20003c79        0x1 ./ra/fsp/src/r_dtc/r_dtc.o
 *fill*         0x20003c7a        0x2 
 .bss.gp_prv_agt_periods
                0x20003c7c       0x18 ./ra/fsp/src/r_agt/r_agt.o
 .bss.g_bsp_group_irq_sources
                0x20003c94       0x40 ./ra/fsp/src/bsp/mcu/all/bsp_group_irq.o
                0x20003c94                g_bsp_group_irq_sources
 .bss.g_protect_pfswe_counter
                0x20003cd4        0x4 ./ra/fsp/src/bsp/mcu/all/bsp_io.o
                0x20003cd4                g_protect_pfswe_counter
 .bss.gp_renesas_isr_context
                0x20003cd8      0x180 ./ra/fsp/src/bsp/mcu/all/bsp_irq.o
                0x20003cd8                gp_renesas_isr_context
 .bss.g_protect_counters
                0x20003e58        0x8 ./ra/fsp/src/bsp/mcu/all/bsp_register_protection.o
                0x20003e58                g_protect_counters
 .bss.SystemCoreClock
                0x20003e60        0x4 ./ra/fsp/src/bsp/cmsis/Device/RENESAS/Source/system.o
                0x20003e60                SystemCoreClock
 .bss.__sf      0x20003e64      0x138 c:/renesas/ra/e2studio_v2023-07_fsp_v4.6.0/toolchains/gcc_arm/arm-gnu-toolchain-12.2.mpacbti-rel1-mingw-w64-i686-arm-none-eabi/bin/../lib/gcc/arm-none-eabi/12.2.1/thumb/v8-m.main+fp/hard\libg_nano.a(libc_a-findfp.o)
                0x20003e64                __sf
 *(COMMON)
                0x20003f9c                        . = ALIGN (0x4)
                0x20003f9c                        __bss_end__ = .

.heap           0x20003f9c        0x4
                0x20003fa0                        . = ALIGN (0x8)
 *fill*         0x20003f9c        0x4 
                0x20003fa0                        __HeapBase = .
 *(.heap)
                0x20003fa0                        __HeapLimit = .

.stack_dummy    0x20003fa0     0x1000
                0x20003fa0                        . = ALIGN (0x8)
                0x20003fa0                        __StackLimit = .
 *(.stack)
 .stack         0x20003fa0     0x1000 ./ra/fsp/src/bsp/cmsis/Device/RENESAS/Source/startup.o
                0x20004fa0                        __StackTop = .
 *(.stack*)
                0x20004fa0                        __StackTopAll = .
                0x20004fa0                        PROVIDE (__stack = __StackTopAll)
                0x20004fa0                        __RAM_segment_used_end__ = ALIGN (__StackTopAll, 0x4)
                0x20005000                        __tz_RAM_C = DEFINED (RAM_NSC_START)?ABSOLUTE (RAM_NSC_START):__RESERVE_NS_RAM?ABSOLUTE (RAM_NS_BUFFER_BLOCK_START):ALIGN (__RAM_segment_used_end__, 0x400)
                0x20006000                        __tz_RAM_N = DEFINED (RAM_NS_START)?ABSOLUTE (RAM_NS_START):__RESERVE_NS_RAM?ABSOLUTE (RAM_NS_BUFFER_BLOCK_START):ALIGN (__tz_RAM_C, 0x2000)

.ns_buffer      0x20004fa0        0x0
                0x20004fa0                        . = __RESERVE_NS_RAM?ABSOLUTE ((RAM_NS_BUFFER_START & 0xffffffe0)):.
 *(.ns_buffer*)

.data_flash     0x08000000        0x0
                0x08000000                        . = ORIGIN (DATA_FLASH)
                0x08000000                        __tz_DATA_FLASH_S = .
                0x08000000                        __Data_Flash_Start = .
 *(.data_flash*)
                0x08000000                        __Data_Flash_End = .
                0x08000000                        __tz_DATA_FLASH_N = DEFINED (DATA_FLASH_NS_START)?ABSOLUTE (DATA_FLASH_NS_START):__RESERVE_NS_RAM?ABSOLUTE ((DATA_FLASH_START + DATA_FLASH_LENGTH)):ALIGN (0x400)
                0x80010000                        __tz_SDRAM_S = ORIGIN (SDRAM)

.sdram          0x80010000        0x0
                0x80010000                        __SDRAM_Start = .
 *(.sdram*)
 *(.frame*)
                0x80010000                        __SDRAM_End = .
                0x80010000                        __tz_SDRAM_N = __SDRAM_End
                0x00000000                        __tz_ID_CODE_S = ORIGIN (ID_CODE)

.id_code        0x00000000        0x0
                0x00000000                        __ID_Code_Start = .
 *(.id_code*)
                0x00000000                        __ID_Code_End = .
                0x00000000                        __tz_ID_CODE_N = __ID_Code_End
                0x0100a100                        __tz_OPTION_SETTING_S = ORIGIN (OPTION_SETTING)

.option_setting
                0x0100a100       0x38
                0x0100a100                        __OPTION_SETTING_Start = .
 *(.option_setting_ofs0)
 .option_setting_ofs0
                0x0100a100        0x4 ./ra/fsp/src/bsp/mcu/all/bsp_rom_registers.o
                0x0100a110                        . = PROJECT_SECURE_OR_FLAT?(__OPTION_SETTING_Start + 0x10):__OPTION_SETTING_Start
 *fill*         0x0100a104        0xc ff
 *(.option_setting_dualsel)
                0x0100a134                        . = PROJECT_SECURE_OR_FLAT?(__OPTION_SETTING_Start + 0x34):__OPTION_SETTING_Start
 *fill*         0x0100a110       0x24 ff
 *(.option_setting_sas)
 .option_setting_sas
                0x0100a134        0x4 ./ra/fsp/src/bsp/mcu/all/bsp_rom_registers.o
                0x0100a138                        __OPTION_SETTING_End = .
                0x0100a180                        __tz_OPTION_SETTING_N = OPTION_SETTING_START_NS

.option_setting_ns
                0x0100a138        0x0
                0x0100a138                        __OPTION_SETTING_NS_Start = .
 *(.option_setting_ofs1)
                0x0100a138                        . = USE_OPTION_SETTING_NS?(__OPTION_SETTING_NS_Start + 0x10):__OPTION_SETTING_NS_Start
 *(.option_setting_banksel)
                0x0100a138                        . = USE_OPTION_SETTING_NS?(__OPTION_SETTING_NS_Start + 0x40):__OPTION_SETTING_NS_Start
 *(.option_setting_bps0)
                0x0100a138                        . = USE_OPTION_SETTING_NS?(__OPTION_SETTING_NS_Start + 0x44):__OPTION_SETTING_NS_Start
 *(.option_setting_bps1)
                0x0100a138                        . = USE_OPTION_SETTING_NS?(__OPTION_SETTING_NS_Start + 0x48):__OPTION_SETTING_NS_Start
 *(.option_setting_bps2)
                0x0100a138                        . = USE_OPTION_SETTING_NS?(__OPTION_SETTING_NS_Start + 0x60):__OPTION_SETTING_NS_Start
 *(.option_setting_pbps0)
                0x0100a138                        . = USE_OPTION_SETTING_NS?(__OPTION_SETTING_NS_Start + 0x64):__OPTION_SETTING_NS_Start
 *(.option_setting_pbps1)
                0x0100a138                        . = USE_OPTION_SETTING_NS?(__OPTION_SETTING_NS_Start + 0x68):__OPTION_SETTING_NS_Start
 *(.option_setting_pbps2)
                0x0100a138                        __OPTION_SETTING_NS_End = .
                0x0100a200                        __tz_OPTION_SETTING_S_S = ORIGIN (OPTION_SETTING_S)

.option_setting_s
                0x0100a200       0xcc
                0x0100a200                        __OPTION_SETTING_S_Start = .
 *(.option_setting_ofs1_sec)
 .option_setting_ofs1_sec
                0x0100a200        0x4 ./ra/fsp/src/bsp/mcu/all/bsp_rom_registers.o
                0x0100a210                        . = PROJECT_SECURE_OR_FLAT?(__OPTION_SETTING_S_Start + 0x10):__OPTION_SETTING_S_Start
 *fill*         0x0100a204        0xc ff
 *(.option_setting_banksel_sec)
 .option_setting_banksel_sec
                0x0100a210        0x4 ./ra/fsp/src/bsp/mcu/all/bsp_rom_registers.o
                0x0100a240                        . = PROJECT_SECURE_OR_FLAT?(__OPTION_SETTING_S_Start + 0x40):__OPTION_SETTING_S_Start
 *fill*         0x0100a214       0x2c ff
 *(.option_setting_bps_sec0)
 .option_setting_bps_sec0
                0x0100a240        0x4 ./ra/fsp/src/bsp/mcu/all/bsp_rom_registers.o
                0x0100a244                        . = PROJECT_SECURE_OR_FLAT?(__OPTION_SETTING_S_Start + 0x44):__OPTION_SETTING_S_Start
 *(.option_setting_bps_sec1)
 .option_setting_bps_sec1
                0x0100a244        0x4 ./ra/fsp/src/bsp/mcu/all/bsp_rom_registers.o
                0x0100a248                        . = PROJECT_SECURE_OR_FLAT?(__OPTION_SETTING_S_Start + 0x48):__OPTION_SETTING_S_Start
 *(.option_setting_bps_sec2)
 .option_setting_bps_sec2
                0x0100a248        0x4 ./ra/fsp/src/bsp/mcu/all/bsp_rom_registers.o
                0x0100a260                        . = PROJECT_SECURE_OR_FLAT?(__OPTION_SETTING_S_Start + 0x60):__OPTION_SETTING_S_Start
 *fill*         0x0100a24c       0x14 ff
 *(.option_setting_pbps_sec0)
 .option_setting_pbps_sec0
                0x0100a260        0x4 ./ra/fsp/src/bsp/mcu/all/bsp_rom_registers.o
                0x0100a264                        . = PROJECT_SECURE_OR_FLAT?(__OPTION_SETTING_S_Start + 0x64):__OPTION_SETTING_S_Start
 *(.option_setting_pbps_sec1)
 .option_setting_pbps_sec1
                0x0100a264        0x4 ./ra/fsp/src/bsp/mcu/all/bsp_rom_registers.o
                0x0100a268                        . = PROJECT_SECURE_OR_FLAT?(__OPTION_SETTING_S_Start + 0x68):__OPTION_SETTING_S_Start
 *(.option_setting_pbps_sec2)
 .option_setting_pbps_sec2
                0x0100a268        0x4 ./ra/fsp/src/bsp/mcu/all/bsp_rom_registers.o
                0x0100a280                        . = PROJECT_SECURE_OR_FLAT?(__OPTION_SETTING_S_Start + 0x80):__OPTION_SETTING_S_Start
 *fill*         0x0100a26c       0x14 ff
 *(.option_setting_ofs1_sel)
 .option_setting_ofs1_sel
                0x0100a280        0x4 ./ra/fsp/src/bsp/mcu/all/bsp_rom_registers.o
                0x0100a290                        . = PROJECT_SECURE_OR_FLAT?(__OPTION_SETTING_S_Start + 0x90):__OPTION_SETTING_S_Start
 *fill*         0x0100a284        0xc ff
 *(.option_setting_banksel_sel)
                0x0100a2c0                        . = PROJECT_SECURE_OR_FLAT?(__OPTION_SETTING_S_Start + 0xc0):__OPTION_SETTING_S_Start
 *fill*         0x0100a290       0x30 ff
 *(.option_setting_bps_sel0)
 .option_setting_bps_sel0
                0x0100a2c0        0x4 ./ra/fsp/src/bsp/mcu/all/bsp_rom_registers.o
                0x0100a2c4                        . = PROJECT_SECURE_OR_FLAT?(__OPTION_SETTING_S_Start + 0xc4):__OPTION_SETTING_S_Start
 *(.option_setting_bps_sel1)
 .option_setting_bps_sel1
                0x0100a2c4        0x4 ./ra/fsp/src/bsp/mcu/all/bsp_rom_registers.o
                0x0100a2c8                        . = PROJECT_SECURE_OR_FLAT?(__OPTION_SETTING_S_Start + 0xc8):__OPTION_SETTING_S_Start
 *(.option_setting_bps_sel2)
 .option_setting_bps_sel2
                0x0100a2c8        0x4 ./ra/fsp/src/bsp/mcu/all/bsp_rom_registers.o
                0x0100a2cc                        __OPTION_SETTING_S_End = .
                0x0100a2cc                        __tz_OPTION_SETTING_S_N = __OPTION_SETTING_S_End
OUTPUT(JP200.elf elf32-littlearm)
LOAD linker stubs

.rel.dyn        0x0100a2cc        0x0
 .rel.iplt      0x0100a2cc        0x0 c:/renesas/ra/e2studio_v2023-07_fsp_v4.6.0/toolchains/gcc_arm/arm-gnu-toolchain-12.2.mpacbti-rel1-mingw-w64-i686-arm-none-eabi/bin/../lib/gcc/arm-none-eabi/12.2.1/thumb/v8-m.main+fp/hard/crtbegin.o

.ARM.attributes
                0x00000000       0x36
 .ARM.attributes
                0x00000000       0x26 c:/renesas/ra/e2studio_v2023-07_fsp_v4.6.0/toolchains/gcc_arm/arm-gnu-toolchain-12.2.mpacbti-rel1-mingw-w64-i686-arm-none-eabi/bin/../lib/gcc/arm-none-eabi/12.2.1/thumb/v8-m.main+fp/hard/crti.o
 .ARM.attributes
                0x00000026       0x38 c:/renesas/ra/e2studio_v2023-07_fsp_v4.6.0/toolchains/gcc_arm/arm-gnu-toolchain-12.2.mpacbti-rel1-mingw-w64-i686-arm-none-eabi/bin/../lib/gcc/arm-none-eabi/12.2.1/thumb/v8-m.main+fp/hard/crtbegin.o
 .ARM.attributes
                0x0000005e       0x3a ./src/adc_temp.o
 .ARM.attributes
                0x00000098       0x3a ./src/angle.o
 .ARM.attributes
                0x000000d2       0x3a ./src/control_table.o
 .ARM.attributes
                0x0000010c       0x3a ./src/global_variables.o
 .ARM.attributes
                0x00000146       0x3a ./src/hal_entry.o
 .ARM.attributes
                0x00000180       0x3a ./src/interpolation.o
 .ARM.attributes
                0x000001ba       0x3a ./src/monitor.o
 .ARM.attributes
                0x000001f4       0x3a ./src/packet.o
 .ARM.attributes
                0x0000022e       0x3a ./src/pid.o
 .ARM.attributes
                0x00000268       0x3a ./src/power_monitor.o
 .ARM.attributes
                0x000002a2       0x3a ./src/sintable.o
 .ARM.attributes
                0x000002dc       0x3a ./src/usart.o
 .ARM.attributes
                0x00000316       0x3a ./ra_gen/common_data.o
 .ARM.attributes
                0x00000350       0x3a ./ra_gen/hal_data.o
 .ARM.attributes
                0x0000038a       0x3a ./ra_gen/main.o
 .ARM.attributes
                0x000003c4       0x3a ./ra_gen/pin_data.o
 .ARM.attributes
                0x000003fe       0x3a ./ra_gen/vector_data.o
 .ARM.attributes
                0x00000438       0x3a ./ra/fsp/src/r_sci_uart/r_sci_uart.o
 .ARM.attributes
                0x00000472       0x3a ./ra/fsp/src/r_sci_spi/r_sci_spi.o
 .ARM.attributes
                0x000004ac       0x3a ./ra/fsp/src/r_sci_i2c/r_sci_i2c.o
 .ARM.attributes
                0x000004e6       0x3a ./ra/fsp/src/r_rtc/r_rtc.o
 .ARM.attributes
                0x00000520       0x3a ./ra/fsp/src/r_ioport/r_ioport.o
 .ARM.attributes
                0x0000055a       0x3a ./ra/fsp/src/r_gpt/r_gpt.o
 .ARM.attributes
                0x00000594       0x3a ./ra/fsp/src/r_flash_hp/r_flash_hp.o
 .ARM.attributes
                0x000005ce       0x3a ./ra/fsp/src/r_dtc/r_dtc.o
 .ARM.attributes
                0x00000608       0x3a ./ra/fsp/src/r_crc/r_crc.o
 .ARM.attributes
                0x00000642       0x3a ./ra/fsp/src/r_agt/r_agt.o
 .ARM.attributes
                0x0000067c       0x3a ./ra/fsp/src/r_adc/r_adc.o
 .ARM.attributes
                0x000006b6       0x3a ./ra/fsp/src/bsp/mcu/all/bsp_clocks.o
 .ARM.attributes
                0x000006f0       0x3a ./ra/fsp/src/bsp/mcu/all/bsp_common.o
 .ARM.attributes
                0x0000072a       0x3a ./ra/fsp/src/bsp/mcu/all/bsp_delay.o
 .ARM.attributes
                0x00000764       0x3a ./ra/fsp/src/bsp/mcu/all/bsp_group_irq.o
 .ARM.attributes
                0x0000079e       0x3a ./ra/fsp/src/bsp/mcu/all/bsp_io.o
 .ARM.attributes
                0x000007d8       0x3a ./ra/fsp/src/bsp/mcu/all/bsp_irq.o
 .ARM.attributes
                0x00000812       0x3a ./ra/fsp/src/bsp/mcu/all/bsp_register_protection.o
 .ARM.attributes
                0x0000084c       0x3a ./ra/fsp/src/bsp/mcu/all/bsp_rom_registers.o
 .ARM.attributes
                0x00000886       0x3a ./ra/fsp/src/bsp/cmsis/Device/RENESAS/Source/startup.o
 .ARM.attributes
                0x000008c0       0x3a ./ra/fsp/src/bsp/cmsis/Device/RENESAS/Source/system.o
 .ARM.attributes
                0x000008fa       0x26 c:/renesas/ra/e2studio_v2023-07_fsp_v4.6.0/toolchains/gcc_arm/arm-gnu-toolchain-12.2.mpacbti-rel1-mingw-w64-i686-arm-none-eabi/bin/../lib/gcc/arm-none-eabi/12.2.1/thumb/v8-m.main+fp/hard\libgcc.a(_arm_addsubdf3.o)
 .ARM.attributes
                0x00000920       0x26 c:/renesas/ra/e2studio_v2023-07_fsp_v4.6.0/toolchains/gcc_arm/arm-gnu-toolchain-12.2.mpacbti-rel1-mingw-w64-i686-arm-none-eabi/bin/../lib/gcc/arm-none-eabi/12.2.1/thumb/v8-m.main+fp/hard\libgcc.a(_arm_muldivdf3.o)
 .ARM.attributes
                0x00000946       0x26 c:/renesas/ra/e2studio_v2023-07_fsp_v4.6.0/toolchains/gcc_arm/arm-gnu-toolchain-12.2.mpacbti-rel1-mingw-w64-i686-arm-none-eabi/bin/../lib/gcc/arm-none-eabi/12.2.1/thumb/v8-m.main+fp/hard\libgcc.a(_arm_cmpdf2.o)
 .ARM.attributes
                0x0000096c       0x26 c:/renesas/ra/e2studio_v2023-07_fsp_v4.6.0/toolchains/gcc_arm/arm-gnu-toolchain-12.2.mpacbti-rel1-mingw-w64-i686-arm-none-eabi/bin/../lib/gcc/arm-none-eabi/12.2.1/thumb/v8-m.main+fp/hard\libgcc.a(_arm_fixdfsi.o)
 .ARM.attributes
                0x00000992       0x26 c:/renesas/ra/e2studio_v2023-07_fsp_v4.6.0/toolchains/gcc_arm/arm-gnu-toolchain-12.2.mpacbti-rel1-mingw-w64-i686-arm-none-eabi/bin/../lib/gcc/arm-none-eabi/12.2.1/thumb/v8-m.main+fp/hard\libgcc.a(_arm_fixunsdfsi.o)
 .ARM.attributes
                0x000009b8       0x26 c:/renesas/ra/e2studio_v2023-07_fsp_v4.6.0/toolchains/gcc_arm/arm-gnu-toolchain-12.2.mpacbti-rel1-mingw-w64-i686-arm-none-eabi/bin/../lib/gcc/arm-none-eabi/12.2.1/thumb/v8-m.main+fp/hard\libgcc.a(_aeabi_ldivmod.o)
 .ARM.attributes
                0x000009de       0x38 c:/renesas/ra/e2studio_v2023-07_fsp_v4.6.0/toolchains/gcc_arm/arm-gnu-toolchain-12.2.mpacbti-rel1-mingw-w64-i686-arm-none-eabi/bin/../lib/gcc/arm-none-eabi/12.2.1/thumb/v8-m.main+fp/hard\libgcc.a(_udivmoddi4.o)
 .ARM.attributes
                0x00000a16       0x26 c:/renesas/ra/e2studio_v2023-07_fsp_v4.6.0/toolchains/gcc_arm/arm-gnu-toolchain-12.2.mpacbti-rel1-mingw-w64-i686-arm-none-eabi/bin/../lib/gcc/arm-none-eabi/12.2.1/thumb/v8-m.main+fp/hard\libgcc.a(_dvmd_tls.o)
 .ARM.attributes
                0x00000a3c       0x38 c:/renesas/ra/e2studio_v2023-07_fsp_v4.6.0/toolchains/gcc_arm/arm-gnu-toolchain-12.2.mpacbti-rel1-mingw-w64-i686-arm-none-eabi/bin/../lib/gcc/arm-none-eabi/12.2.1/thumb/v8-m.main+fp/hard\libg_nano.a(libc_a-itoa.o)
 .ARM.attributes
                0x00000a74       0x38 c:/renesas/ra/e2studio_v2023-07_fsp_v4.6.0/toolchains/gcc_arm/arm-gnu-toolchain-12.2.mpacbti-rel1-mingw-w64-i686-arm-none-eabi/bin/../lib/gcc/arm-none-eabi/12.2.1/thumb/v8-m.main+fp/hard\libg_nano.a(libc_a-strtol.o)
 .ARM.attributes
                0x00000aac       0x38 c:/renesas/ra/e2studio_v2023-07_fsp_v4.6.0/toolchains/gcc_arm/arm-gnu-toolchain-12.2.mpacbti-rel1-mingw-w64-i686-arm-none-eabi/bin/../lib/gcc/arm-none-eabi/12.2.1/thumb/v8-m.main+fp/hard\libg_nano.a(libc_a-utoa.o)
 .ARM.attributes
                0x00000ae4       0x38 c:/renesas/ra/e2studio_v2023-07_fsp_v4.6.0/toolchains/gcc_arm/arm-gnu-toolchain-12.2.mpacbti-rel1-mingw-w64-i686-arm-none-eabi/bin/../lib/gcc/arm-none-eabi/12.2.1/thumb/v8-m.main+fp/hard\libg_nano.a(libc_a-ctype_.o)
 .ARM.attributes
                0x00000b1c       0x38 c:/renesas/ra/e2studio_v2023-07_fsp_v4.6.0/toolchains/gcc_arm/arm-gnu-toolchain-12.2.mpacbti-rel1-mingw-w64-i686-arm-none-eabi/bin/../lib/gcc/arm-none-eabi/12.2.1/thumb/v8-m.main+fp/hard\libg_nano.a(libc_a-findfp.o)
 .ARM.attributes
                0x00000b54       0x38 c:/renesas/ra/e2studio_v2023-07_fsp_v4.6.0/toolchains/gcc_arm/arm-gnu-toolchain-12.2.mpacbti-rel1-mingw-w64-i686-arm-none-eabi/bin/../lib/gcc/arm-none-eabi/12.2.1/thumb/v8-m.main+fp/hard\libg_nano.a(libc_a-memset.o)
 .ARM.attributes
                0x00000b8c       0x38 c:/renesas/ra/e2studio_v2023-07_fsp_v4.6.0/toolchains/gcc_arm/arm-gnu-toolchain-12.2.mpacbti-rel1-mingw-w64-i686-arm-none-eabi/bin/../lib/gcc/arm-none-eabi/12.2.1/thumb/v8-m.main+fp/hard\libg_nano.a(libc_a-strncmp.o)
 .ARM.attributes
                0x00000bc4       0x38 c:/renesas/ra/e2studio_v2023-07_fsp_v4.6.0/toolchains/gcc_arm/arm-gnu-toolchain-12.2.mpacbti-rel1-mingw-w64-i686-arm-none-eabi/bin/../lib/gcc/arm-none-eabi/12.2.1/thumb/v8-m.main+fp/hard\libg_nano.a(libc_a-impure.o)
 .ARM.attributes
                0x00000bfc       0x38 c:/renesas/ra/e2studio_v2023-07_fsp_v4.6.0/toolchains/gcc_arm/arm-gnu-toolchain-12.2.mpacbti-rel1-mingw-w64-i686-arm-none-eabi/bin/../lib/gcc/arm-none-eabi/12.2.1/thumb/v8-m.main+fp/hard\libg_nano.a(libc_a-errno.o)
 .ARM.attributes
                0x00000c34       0x38 c:/renesas/ra/e2studio_v2023-07_fsp_v4.6.0/toolchains/gcc_arm/arm-gnu-toolchain-12.2.mpacbti-rel1-mingw-w64-i686-arm-none-eabi/bin/../lib/gcc/arm-none-eabi/12.2.1/thumb/v8-m.main+fp/hard\libg_nano.a(libc_a-strcpy.o)
 .ARM.attributes
                0x00000c6c       0x38 c:/renesas/ra/e2studio_v2023-07_fsp_v4.6.0/toolchains/gcc_arm/arm-gnu-toolchain-12.2.mpacbti-rel1-mingw-w64-i686-arm-none-eabi/bin/../lib/gcc/arm-none-eabi/12.2.1/thumb/v8-m.main+fp/hard\libg_nano.a(libc_a-aeabi_memcpy.o)
 .ARM.attributes
                0x00000ca4       0x38 c:/renesas/ra/e2studio_v2023-07_fsp_v4.6.0/toolchains/gcc_arm/arm-gnu-toolchain-12.2.mpacbti-rel1-mingw-w64-i686-arm-none-eabi/bin/../lib/gcc/arm-none-eabi/12.2.1/thumb/v8-m.main+fp/hard\libg_nano.a(libc_a-aeabi_memclr.o)
 .ARM.attributes
                0x00000cdc       0x38 c:/renesas/ra/e2studio_v2023-07_fsp_v4.6.0/toolchains/gcc_arm/arm-gnu-toolchain-12.2.mpacbti-rel1-mingw-w64-i686-arm-none-eabi/bin/../lib/gcc/arm-none-eabi/12.2.1/thumb/v8-m.main+fp/hard\libg_nano.a(libc_a-memcpy-stub.o)
 .ARM.attributes
                0x00000d14       0x24 c:/renesas/ra/e2studio_v2023-07_fsp_v4.6.0/toolchains/gcc_arm/arm-gnu-toolchain-12.2.mpacbti-rel1-mingw-w64-i686-arm-none-eabi/bin/../lib/gcc/arm-none-eabi/12.2.1/thumb/v8-m.main+fp/hard\libg_nano.a(libc_a-strlen.o)
 .ARM.attributes
                0x00000d38       0x24 c:/renesas/ra/e2studio_v2023-07_fsp_v4.6.0/toolchains/gcc_arm/arm-gnu-toolchain-12.2.mpacbti-rel1-mingw-w64-i686-arm-none-eabi/bin/../lib/gcc/arm-none-eabi/12.2.1/thumb/v8-m.main+fp/hard\libg_nano.a(libc_a-aeabi_memset-soft.o)
 .ARM.attributes
                0x00000d5c       0x38 c:/renesas/ra/e2studio_v2023-07_fsp_v4.6.0/toolchains/gcc_arm/arm-gnu-toolchain-12.2.mpacbti-rel1-mingw-w64-i686-arm-none-eabi/bin/../lib/gcc/arm-none-eabi/12.2.1/thumb/v8-m.main+fp/hard/crtend.o
 .ARM.attributes
                0x00000d94       0x26 c:/renesas/ra/e2studio_v2023-07_fsp_v4.6.0/toolchains/gcc_arm/arm-gnu-toolchain-12.2.mpacbti-rel1-mingw-w64-i686-arm-none-eabi/bin/../lib/gcc/arm-none-eabi/12.2.1/thumb/v8-m.main+fp/hard/crtn.o

.comment        0x00000000       0x55
 .comment       0x00000000       0x55 ./src/adc_temp.o
                                 0x56 (size before relaxing)
 .comment       0x00000055       0x56 ./src/angle.o
 .comment       0x00000055       0x56 ./src/control_table.o
 .comment       0x00000055       0x56 ./src/global_variables.o
 .comment       0x00000055       0x56 ./src/hal_entry.o
 .comment       0x00000055       0x56 ./src/interpolation.o
 .comment       0x00000055       0x56 ./src/monitor.o
 .comment       0x00000055       0x56 ./src/packet.o
 .comment       0x00000055       0x56 ./src/pid.o
 .comment       0x00000055       0x56 ./src/power_monitor.o
 .comment       0x00000055       0x56 ./src/sintable.o
 .comment       0x00000055       0x56 ./src/usart.o
 .comment       0x00000055       0x56 ./ra_gen/common_data.o
 .comment       0x00000055       0x56 ./ra_gen/hal_data.o
 .comment       0x00000055       0x56 ./ra_gen/main.o
 .comment       0x00000055       0x56 ./ra_gen/pin_data.o
 .comment       0x00000055       0x56 ./ra_gen/vector_data.o
 .comment       0x00000055       0x56 ./ra/fsp/src/r_sci_uart/r_sci_uart.o
 .comment       0x00000055       0x56 ./ra/fsp/src/r_sci_spi/r_sci_spi.o
 .comment       0x00000055       0x56 ./ra/fsp/src/r_sci_i2c/r_sci_i2c.o
 .comment       0x00000055       0x56 ./ra/fsp/src/r_rtc/r_rtc.o
 .comment       0x00000055       0x56 ./ra/fsp/src/r_ioport/r_ioport.o
 .comment       0x00000055       0x56 ./ra/fsp/src/r_gpt/r_gpt.o
 .comment       0x00000055       0x56 ./ra/fsp/src/r_flash_hp/r_flash_hp.o
 .comment       0x00000055       0x56 ./ra/fsp/src/r_dtc/r_dtc.o
 .comment       0x00000055       0x56 ./ra/fsp/src/r_crc/r_crc.o
 .comment       0x00000055       0x56 ./ra/fsp/src/r_agt/r_agt.o
 .comment       0x00000055       0x56 ./ra/fsp/src/r_adc/r_adc.o
 .comment       0x00000055       0x56 ./ra/fsp/src/bsp/mcu/all/bsp_clocks.o
 .comment       0x00000055       0x56 ./ra/fsp/src/bsp/mcu/all/bsp_common.o
 .comment       0x00000055       0x56 ./ra/fsp/src/bsp/mcu/all/bsp_delay.o
 .comment       0x00000055       0x56 ./ra/fsp/src/bsp/mcu/all/bsp_group_irq.o
 .comment       0x00000055       0x56 ./ra/fsp/src/bsp/mcu/all/bsp_io.o
 .comment       0x00000055       0x56 ./ra/fsp/src/bsp/mcu/all/bsp_irq.o
 .comment       0x00000055       0x56 ./ra/fsp/src/bsp/mcu/all/bsp_register_protection.o
 .comment       0x00000055       0x56 ./ra/fsp/src/bsp/mcu/all/bsp_rom_registers.o
 .comment       0x00000055       0x56 ./ra/fsp/src/bsp/cmsis/Device/RENESAS/Source/startup.o
 .comment       0x00000055       0x56 ./ra/fsp/src/bsp/cmsis/Device/RENESAS/Source/system.o

.debug_info     0x00000000    0x85a8c
 .debug_info    0x00000000     0x3226 ./src/adc_temp.o
 .debug_info    0x00003226     0x6c38 ./src/angle.o
 .debug_info    0x00009e5e     0x194c ./src/control_table.o
 .debug_info    0x0000b7aa      0x237 ./src/global_variables.o
 .debug_info    0x0000b9e1     0x8d27 ./src/hal_entry.o
 .debug_info    0x00014708       0xee ./src/interpolation.o
 .debug_info    0x000147f6      0x603 ./src/monitor.o
 .debug_info    0x00014df9     0x3fa6 ./src/packet.o
 .debug_info    0x00018d9f      0x3f2 ./src/pid.o
 .debug_info    0x00019191     0x282e ./src/power_monitor.o
 .debug_info    0x0001b9bf      0x120 ./src/sintable.o
 .debug_info    0x0001badf     0x3d8e ./src/usart.o
 .debug_info    0x0001f86d     0x11d4 ./ra_gen/common_data.o
 .debug_info    0x00020a41     0xc0cb ./ra_gen/hal_data.o
 .debug_info    0x0002cb0c       0xa3 ./ra_gen/main.o
 .debug_info    0x0002cbaf      0x9f7 ./ra_gen/pin_data.o
 .debug_info    0x0002d5a6      0x6a6 ./ra_gen/vector_data.o
 .debug_info    0x0002dc4c     0x9f81 ./ra/fsp/src/r_sci_uart/r_sci_uart.o
 .debug_info    0x00037bcd     0x916e ./ra/fsp/src/r_sci_spi/r_sci_spi.o
 .debug_info    0x00040d3b     0x4ef6 ./ra/fsp/src/r_sci_i2c/r_sci_i2c.o
 .debug_info    0x00045c31     0x42ee ./ra/fsp/src/r_rtc/r_rtc.o
 .debug_info    0x00049f1f     0x6496 ./ra/fsp/src/r_ioport/r_ioport.o
 .debug_info    0x000503b5     0xa65f ./ra/fsp/src/r_gpt/r_gpt.o
 .debug_info    0x0005aa14     0x7af3 ./ra/fsp/src/r_flash_hp/r_flash_hp.o
 .debug_info    0x00062507     0x28a5 ./ra/fsp/src/r_dtc/r_dtc.o
 .debug_info    0x00064dac     0x1c14 ./ra/fsp/src/r_crc/r_crc.o
 .debug_info    0x000669c0     0x7455 ./ra/fsp/src/r_agt/r_agt.o
 .debug_info    0x0006de15     0xae78 ./ra/fsp/src/r_adc/r_adc.o
 .debug_info    0x00078c8d     0x5238 ./ra/fsp/src/bsp/mcu/all/bsp_clocks.o
 .debug_info    0x0007dec5      0x903 ./ra/fsp/src/bsp/mcu/all/bsp_common.o
 .debug_info    0x0007e7c8      0x1c4 ./ra/fsp/src/bsp/mcu/all/bsp_delay.o
 .debug_info    0x0007e98c     0x125f ./ra/fsp/src/bsp/mcu/all/bsp_group_irq.o
 .debug_info    0x0007fbeb       0xa4 ./ra/fsp/src/bsp/mcu/all/bsp_io.o
 .debug_info    0x0007fc8f     0x1a5f ./ra/fsp/src/bsp/mcu/all/bsp_irq.o
 .debug_info    0x000816ee     0x3772 ./ra/fsp/src/bsp/mcu/all/bsp_register_protection.o
 .debug_info    0x00084e60      0x1aa ./ra/fsp/src/bsp/mcu/all/bsp_rom_registers.o
 .debug_info    0x0008500a      0x15a ./ra/fsp/src/bsp/cmsis/Device/RENESAS/Source/startup.o
 .debug_info    0x00085164      0x928 ./ra/fsp/src/bsp/cmsis/Device/RENESAS/Source/system.o

.debug_abbrev   0x00000000     0x78cc
 .debug_abbrev  0x00000000      0x263 ./src/adc_temp.o
 .debug_abbrev  0x00000263      0x4f3 ./src/angle.o
 .debug_abbrev  0x00000756      0x45b ./src/control_table.o
 .debug_abbrev  0x00000bb1       0xbd ./src/global_variables.o
 .debug_abbrev  0x00000c6e      0x5f1 ./src/hal_entry.o
 .debug_abbrev  0x0000125f       0x90 ./src/interpolation.o
 .debug_abbrev  0x000012ef      0x1ca ./src/monitor.o
 .debug_abbrev  0x000014b9      0x66d ./src/packet.o
 .debug_abbrev  0x00001b26      0x118 ./src/pid.o
 .debug_abbrev  0x00001c3e      0x321 ./src/power_monitor.o
 .debug_abbrev  0x00001f5f       0xb1 ./src/sintable.o
 .debug_abbrev  0x00002010      0x62c ./src/usart.o
 .debug_abbrev  0x0000263c      0x159 ./ra_gen/common_data.o
 .debug_abbrev  0x00002795      0x325 ./ra_gen/hal_data.o
 .debug_abbrev  0x00002aba       0x61 ./ra_gen/main.o
 .debug_abbrev  0x00002b1b       0xe3 ./ra_gen/pin_data.o
 .debug_abbrev  0x00002bfe       0xbd ./ra_gen/vector_data.o
 .debug_abbrev  0x00002cbb      0x5fb ./ra/fsp/src/r_sci_uart/r_sci_uart.o
 .debug_abbrev  0x000032b6      0x617 ./ra/fsp/src/r_sci_spi/r_sci_spi.o
 .debug_abbrev  0x000038cd      0x567 ./ra/fsp/src/r_sci_i2c/r_sci_i2c.o
 .debug_abbrev  0x00003e34      0x57d ./ra/fsp/src/r_rtc/r_rtc.o
 .debug_abbrev  0x000043b1      0x47f ./ra/fsp/src/r_ioport/r_ioport.o
 .debug_abbrev  0x00004830      0x626 ./ra/fsp/src/r_gpt/r_gpt.o
 .debug_abbrev  0x00004e56      0x591 ./ra/fsp/src/r_flash_hp/r_flash_hp.o
 .debug_abbrev  0x000053e7      0x4b1 ./ra/fsp/src/r_dtc/r_dtc.o
 .debug_abbrev  0x00005898      0x329 ./ra/fsp/src/r_crc/r_crc.o
 .debug_abbrev  0x00005bc1      0x592 ./ra/fsp/src/r_agt/r_agt.o
 .debug_abbrev  0x00006153      0x583 ./ra/fsp/src/r_adc/r_adc.o
 .debug_abbrev  0x000066d6      0x3cd ./ra/fsp/src/bsp/mcu/all/bsp_clocks.o
 .debug_abbrev  0x00006aa3      0x175 ./ra/fsp/src/bsp/mcu/all/bsp_common.o
 .debug_abbrev  0x00006c18      0x10b ./ra/fsp/src/bsp/mcu/all/bsp_delay.o
 .debug_abbrev  0x00006d23      0x254 ./ra/fsp/src/bsp/mcu/all/bsp_group_irq.o
 .debug_abbrev  0x00006f77       0x5e ./ra/fsp/src/bsp/mcu/all/bsp_io.o
 .debug_abbrev  0x00006fd5      0x271 ./ra/fsp/src/bsp/mcu/all/bsp_irq.o
 .debug_abbrev  0x00007246      0x27d ./ra/fsp/src/bsp/mcu/all/bsp_register_protection.o
 .debug_abbrev  0x000074c3       0x4e ./ra/fsp/src/bsp/mcu/all/bsp_rom_registers.o
 .debug_abbrev  0x00007511       0xf5 ./ra/fsp/src/bsp/cmsis/Device/RENESAS/Source/startup.o
 .debug_abbrev  0x00007606      0x2c6 ./ra/fsp/src/bsp/cmsis/Device/RENESAS/Source/system.o

.debug_aranges  0x00000000      0xba0
 .debug_aranges
                0x00000000       0x40 ./src/adc_temp.o
 .debug_aranges
                0x00000040       0x48 ./src/angle.o
 .debug_aranges
                0x00000088       0x40 ./src/control_table.o
 .debug_aranges
                0x000000c8       0x18 ./src/global_variables.o
 .debug_aranges
                0x000000e0       0x60 ./src/hal_entry.o
 .debug_aranges
                0x00000140       0x20 ./src/interpolation.o
 .debug_aranges
                0x00000160       0x20 ./src/monitor.o
 .debug_aranges
                0x00000180       0xe8 ./src/packet.o
 .debug_aranges
                0x00000268       0x38 ./src/pid.o
 .debug_aranges
                0x000002a0       0x50 ./src/power_monitor.o
 .debug_aranges
                0x000002f0       0x28 ./src/sintable.o
 .debug_aranges
                0x00000318       0x80 ./src/usart.o
 .debug_aranges
                0x00000398       0x20 ./ra_gen/common_data.o
 .debug_aranges
                0x000003b8       0x20 ./ra_gen/hal_data.o
 .debug_aranges
                0x000003d8       0x20 ./ra_gen/main.o
 .debug_aranges
                0x000003f8       0x18 ./ra_gen/pin_data.o
 .debug_aranges
                0x00000410       0x18 ./ra_gen/vector_data.o
 .debug_aranges
                0x00000428       0x88 ./ra/fsp/src/r_sci_uart/r_sci_uart.o
 .debug_aranges
                0x000004b0       0x70 ./ra/fsp/src/r_sci_spi/r_sci_spi.o
 .debug_aranges
                0x00000520       0x70 ./ra/fsp/src/r_sci_i2c/r_sci_i2c.o
 .debug_aranges
                0x00000590       0x80 ./ra/fsp/src/r_rtc/r_rtc.o
 .debug_aranges
                0x00000610       0x90 ./ra/fsp/src/r_ioport/r_ioport.o
 .debug_aranges
                0x000006a0       0xc8 ./ra/fsp/src/r_gpt/r_gpt.o
 .debug_aranges
                0x00000768       0xb0 ./ra/fsp/src/r_flash_hp/r_flash_hp.o
 .debug_aranges
                0x00000818       0x60 ./ra/fsp/src/r_dtc/r_dtc.o
 .debug_aranges
                0x00000878       0x48 ./ra/fsp/src/r_crc/r_crc.o
 .debug_aranges
                0x000008c0       0x80 ./ra/fsp/src/r_agt/r_agt.o
 .debug_aranges
                0x00000940       0xa8 ./ra/fsp/src/r_adc/r_adc.o
 .debug_aranges
                0x000009e8       0x70 ./ra/fsp/src/bsp/mcu/all/bsp_clocks.o
 .debug_aranges
                0x00000a58       0x30 ./ra/fsp/src/bsp/mcu/all/bsp_common.o
 .debug_aranges
                0x00000a88       0x28 ./ra/fsp/src/bsp/mcu/all/bsp_delay.o
 .debug_aranges
                0x00000ab0       0x28 ./ra/fsp/src/bsp/mcu/all/bsp_group_irq.o
 .debug_aranges
                0x00000ad8       0x18 ./ra/fsp/src/bsp/mcu/all/bsp_io.o
 .debug_aranges
                0x00000af0       0x20 ./ra/fsp/src/bsp/mcu/all/bsp_irq.o
 .debug_aranges
                0x00000b10       0x28 ./ra/fsp/src/bsp/mcu/all/bsp_register_protection.o
 .debug_aranges
                0x00000b38       0x18 ./ra/fsp/src/bsp/mcu/all/bsp_rom_registers.o
 .debug_aranges
                0x00000b50       0x28 ./ra/fsp/src/bsp/cmsis/Device/RENESAS/Source/startup.o
 .debug_aranges
                0x00000b78       0x28 ./ra/fsp/src/bsp/cmsis/Device/RENESAS/Source/system.o

.debug_rnglists
                0x00000000     0x28b2
 .debug_rnglists
                0x00000000       0x2d ./src/adc_temp.o
 .debug_rnglists
                0x0000002d       0xd4 ./src/angle.o
 .debug_rnglists
                0x00000101       0xb6 ./src/control_table.o
 .debug_rnglists
                0x000001b7      0x115 ./src/hal_entry.o
 .debug_rnglists
                0x000002cc       0x14 ./src/interpolation.o
 .debug_rnglists
                0x000002e0       0x24 ./src/monitor.o
 .debug_rnglists
                0x00000304      0x6d2 ./src/packet.o
 .debug_rnglists
                0x000009d6       0x26 ./src/pid.o
 .debug_rnglists
                0x000009fc       0x3b ./src/power_monitor.o
 .debug_rnglists
                0x00000a37       0x1a ./src/sintable.o
 .debug_rnglists
                0x00000a51      0x1ba ./src/usart.o
 .debug_rnglists
                0x00000c0b       0x13 ./ra_gen/common_data.o
 .debug_rnglists
                0x00000c1e       0x13 ./ra_gen/hal_data.o
 .debug_rnglists
                0x00000c31       0x13 ./ra_gen/main.o
 .debug_rnglists
                0x00000c44      0x369 ./ra/fsp/src/r_sci_uart/r_sci_uart.o
 .debug_rnglists
                0x00000fad      0x3f5 ./ra/fsp/src/r_sci_spi/r_sci_spi.o
 .debug_rnglists
                0x000013a2      0x28e ./ra/fsp/src/r_sci_i2c/r_sci_i2c.o
 .debug_rnglists
                0x00001630      0x2a4 ./ra/fsp/src/r_rtc/r_rtc.o
 .debug_rnglists
                0x000018d4       0xda ./ra/fsp/src/r_ioport/r_ioport.o
 .debug_rnglists
                0x000019ae      0x302 ./ra/fsp/src/r_gpt/r_gpt.o
 .debug_rnglists
                0x00001cb0      0x3d3 ./ra/fsp/src/r_flash_hp/r_flash_hp.o
 .debug_rnglists
                0x00002083       0xd4 ./ra/fsp/src/r_dtc/r_dtc.o
 .debug_rnglists
                0x00002157       0xee ./ra/fsp/src/r_crc/r_crc.o
 .debug_rnglists
                0x00002245      0x1ce ./ra/fsp/src/r_agt/r_agt.o
 .debug_rnglists
                0x00002413      0x2ca ./ra/fsp/src/r_adc/r_adc.o
 .debug_rnglists
                0x000026dd       0xac ./ra/fsp/src/bsp/mcu/all/bsp_clocks.o
 .debug_rnglists
                0x00002789       0x1f ./ra/fsp/src/bsp/mcu/all/bsp_common.o
 .debug_rnglists
                0x000027a8       0x19 ./ra/fsp/src/bsp/mcu/all/bsp_delay.o
 .debug_rnglists
                0x000027c1       0x37 ./ra/fsp/src/bsp/mcu/all/bsp_group_irq.o
 .debug_rnglists
                0x000027f8       0x3e ./ra/fsp/src/bsp/mcu/all/bsp_irq.o
 .debug_rnglists
                0x00002836       0x31 ./ra/fsp/src/bsp/mcu/all/bsp_register_protection.o
 .debug_rnglists
                0x00002867       0x19 ./ra/fsp/src/bsp/cmsis/Device/RENESAS/Source/startup.o
 .debug_rnglists
                0x00002880       0x32 ./ra/fsp/src/bsp/cmsis/Device/RENESAS/Source/system.o

.debug_line     0x00000000    0x199fa
 .debug_line    0x00000000      0x401 ./src/adc_temp.o
 .debug_line    0x00000401      0xb31 ./src/angle.o
 .debug_line    0x00000f32      0xa7d ./src/control_table.o
 .debug_line    0x000019af      0x1b0 ./src/global_variables.o
 .debug_line    0x00001b5f     0x1bb6 ./src/hal_entry.o
 .debug_line    0x00003715      0x248 ./src/interpolation.o
 .debug_line    0x0000395d      0x337 ./src/monitor.o
 .debug_line    0x00003c94     0x277d ./src/packet.o
 .debug_line    0x00006411      0x30b ./src/pid.o
 .debug_line    0x0000671c      0x5e3 ./src/power_monitor.o
 .debug_line    0x00006cff      0x2c2 ./src/sintable.o
 .debug_line    0x00006fc1     0x16d2 ./src/usart.o
 .debug_line    0x00008693      0x303 ./ra_gen/common_data.o
 .debug_line    0x00008996      0x53b ./ra_gen/hal_data.o
 .debug_line    0x00008ed1       0x5e ./ra_gen/main.o
 .debug_line    0x00008f2f      0x22a ./ra_gen/pin_data.o
 .debug_line    0x00009159      0x12c ./ra_gen/vector_data.o
 .debug_line    0x00009285     0x202c ./ra/fsp/src/r_sci_uart/r_sci_uart.o
 .debug_line    0x0000b2b1     0x1942 ./ra/fsp/src/r_sci_spi/r_sci_spi.o
 .debug_line    0x0000cbf3     0x112b ./ra/fsp/src/r_sci_i2c/r_sci_i2c.o
 .debug_line    0x0000dd1e     0x17c3 ./ra/fsp/src/r_rtc/r_rtc.o
 .debug_line    0x0000f4e1      0xc26 ./ra/fsp/src/r_ioport/r_ioport.o
 .debug_line    0x00010107     0x17a2 ./ra/fsp/src/r_gpt/r_gpt.o
 .debug_line    0x000118a9     0x1f96 ./ra/fsp/src/r_flash_hp/r_flash_hp.o
 .debug_line    0x0001383f      0x9e6 ./ra/fsp/src/r_dtc/r_dtc.o
 .debug_line    0x00014225      0x6d4 ./ra/fsp/src/r_crc/r_crc.o
 .debug_line    0x000148f9     0x10ef ./ra/fsp/src/r_agt/r_agt.o
 .debug_line    0x000159e8     0x16d7 ./ra/fsp/src/r_adc/r_adc.o
 .debug_line    0x000170bf      0x928 ./ra/fsp/src/bsp/mcu/all/bsp_clocks.o
 .debug_line    0x000179e7      0x35a ./ra/fsp/src/bsp/mcu/all/bsp_common.o
 .debug_line    0x00017d41      0x30a ./ra/fsp/src/bsp/mcu/all/bsp_delay.o
 .debug_line    0x0001804b      0x35f ./ra/fsp/src/bsp/mcu/all/bsp_group_irq.o
 .debug_line    0x000183aa      0x1ea ./ra/fsp/src/bsp/mcu/all/bsp_io.o
 .debug_line    0x00018594      0x5d4 ./ra/fsp/src/bsp/mcu/all/bsp_irq.o
 .debug_line    0x00018b68      0x413 ./ra/fsp/src/bsp/mcu/all/bsp_register_protection.o
 .debug_line    0x00018f7b      0x1a5 ./ra/fsp/src/bsp/mcu/all/bsp_rom_registers.o
 .debug_line    0x00019120      0x26e ./ra/fsp/src/bsp/cmsis/Device/RENESAS/Source/startup.o
 .debug_line    0x0001938e      0x66c ./ra/fsp/src/bsp/cmsis/Device/RENESAS/Source/system.o

.debug_str      0x00000000    0x13d0f
 .debug_str     0x00000000     0x30c7 ./src/adc_temp.o
                               0x31c6 (size before relaxing)
 .debug_str     0x000030c7     0x4289 ./src/angle.o
                               0x5fb3 (size before relaxing)
 .debug_str     0x00007350      0x9ba ./src/control_table.o
                               0x25ee (size before relaxing)
 .debug_str     0x00007d0a       0xf4 ./src/global_variables.o
                                0x2aa (size before relaxing)
 .debug_str     0x00007dfe      0xee4 ./src/hal_entry.o
                               0x705a (size before relaxing)
 .debug_str     0x00008ce2       0x17 ./src/interpolation.o
                                0x1b1 (size before relaxing)
 .debug_str     0x00008cf9       0x66 ./src/monitor.o
                                0x609 (size before relaxing)
 .debug_str     0x00008d5f      0x20f ./src/packet.o
                                0xaa9 (size before relaxing)
 .debug_str     0x00008f6e       0x69 ./src/pid.o
                                0x293 (size before relaxing)
 .debug_str     0x00008fd7      0x3c4 ./src/power_monitor.o
                               0x2a8a (size before relaxing)
 .debug_str     0x0000939b       0x2f ./src/sintable.o
                                0x1db (size before relaxing)
 .debug_str     0x000093ca      0x4a7 ./src/usart.o
                               0x407b (size before relaxing)
 .debug_str     0x00009871       0x39 ./ra_gen/common_data.o
                               0x3244 (size before relaxing)
 .debug_str     0x000098aa     0x4221 ./ra_gen/hal_data.o
                               0xc116 (size before relaxing)
 .debug_str     0x0000dacb       0x11 ./ra_gen/main.o
                                0x1a8 (size before relaxing)
 .debug_str     0x0000dadc       0x28 ./ra_gen/pin_data.o
                               0x1d2a (size before relaxing)
 .debug_str     0x0000db04      0x126 ./ra_gen/vector_data.o
                               0x16de (size before relaxing)
 .debug_str     0x0000dc2a     0x2310 ./ra/fsp/src/r_sci_uart/r_sci_uart.o
                               0x68f9 (size before relaxing)
 .debug_str     0x0000ff3a      0x156 ./ra/fsp/src/r_sci_spi/r_sci_spi.o
                               0x5020 (size before relaxing)
 .debug_str     0x00010090      0x207 ./ra/fsp/src/r_sci_i2c/r_sci_i2c.o
                               0x3731 (size before relaxing)
 .debug_str     0x00010297      0x5a1 ./ra/fsp/src/r_rtc/r_rtc.o
                               0x2fa4 (size before relaxing)
 .debug_str     0x00010838      0x874 ./ra/fsp/src/r_ioport/r_ioport.o
                               0x56f7 (size before relaxing)
 .debug_str     0x000110ac      0xa87 ./ra/fsp/src/r_gpt/r_gpt.o
                               0x69e7 (size before relaxing)
 .debug_str     0x00011b33      0x6a1 ./ra/fsp/src/r_flash_hp/r_flash_hp.o
                               0x46a2 (size before relaxing)
 .debug_str     0x000121d4      0x1d2 ./ra/fsp/src/r_dtc/r_dtc.o
                               0x2c4c (size before relaxing)
 .debug_str     0x000123a6      0x197 ./ra/fsp/src/r_crc/r_crc.o
                               0x23e5 (size before relaxing)
 .debug_str     0x0001253d      0x1e3 ./ra/fsp/src/r_agt/r_agt.o
                               0x4a2f (size before relaxing)
 .debug_str     0x00012720      0x5f8 ./ra/fsp/src/r_adc/r_adc.o
                               0x7cf2 (size before relaxing)
 .debug_str     0x00012d18      0x5b5 ./ra/fsp/src/bsp/mcu/all/bsp_clocks.o
                               0x24de (size before relaxing)
 .debug_str     0x000132cd      0x10b ./ra/fsp/src/bsp/mcu/all/bsp_common.o
                               0x1b58 (size before relaxing)
 .debug_str     0x000133d8       0x9f ./ra/fsp/src/bsp/mcu/all/bsp_delay.o
                                0x2d1 (size before relaxing)
 .debug_str     0x00013477      0x1de ./ra/fsp/src/bsp/mcu/all/bsp_group_irq.o
                               0x2063 (size before relaxing)
 .debug_str     0x00013655       0x23 ./ra/fsp/src/bsp/mcu/all/bsp_io.o
                                0x1d1 (size before relaxing)
 .debug_str     0x00013678      0x36f ./ra/fsp/src/bsp/mcu/all/bsp_irq.o
                               0x1ef0 (size before relaxing)
 .debug_str     0x000139e7       0x76 ./ra/fsp/src/bsp/mcu/all/bsp_register_protection.o
                               0x1a88 (size before relaxing)
 .debug_str     0x00013a5d      0x16f ./ra/fsp/src/bsp/mcu/all/bsp_rom_registers.o
                                0x305 (size before relaxing)
 .debug_str     0x00013bcc       0x82 ./ra/fsp/src/bsp/cmsis/Device/RENESAS/Source/startup.o
                                0x239 (size before relaxing)
 .debug_str     0x00013c4e       0xc1 ./ra/fsp/src/bsp/cmsis/Device/RENESAS/Source/system.o
                                0x63c (size before relaxing)

.debug_frame    0x00000000     0x24a8
 .debug_frame   0x00000000       0xb0 ./src/adc_temp.o
 .debug_frame   0x000000b0       0xd0 ./src/angle.o
 .debug_frame   0x00000180       0xfc ./src/control_table.o
 .debug_frame   0x0000027c       0xfc ./src/hal_entry.o
 .debug_frame   0x00000378       0x34 ./src/interpolation.o
 .debug_frame   0x000003ac       0x38 ./src/monitor.o
 .debug_frame   0x000003e4      0x418 ./src/packet.o
 .debug_frame   0x000007fc       0x7c ./src/pid.o
 .debug_frame   0x00000878      0x108 ./src/power_monitor.o
 .debug_frame   0x00000980       0x30 ./src/sintable.o
 .debug_frame   0x000009b0      0x1a8 ./src/usart.o
 .debug_frame   0x00000b58       0x20 ./ra_gen/common_data.o
 .debug_frame   0x00000b78       0x20 ./ra_gen/hal_data.o
 .debug_frame   0x00000b98       0x28 ./ra_gen/main.o
 .debug_frame   0x00000bc0      0x1e8 ./ra/fsp/src/r_sci_uart/r_sci_uart.o
 .debug_frame   0x00000da8      0x168 ./ra/fsp/src/r_sci_spi/r_sci_spi.o
 .debug_frame   0x00000f10      0x118 ./ra/fsp/src/r_sci_i2c/r_sci_i2c.o
 .debug_frame   0x00001028      0x174 ./ra/fsp/src/r_rtc/r_rtc.o
 .debug_frame   0x0000119c      0x168 ./ra/fsp/src/r_ioport/r_ioport.o
 .debug_frame   0x00001304      0x230 ./ra/fsp/src/r_gpt/r_gpt.o
 .debug_frame   0x00001534      0x254 ./ra/fsp/src/r_flash_hp/r_flash_hp.o
 .debug_frame   0x00001788       0xf4 ./ra/fsp/src/r_dtc/r_dtc.o
 .debug_frame   0x0000187c       0x90 ./ra/fsp/src/r_crc/r_crc.o
 .debug_frame   0x0000190c      0x198 ./ra/fsp/src/r_agt/r_agt.o
 .debug_frame   0x00001aa4      0x1bc ./ra/fsp/src/r_adc/r_adc.o
 .debug_frame   0x00001c60       0xf4 ./ra/fsp/src/bsp/mcu/all/bsp_clocks.o
 .debug_frame   0x00001d54       0x40 ./ra/fsp/src/bsp/mcu/all/bsp_common.o
 .debug_frame   0x00001d94       0x48 ./ra/fsp/src/bsp/mcu/all/bsp_delay.o
 .debug_frame   0x00001ddc       0x3c ./ra/fsp/src/bsp/mcu/all/bsp_group_irq.o
 .debug_frame   0x00001e18       0x30 ./ra/fsp/src/bsp/mcu/all/bsp_irq.o
 .debug_frame   0x00001e48       0x48 ./ra/fsp/src/bsp/mcu/all/bsp_register_protection.o
 .debug_frame   0x00001e90       0x38 ./ra/fsp/src/bsp/cmsis/Device/RENESAS/Source/startup.o
 .debug_frame   0x00001ec8       0x44 ./ra/fsp/src/bsp/cmsis/Device/RENESAS/Source/system.o
 .debug_frame   0x00001f0c       0xac c:/renesas/ra/e2studio_v2023-07_fsp_v4.6.0/toolchains/gcc_arm/arm-gnu-toolchain-12.2.mpacbti-rel1-mingw-w64-i686-arm-none-eabi/bin/../lib/gcc/arm-none-eabi/12.2.1/thumb/v8-m.main+fp/hard\libgcc.a(_arm_addsubdf3.o)
 .debug_frame   0x00001fb8       0x50 c:/renesas/ra/e2studio_v2023-07_fsp_v4.6.0/toolchains/gcc_arm/arm-gnu-toolchain-12.2.mpacbti-rel1-mingw-w64-i686-arm-none-eabi/bin/../lib/gcc/arm-none-eabi/12.2.1/thumb/v8-m.main+fp/hard\libgcc.a(_arm_muldivdf3.o)
 .debug_frame   0x00002008       0xc4 c:/renesas/ra/e2studio_v2023-07_fsp_v4.6.0/toolchains/gcc_arm/arm-gnu-toolchain-12.2.mpacbti-rel1-mingw-w64-i686-arm-none-eabi/bin/../lib/gcc/arm-none-eabi/12.2.1/thumb/v8-m.main+fp/hard\libgcc.a(_arm_cmpdf2.o)
 .debug_frame   0x000020cc       0x24 c:/renesas/ra/e2studio_v2023-07_fsp_v4.6.0/toolchains/gcc_arm/arm-gnu-toolchain-12.2.mpacbti-rel1-mingw-w64-i686-arm-none-eabi/bin/../lib/gcc/arm-none-eabi/12.2.1/thumb/v8-m.main+fp/hard\libgcc.a(_arm_fixdfsi.o)
 .debug_frame   0x000020f0       0x24 c:/renesas/ra/e2studio_v2023-07_fsp_v4.6.0/toolchains/gcc_arm/arm-gnu-toolchain-12.2.mpacbti-rel1-mingw-w64-i686-arm-none-eabi/bin/../lib/gcc/arm-none-eabi/12.2.1/thumb/v8-m.main+fp/hard\libgcc.a(_arm_fixunsdfsi.o)
 .debug_frame   0x00002114       0x44 c:/renesas/ra/e2studio_v2023-07_fsp_v4.6.0/toolchains/gcc_arm/arm-gnu-toolchain-12.2.mpacbti-rel1-mingw-w64-i686-arm-none-eabi/bin/../lib/gcc/arm-none-eabi/12.2.1/thumb/v8-m.main+fp/hard\libgcc.a(_aeabi_ldivmod.o)
 .debug_frame   0x00002158       0x38 c:/renesas/ra/e2studio_v2023-07_fsp_v4.6.0/toolchains/gcc_arm/arm-gnu-toolchain-12.2.mpacbti-rel1-mingw-w64-i686-arm-none-eabi/bin/../lib/gcc/arm-none-eabi/12.2.1/thumb/v8-m.main+fp/hard\libgcc.a(_udivmoddi4.o)
 .debug_frame   0x00002190       0x38 c:/renesas/ra/e2studio_v2023-07_fsp_v4.6.0/toolchains/gcc_arm/arm-gnu-toolchain-12.2.mpacbti-rel1-mingw-w64-i686-arm-none-eabi/bin/../lib/gcc/arm-none-eabi/12.2.1/thumb/v8-m.main+fp/hard\libg_nano.a(libc_a-itoa.o)
 .debug_frame   0x000021c8       0x64 c:/renesas/ra/e2studio_v2023-07_fsp_v4.6.0/toolchains/gcc_arm/arm-gnu-toolchain-12.2.mpacbti-rel1-mingw-w64-i686-arm-none-eabi/bin/../lib/gcc/arm-none-eabi/12.2.1/thumb/v8-m.main+fp/hard\libg_nano.a(libc_a-strtol.o)
 .debug_frame   0x0000222c       0x48 c:/renesas/ra/e2studio_v2023-07_fsp_v4.6.0/toolchains/gcc_arm/arm-gnu-toolchain-12.2.mpacbti-rel1-mingw-w64-i686-arm-none-eabi/bin/../lib/gcc/arm-none-eabi/12.2.1/thumb/v8-m.main+fp/hard\libg_nano.a(libc_a-utoa.o)
 .debug_frame   0x00002274      0x144 c:/renesas/ra/e2studio_v2023-07_fsp_v4.6.0/toolchains/gcc_arm/arm-gnu-toolchain-12.2.mpacbti-rel1-mingw-w64-i686-arm-none-eabi/bin/../lib/gcc/arm-none-eabi/12.2.1/thumb/v8-m.main+fp/hard\libg_nano.a(libc_a-findfp.o)
 .debug_frame   0x000023b8       0x20 c:/renesas/ra/e2studio_v2023-07_fsp_v4.6.0/toolchains/gcc_arm/arm-gnu-toolchain-12.2.mpacbti-rel1-mingw-w64-i686-arm-none-eabi/bin/../lib/gcc/arm-none-eabi/12.2.1/thumb/v8-m.main+fp/hard\libg_nano.a(libc_a-memset.o)
 .debug_frame   0x000023d8       0x28 c:/renesas/ra/e2studio_v2023-07_fsp_v4.6.0/toolchains/gcc_arm/arm-gnu-toolchain-12.2.mpacbti-rel1-mingw-w64-i686-arm-none-eabi/bin/../lib/gcc/arm-none-eabi/12.2.1/thumb/v8-m.main+fp/hard\libg_nano.a(libc_a-strncmp.o)
 .debug_frame   0x00002400       0x20 c:/renesas/ra/e2studio_v2023-07_fsp_v4.6.0/toolchains/gcc_arm/arm-gnu-toolchain-12.2.mpacbti-rel1-mingw-w64-i686-arm-none-eabi/bin/../lib/gcc/arm-none-eabi/12.2.1/thumb/v8-m.main+fp/hard\libg_nano.a(libc_a-errno.o)
 .debug_frame   0x00002420       0x20 c:/renesas/ra/e2studio_v2023-07_fsp_v4.6.0/toolchains/gcc_arm/arm-gnu-toolchain-12.2.mpacbti-rel1-mingw-w64-i686-arm-none-eabi/bin/../lib/gcc/arm-none-eabi/12.2.1/thumb/v8-m.main+fp/hard\libg_nano.a(libc_a-strcpy.o)
 .debug_frame   0x00002440       0x20 c:/renesas/ra/e2studio_v2023-07_fsp_v4.6.0/toolchains/gcc_arm/arm-gnu-toolchain-12.2.mpacbti-rel1-mingw-w64-i686-arm-none-eabi/bin/../lib/gcc/arm-none-eabi/12.2.1/thumb/v8-m.main+fp/hard\libg_nano.a(libc_a-aeabi_memcpy.o)
 .debug_frame   0x00002460       0x20 c:/renesas/ra/e2studio_v2023-07_fsp_v4.6.0/toolchains/gcc_arm/arm-gnu-toolchain-12.2.mpacbti-rel1-mingw-w64-i686-arm-none-eabi/bin/../lib/gcc/arm-none-eabi/12.2.1/thumb/v8-m.main+fp/hard\libg_nano.a(libc_a-aeabi_memclr.o)
 .debug_frame   0x00002480       0x28 c:/renesas/ra/e2studio_v2023-07_fsp_v4.6.0/toolchains/gcc_arm/arm-gnu-toolchain-12.2.mpacbti-rel1-mingw-w64-i686-arm-none-eabi/bin/../lib/gcc/arm-none-eabi/12.2.1/thumb/v8-m.main+fp/hard\libg_nano.a(libc_a-memcpy-stub.o)

.debug_loclists
                0x00000000     0xefbd
 .debug_loclists
                0x00000000      0x39e ./src/angle.o
 .debug_loclists
                0x0000039e      0x2dc ./src/control_table.o
 .debug_loclists
                0x0000067a      0x64b ./src/hal_entry.o
 .debug_loclists
                0x00000cc5       0xcf ./src/interpolation.o
 .debug_loclists
                0x00000d94       0x9b ./src/monitor.o
 .debug_loclists
                0x00000e2f     0x2be6 ./src/packet.o
 .debug_loclists
                0x00003a15      0x268 ./src/pid.o
 .debug_loclists
                0x00003c7d       0x86 ./src/sintable.o
 .debug_loclists
                0x00003d03     0x180a ./src/usart.o
 .debug_loclists
                0x0000550d     0x1412 ./ra/fsp/src/r_sci_uart/r_sci_uart.o
 .debug_loclists
                0x0000691f     0x13df ./ra/fsp/src/r_sci_spi/r_sci_spi.o
 .debug_loclists
                0x00007cfe      0x9bf ./ra/fsp/src/r_sci_i2c/r_sci_i2c.o
 .debug_loclists
                0x000086bd      0xb5a ./ra/fsp/src/r_rtc/r_rtc.o
 .debug_loclists
                0x00009217      0x724 ./ra/fsp/src/r_ioport/r_ioport.o
 .debug_loclists
                0x0000993b     0x155f ./ra/fsp/src/r_gpt/r_gpt.o
 .debug_loclists
                0x0000ae9a     0x166e ./ra/fsp/src/r_flash_hp/r_flash_hp.o
 .debug_loclists
                0x0000c508      0x334 ./ra/fsp/src/r_dtc/r_dtc.o
 .debug_loclists
                0x0000c83c      0x447 ./ra/fsp/src/r_crc/r_crc.o
 .debug_loclists
                0x0000cc83      0xe56 ./ra/fsp/src/r_agt/r_agt.o
 .debug_loclists
                0x0000dad9      0xf8c ./ra/fsp/src/r_adc/r_adc.o
 .debug_loclists
                0x0000ea65      0x1ae ./ra/fsp/src/bsp/mcu/all/bsp_clocks.o
 .debug_loclists
                0x0000ec13       0x20 ./ra/fsp/src/bsp/mcu/all/bsp_common.o
 .debug_loclists
                0x0000ec33      0x110 ./ra/fsp/src/bsp/mcu/all/bsp_delay.o
 .debug_loclists
                0x0000ed43       0x62 ./ra/fsp/src/bsp/mcu/all/bsp_group_irq.o
 .debug_loclists
                0x0000eda5       0xbd ./ra/fsp/src/bsp/mcu/all/bsp_irq.o
 .debug_loclists
                0x0000ee62       0xa1 ./ra/fsp/src/bsp/mcu/all/bsp_register_protection.o
 .debug_loclists
                0x0000ef03       0xba ./ra/fsp/src/bsp/cmsis/Device/RENESAS/Source/system.o

.debug_line_str
                0x00000000      0x20b
 .debug_line_str
                0x00000000       0xe2 c:/renesas/ra/e2studio_v2023-07_fsp_v4.6.0/toolchains/gcc_arm/arm-gnu-toolchain-12.2.mpacbti-rel1-mingw-w64-i686-arm-none-eabi/bin/../lib/gcc/arm-none-eabi/12.2.1/thumb/v8-m.main+fp/hard\libgcc.a(_arm_addsubdf3.o)
 .debug_line_str
                0x000000e2       0xe2 c:/renesas/ra/e2studio_v2023-07_fsp_v4.6.0/toolchains/gcc_arm/arm-gnu-toolchain-12.2.mpacbti-rel1-mingw-w64-i686-arm-none-eabi/bin/../lib/gcc/arm-none-eabi/12.2.1/thumb/v8-m.main+fp/hard\libgcc.a(_arm_muldivdf3.o)
 .debug_line_str
                0x000000e2       0xe2 c:/renesas/ra/e2studio_v2023-07_fsp_v4.6.0/toolchains/gcc_arm/arm-gnu-toolchain-12.2.mpacbti-rel1-mingw-w64-i686-arm-none-eabi/bin/../lib/gcc/arm-none-eabi/12.2.1/thumb/v8-m.main+fp/hard\libgcc.a(_arm_cmpdf2.o)
 .debug_line_str
                0x000000e2       0xe2 c:/renesas/ra/e2studio_v2023-07_fsp_v4.6.0/toolchains/gcc_arm/arm-gnu-toolchain-12.2.mpacbti-rel1-mingw-w64-i686-arm-none-eabi/bin/../lib/gcc/arm-none-eabi/12.2.1/thumb/v8-m.main+fp/hard\libgcc.a(_arm_fixdfsi.o)
 .debug_line_str
                0x000000e2       0xe2 c:/renesas/ra/e2studio_v2023-07_fsp_v4.6.0/toolchains/gcc_arm/arm-gnu-toolchain-12.2.mpacbti-rel1-mingw-w64-i686-arm-none-eabi/bin/../lib/gcc/arm-none-eabi/12.2.1/thumb/v8-m.main+fp/hard\libgcc.a(_arm_fixunsdfsi.o)
 .debug_line_str
                0x000000e2        0x8 c:/renesas/ra/e2studio_v2023-07_fsp_v4.6.0/toolchains/gcc_arm/arm-gnu-toolchain-12.2.mpacbti-rel1-mingw-w64-i686-arm-none-eabi/bin/../lib/gcc/arm-none-eabi/12.2.1/thumb/v8-m.main+fp/hard\libgcc.a(_aeabi_ldivmod.o)
                                 0xdd (size before relaxing)
 .debug_line_str
                0x000000ea        0xc c:/renesas/ra/e2studio_v2023-07_fsp_v4.6.0/toolchains/gcc_arm/arm-gnu-toolchain-12.2.mpacbti-rel1-mingw-w64-i686-arm-none-eabi/bin/../lib/gcc/arm-none-eabi/12.2.1/thumb/v8-m.main+fp/hard\libgcc.a(_dvmd_tls.o)
                                 0xe1 (size before relaxing)
 .debug_line_str
                0x000000f6       0xff c:/renesas/ra/e2studio_v2023-07_fsp_v4.6.0/toolchains/gcc_arm/arm-gnu-toolchain-12.2.mpacbti-rel1-mingw-w64-i686-arm-none-eabi/bin/../lib/gcc/arm-none-eabi/12.2.1/thumb/v8-m.main+fp/hard\libg_nano.a(libc_a-strlen.o)
 .debug_line_str
                0x000001f5       0x16 c:/renesas/ra/e2studio_v2023-07_fsp_v4.6.0/toolchains/gcc_arm/arm-gnu-toolchain-12.2.mpacbti-rel1-mingw-w64-i686-arm-none-eabi/bin/../lib/gcc/arm-none-eabi/12.2.1/thumb/v8-m.main+fp/hard\libg_nano.a(libc_a-aeabi_memset-soft.o)
                                0x102 (size before relaxing)
